:020000040800F2
:10000000687D002029030008F9870008C96B0008F3
:10001000658600085D260008819A0008000000003F
:10002000000000000000000000000000690200085D
:10003000FB28000800000000C5020008618F0008CE
:100040004303000843030008430300084303000878
:100050004303000843030008FD2800084303000889
:10006000430300080729000811290008430300087A
:100070007D270008430300084303000843030008EA
:1000800043030008430300084303000881260008D7
:100090006126000871260008430300081B29000898
:1000A0004303000843030008430300084303000818
:1000B000430300084303000843030008DD6B000806
:1000C000CD6B000843030008430300084303000806
:1000D000430300084303000843030008519A000843
:1000E00043030008430300084303000843030008D8
:1000F00043030008430300084303000843030008C8
:1001000043030008430300084303000843030008B7
:100110004303000843030008430300083D90000820
:100120004303000843030008D1270008E127000823
:100130004303000843030008430300084303000887
:1001400091260008A1260008430300084303000885
:100150004303000843030008430300084303000867
:100160004303000843030008430300084303000857
:100170004303000843030008430300080000000095
:10018000430300084303000800F002F800F05CF8A5
:100190000AA090E8000C82448344AAF10107DA45E2
:1001A00001D100F051F8AFF2090EBAE80F0013F0D8
:1001B000010F18BFFB1A43F001031847ACEB000016
:1001C000CCEB00000A444FF0000C10F8013B13F098
:1001D000070408BF10F8014B1D1108BF10F8015BA0
:1001E000641E05D010F8016B641E01F8016BF9D193
:1001F00013F0080F1EBF10F8014BAD1C0C1B09D1EA
:100200006D1E58BF01F801CBFAD505E014F8016B5B
:1002100001F8016B6D1EF9D59142D6D370470000ED
:100220000023002400250026103A28BF78C1FBD8FF
:10023000520728BF30C148BF0B6070471FB50EF092
:1002400070FC1FBD10B510BD00F0E4F91146FFF7BA
:10025000F5FF0AF027FC00F002FA03B4FFF7F2FF03
:1002600003BC00F005FA00002C4B19680868B0E8E0
:10027000F04F80F30988BFF36F8F4FF0000080F3D9
:10028000118870470000000008480068006880F38B
:1002900008884FF0000080F3148862B661B6BFF39F
:1002A0004F8FBFF36F8F00DF00BF00BF08ED00E08E
:1002B000DFF80C00016841F470010160704700BF75
:1002C00088ED00E0EFF30980BFF36F8F134B1A68DE
:1002D0001EF0100F08BF20ED108A20E9F04F1060CB
:1002E00009B44FF0500080F31188BFF34F8FBFF374
:1002F0006F8F0CF0B3FA4FF0000080F3118809BC47
:1003000019680868B0E8F04F1EF0100F08BFB0EC95
:10031000108A80F30988BFF36F8F704718000020A0
:10032000EFF30580704700000948804709480047FF
:10033000FEE7FEE7FEE7FEE7FEE7FEE7FEE7FEE795
:10034000FEE7FEE704480549054A064B70470000F2
:10035000299000088901000868770020687D002046
:10036000687900206879002053EA020C00F0698067
:100370002DE9F04B4FF00006002B1FBFB3FA83F5B9
:1003800003FA05F424FA05F65E4012BF1643B2FAEA
:1003900082F502FA05F4C5F120051EBF22FA05FC1C
:1003A00044EA0C04203556EA044C4FEA144418BFC2
:1003B000641C4FF000084FF00009904271EB030CF1
:1003C00039D3002919BFB1FA81F701FA07F6B0FA5B
:1003D00080F700FA07F6C7F120071EBF20FA07FCD6
:1003E00046EA0C062037B6FBF4FCA7EB0507103FE6
:1003F00007F01F0BCBF120060CFA0BFB2CFA06F6CC
:1004000044BFB3460026202FA4BF5E464FF0000B2A
:100410005BEA060C08BF4FF0010B19EB0B09ABFBB5
:10042000027C48EB0608C01B06FB02CC0BFB03CC8E
:1004300071EB0C01C1E70B46024641464846BDE858
:10044000F08B13B54FF000004FF00001AFF30080C8
:10045000BDE81C407047032A40F2308010F0030CC6
:1004600000F0158011F8013BBCF1020F624498BF07
:1004700011F801CB00F8013B38BF11F8013BA2F1A4
:10048000040298BF00F801CB38BF00F8013B11F01F
:10049000030300F02580083AC0F0088051F8043BBF
:1004A000083A51F804CBA0E80810F5E7121D5CBF2C
:1004B00051F8043B40F8043BAFF30080D20724BF5F
:1004C00011F8013B11F801CB48BF11F8012B24BFF3
:1004D00000F8013B00F801CB48BF00F8012B704742
:1004E00010B5203AC0F00B80B1E81850203AA0E8CF
:1004F0001850B1E81850A0E81850BFF4F5AF5FEA03
:10050000027C24BFB1E81850A0E8185044BF18C9B5
:1005100018C0BDE810405FEA827C24BF51F8043B5C
:1005200040F8043B08BF7047D20728BF31F8023BB0
:1005300048BF11F8012B28BF20F8023B48BF00F844
:10054000012B704702F0FF0343EA032242EA024212
:1005500000F002B84FF000020429C0F0128010F041
:10056000030C00F01B80CCF1040CBCF1020F18BF8F
:1005700000F8012BA8BF20F8022BA1EB0C0100F022
:100580000DB85FEAC17C24BF00F8012B00F8012BF5
:1005900048BF00F8012B70474FF0000200B513462A
:1005A00094469646203922BFA0E80C50A0E80C5093
:1005B000B1F12001BFF4F7AF090728BFA0E80C5044
:1005C00048BF0CC05DF804EB890028BF40F8042B3D
:1005D00008BF704748BF20F8022B11F0804F18BFAA
:1005E00000F8012B704770477047704710B500F056
:1005F00009F8006810BD10B5044600F003F8046067
:1006000010BD000000487047047700200048704784
:10061000047700207546FFF7F9FFAE4605006946EE
:10062000534620F00700854618B020B5FFF78AFE34
:10063000BDE820404FF000064FF000074FF00008E3
:100640004FF0000B21F00701AC46ACE8C009ACE864
:10065000C009ACE8C009ACE8C0098D46704710B5C8
:100660000446AFF300802046BDE81040FFF7F5BD1B
:1006700001491820ABBEFEE72600020070470000CB
:1006800030B52DED068B81B005460C462DB94FF0E7
:10069000FF3001B0BDEC068B30BD14B94FF0FF3018
:1006A000F7E794ED000AD4ED010A20EE200AD4ED1C
:1006B000020A94ED031A00EE810AF0EE000A60EEE1
:1006C000208A94ED010A20EE000AD4ED020A94ED8E
:1006D000021A00EE810AF7EE000AB0EE001AB0EE40
:1006E000609A01EE409AF0EE490AB0EE680A09F00D
:1006F0001FFD85ED010A94ED000AD4ED020A20EEFB
:10070000200AD4ED030A94ED011A00EEC10AF0EEBE
:10071000000A20EE208AB0EEC80AF7EE000AB4EE16
:10072000E00AF1EE10FA0FDB9FED200A8DED000AD2
:1007300018EE100A0246009961F31E0200929DED28
:10074000000A85ED020A05E0B0EE480A09F0EEF96C
:1007500085ED020A94ED000AD4ED030A20EE200A8A
:10076000D4ED010A94ED021A00EE810AF0EE000ABF
:1007700060EE209A94ED020A20EE000AD4ED030AFE
:1007800094ED031A00EE810AF7EE000AB0EE001AAB
:10079000B0EE60AA01EE40AAF0EE4A0AB0EE690A95
:1007A00009F0C6FC85ED000A002072E7DB0FC93FA7
:1007B00070B52DED0A8B04460D46F0EE408A24B943
:1007C0004FF0FF30BDEC0A8B70BDB7EE000AC0EEF3
:1007D000280AC4ED040AB7EE000A84ED000A9FED72
:1007E0006D0A84ED010A9FED6B0A84ED020A9FED0C
:1007F000690A84ED030A002D7DD095ED000A10EE04
:10080000101A08460EF0B6F841EC1B0B95ED010AE4
:1008100010EE101A08460EF0ADF841EC1C0BB0EECD
:100820004B1AF0EE6B1AB0EE4C0AF0EE6C0A09F0BF
:100830007FFBB0EE40AAF0EE60AA51EC1A0B0DF06F
:1008400025FB41EC190B0DF02DFB08EE100A95ED80
:10085000000AB5EEC00AF1EE10FA1ED195ED010ABC
:10086000B5EEC00AF1EE10FA17D195ED020AB5EE19
:10087000C00AF1EE10FA10D19FED470A84ED000A8C
:100880009FED460A84ED010A9FED450A84ED020AB8
:100890009FED440A84ED030A78E09FED430AB4EE2D
:1008A000C08AF1EE10FA04D3B5EEC08AF1EE10FA68
:1008B00010DD9FED3E0A84ED000A9FED3D0A84EDB8
:1008C000010A9FED3C0A84ED020A9FED3B0A84ED8C
:1008D000030A5BE09FED390AB4EEC08AF1EE10FA2C
:1008E00006D39FED310AB4EEC08AF1EE10FA12DDA4
:1008F0009FED290A00E04AE084ED000A9FED270AF7
:1009000084ED010A9FED260A84ED020A9FED250A77
:1009100084ED030A3AE09FED2A0AB4EEC08AF1EEB4
:1009200010FA06D39FED250AB4EEC08AF1EE10FA54
:1009300010DD9FED190A84ED000A9FED180A84ED81
:10094000010A9FED170A84ED020A9FED160A84ED55
:10095000030A1BE09FED1A0AB4EEC08AF1EE10FA0A
:1009600004D3B5EEC08AF1EE10FA0FDD9FED0A0A4E
:1009700084ED000A9FED090A84ED010A9FED080A43
:1009800084ED020A9FED070A84ED030A00BF0020F0
:1009900018E7000000000000C5064D3F2D4A0D3C41
:1009A00056A439BBAD47193FDB0FC93F6E597F3F96
:1009B0000C53B039AB88BBBB8595973DDB0F4940E5
:1009C0000000B44200210160416081607047000076
:1009D000F0B52DED108B9DB004460D4616461F4612
:1009E0002CB94FF0FF301DB0BDEC108BF0BD15B928
:1009F0004FF0FF30F7E716B94FF0FF30F3E79FED08
:100A0000FE0AFE4880ED000A2FB9324629462046EC
:100A100000F07EFCE7E797ED00BA97ED019AD7ED7D
:100A2000029AB5EEC0BAF1EE10FA0FD1B5EEC09A47
:100A3000F1EE10FA0AD1F5EEC09AF1EE10FA05D1F6
:100A400032462946204600F063FCCCE7D5ED00EAAB
:100A5000D5ED01DA95ED02FA96ED000A8DED030A67
:100A600096ED010A8DED020A96ED020A8DED010A5E
:100A700094ED010AF1EE400A9DED030A20EE800A92
:100A800094ED021ADDED020A01EE600A94ED031AFC
:100A9000DDED010A01EE600AF6EE000A20EE200A02
:100AA0008DED190AD4ED000A9DED030A20EE800AAF
:100AB00094ED021ADDED010A01EE200A94ED031A0D
:100AC000DDED020A01EE600AF6EE000A20EE200AD1
:100AD0008DED180AD4ED000A9DED020A20EE800A81
:100AE00094ED011ADDED010A01EE600A94ED031A9E
:100AF000DDED030A01EE200AF6EE000A20EE200AE0
:100B00008DED170AD4ED000A9DED010A20EE800A52
:100B100094ED011ADDED020A01EE200A94ED021AAD
:100B2000DDED030A01EE600AF6EE000A20EE200A6F
:100B30008DED160AF5EEC0EAF1EE10FA09D1F5EEE8
:100B4000C0DAF1EE10FA04D1B5EEC0FAF1EE10FA07
:100B50007ED06EEEAE0A4DEEAD0A4FEE0F0AB0EE4D
:100B6000600A06F06DFFB0EE40AA2EEE8A0AF0EEA3
:100B700040EA2DEE8A0AF0EE40DA2FEE0A0AB0EED5
:100B800040FA6BEE0B0A49EE090A49EEA90AB0EEEB
:100B9000600A06F055FFB0EE40AA2BEE0A0AB0EE4E
:100BA00040BA29EE0A0AB0EE409A29EE8A0AF0EE1F
:100BB000409A94ED000AF0EE000A20EE200A20EEA2
:100BC0000B0A8DED130A94ED000AF0EE000A20EEF8
:100BD000200A20EE090A8DED120A94ED000AF0EECB
:100BE000000A20EE200A20EE290A8DED110A94ED6C
:100BF000010AF0EE000A20EE200A20EE0B0A8DED2D
:100C0000100A94ED000AF0EE000A20EE200A8DEDA5
:100C10000D0A94ED010AF0EE000A20EE200A8DED97
:100C20000C0A94ED020AF0EE000A20EE200A8DED87
:100C30000B0A94ED030AF0EE000A20EE200A8DED77
:100C40000A0A94ED000AF0EE000A20EE200A00E005
:100C5000FDE2D4ED020A20EE200A8DED090A94EDA2
:100C6000020AF0EE000A20EE200AD4ED030A20EE7C
:100C7000200A8DED080A94ED000A20EE000A8DEDA1
:100C8000070A94ED000AD4ED010A60EE20CA94ED43
:100C9000000AD4ED020A20EE20DA94ED000AD4ED29
:100CA000030A20EE200A8DED060A94ED010A20EEDB
:100CB00000CA94ED010AD4ED020A20EE200A8DED5F
:100CC000050A94ED010AD4ED030A60EE20BA94ED12
:100CD000020A60EE00AA94ED020AD4ED030A20EEA7
:100CE000200A8DED040A94ED030A20EE00EA9DED42
:100CF000070A6BEE000A94ED031A9DED120A40EE0E
:100D0000410A94ED021A9DED110A40EE010AB0EE7F
:100D1000600A0BEE0C0ADDED0C0A60EE890A94ED18
:100D2000021A00EE810ADDED0C0A60EEA90A94EDCC
:100D3000031A00EE810A0BEE6A0A0BEE4E0A8DEDE5
:100D4000150AD4ED030A9DED130A20EE800ADDEDAD
:100D5000070A09EE200A94ED011ADDED110A00EEF2
:100D6000C10A94ED021ADDED100A00EE810A09EEC7
:100D70004C0A09EE2A0ADDED0B0A60EEA90A94ED91
:100D8000031A00EE810A09EE4E0A8DED140ADDED1C
:100D9000150A20EEA01ADDED140A00EEA01AB0EE3E
:100DA000410A06F04DFEF7EE000A80EE808AD4ED8F
:100DB000020A9DED130AB1EE400A60EE800A94ED3E
:100DC000011A9DED120A40EE010A9DED070A49EE57
:100DD000800A94ED031A9DED100A40EE010A49EED7
:100DE000CC0A9DED0B0A20EE091AD4ED031AB0EEE1
:100DF000600A01EE210A03E09EEF273DB0000020CB
:100E000009EEEA0AF0EE408A49EE8E8AB0EE000A58
:100E100068EE000ACDED0F0AB0EE000A28EE800A57
:100E20008DED0E0A9DED090AF0EE000A10EEAB0AF8
:100E300070EE6E0A9DED0B0AB1EE400A20EE801AAC
:100E40009DED080AF0EE000A00EEAC0A70EE6D1A95
:100E5000DDED0C0AB0EE410A00EEA10AF6EE000A42
:100E600070EEEA0A70EECE0A60EE880A3BEECD1A0A
:100E700048EE810A70EECB0A94ED021A21EE281A90
:100E800001EE600AD4ED030AB1EE481A60EE811A51
:100E9000D4ED010A48EEA01ADDED050A9DED061A13
:100EA00070EEC10A20EE881ADDED040A7CEEA00A7D
:100EB00008EEA01A71EE490A01EEA00A7DEE2B0A97
:100EC00060EE880AB6EE001A31EE4C1A31EE6A1A5C
:100ED00048EE810A70EEE90A94ED021A21EE081A32
:100EE00001EE200A8DED1C0A9DED090AF0EE000AC4
:100EF00010EEAB0A70EE6E0A9DED0A0A60EE800AF3
:100F00009DED080AB0EE001A01EE2C0A30EE6D1AC3
:100F10009DED0D0A40EE010AB7EE000AB0EE001A90
:100F200001EE4C0AB0EE001A01EE6A0A30EE4F1ADA
:100F300094ED010AF1EE001A60EE211AB0EE600A9B
:100F400001EEC10AF6EE000A70EEEA0A70EECE0A71
:100F500060EE880A3BEECD1A48EE810A70EECB0AAD
:100F600094ED031A21EE281A01EE200AD4ED020AAC
:100F700060EE881AD4ED000A48EEA01ADDED050AED
:100F80009DED061A70EEC10A20EE881ADDED040A06
:100F90007CEEA00A08EEA01A71EE490A01EEA00A42
:100FA000D4ED030A20EE881AD4ED011ADDED0E0A05
:100FB00000EEE11A7DEE2B0A60EE880AF6EE001ACA
:100FC00071EECC1A71EEEA1A48EEA10A70EEE90A47
:100FD00001EE200AF0EE40FA9DED090AF0EE000A5B
:100FE00010EEAB0A70EE6E0A9DED0D0AB1EE400AEE
:100FF00060EE800A9DED080AB0EE001A01EE2C0AA0
:1010000030EE6D1A9DED0A0A40EE010AB7EE000AB5
:10101000B0EE001A01EE4C0AB0EE001A01EE6A0AB8
:1010200030EE4F1A94ED020AF1EE001A60EE211A2A
:10103000B0EE600A01EEC10A94ED021ADDED0F0A6E
:10104000F1EE600A61EE200A94ED001A48EEC10A42
:10105000B6EE001A31EE6A1A31EE4E1A21EE081A77
:101060007BEECD1A08EEA11A31EE4B1A00EE810A82
:10107000D4ED010A60EE881AD4ED030A48EEA01AF6
:10108000DDED050A9DED061A70EEC10A20EE881A04
:10109000DDED040A7CEEA00A08EEA01A71EE490A02
:1010A00001EEA00AD4ED000A20EE881AD4ED021A4F
:1010B000DDED0E0A00EEE11A7DEE2B0A60EE880AE5
:1010C000F6EE001A71EECC1A71EEEA1A48EEA10A99
:1010D00070EEE90A01EE200A8DED1B0A9DED090A6A
:1010E000F0EE000A10EEAB0A70EE6E0A9DED0C0AEF
:1010F00060EE800A9DED080AB0EE001A01EE2C0A9F
:1011000070EE6D1A9DED0B1AB0EE600A01EE210A29
:1011100094ED031ADDED0F0AF1EE600A61EE200A8C
:1011200094ED011A48EE810AB6EE001A31EE6A1A01
:1011300031EE4E1A21EE081A7BEECD1A08EEA11AF6
:1011400031EE4B1A00EE810AD4ED000AB1EE481AD6
:1011500020EE811AD4ED020A08EEA01ADDED050A90
:10116000DDED061A70EEE10A60EE881ADDED040A84
:101170007CEEA00A48EEA01A71EEC90A01EE200A20
:101180007DEE2B0A60EE880AB6EE001A31EE4C1A9C
:1011900031EE6A1A48EE810A70EEE90A94ED011AFE
:1011A00021EE081A01EE200A8DED1A0ADDED1C0A67
:1011B00060EEA00A4FEEAF0A9DED1B1A41EE010A48
:1011C0009DED1A1A41EE010AB0EE600A06F038FCF5
:1011D000B0EE40AA9DED1C0A20EE0A0A8DED1C0A15
:1011E0002FEE8A0AF0EE40FA9DED1B0A20EE0A0A65
:1011F0008DED1B0A9DED1A0A20EE0A0A8DED1A0AE2
:101200009DED190A414890ED001ADDED1C0A01EE32
:10121000600A8DED190A9DED180AD0ED000A00EE66
:10122000EF0A8DED180A9DED170A90ED001ADDED1D
:101230001B0A01EE600A8DED170A9DED160A90ED6E
:10124000001ADDED1A0A01EE600A8DED160AD4EDE2
:10125000000A94ED041A9DED190A40EE010AC4ED4E
:10126000000AD4ED010A94ED041A9DED180A40EE2F
:10127000010AC4ED010AD4ED020A94ED041A9DEDB1
:10128000170A40EE010AC4ED020AD4ED030A94EDF8
:10129000041A9DED160A40EE010AC4ED030AD4EDCE
:1012A000000A60EEA00A94ED011AD4ED011A41EE95
:1012B000210A94ED021AD4ED021A41EE210A94EDAE
:1012C000031AD4ED031A41EE210AB0EE600A06F0CB
:1012D000B7FBB0EE40AA94ED000A20EE0A0A84EDB6
:1012E000000A94ED010A20EE0A0A84ED010A94ED49
:1012F000020A20EE0A0A84ED020A94ED030A20EEA7
:101300000A0A84ED030A0020FFF76DBBB00000203D
:1013100070B52DED108B8CB004460D4616462CB9D9
:101320004FF0FF300CB0BDEC108B70BD15B94FF015
:10133000FF30F7E716B94FF0FF30F3E79FEDF30A00
:10134000F34880ED000A95ED009AD5ED018AD5EDC0
:10135000029A96ED00AAD6ED01AA96ED02BA94ED96
:10136000010AB1EE400A20EE0A0AD4ED020A00EEAC
:10137000EA0AD4ED030A00EECB0AF6EE000A20EEEC
:10138000200A8DED0B0A94ED000A20EE0A0AD4ED36
:10139000020A00EE8B0AD4ED030A00EEEA0AF6EE2A
:1013A000000A20EE200A8DED0A0A94ED000A20EED4
:1013B0002A0AD4ED010A00EECB0AD4ED030A00EEAE
:1013C0008A0AF6EE000A20EE200A8DED090A94ED55
:1013D000000A20EE0B0AD4ED010A00EEAA0AD4EDB1
:1013E000020A00EECA0AF6EE000A20EE200A8DED8F
:1013F000080AB5EEC09AF1EE10FA09D1F5EEC08AEE
:10140000F1EE10FA04D1F5EEC09AF1EE10FA7CD0AC
:1014100069EE090A48EEA80A49EEA90AB0EE600A88
:1014200006F00EFBB0EE408A29EE080AB0EE409AB4
:1014300028EE880AF0EE408A29EE880AF0EE409AFB
:1014400094ED000AF0EE000A20EE200A8DED070A66
:1014500094ED010AF0EE000A20EE200A8DED060A56
:1014600094ED020AF0EE000A20EE200A8DED050A46
:1014700094ED030AF0EE000A60EE20FA94ED000A03
:10148000F1EE000A20EE200A8DED040A94ED010A27
:10149000F1EE000A20EE20EA94ED020AF1EE000AD5
:1014A00060EE20EA94ED010AF2EE000A20EE200A36
:1014B0008DED030A94ED020AF2EE000A20EE200AF6
:1014C0008DED020A94ED000A20EE000A8DED010A6E
:1014D00094ED010A60EE00BA94ED020A20EE00CA13
:1014E00094ED030A20EE000A8DED000A9DED040A3A
:1014F00020EE0C0ADDED050A00EE890ADDED040A96
:1015000000EEAB0ADDED060A00E0A0E000EEE80A1E
:10151000B0EE40FA9DED000A2EEE000A0FEEC90A69
:10152000DDED010AB1EE001A60EE810A94ED011AB8
:1015300000EE810ADDED070A00EEE80A70EE4E0AC1
:101540009DED030A40EE2B0A9DED030A40EE0C0AC6
:101550004EEE290AF0EE60CA9DED010AF1EE000A96
:1015600020EE200AD4ED020A20EE200ADDED070A63
:1015700000EE890ADDED000A0EEEA00A0FEEE80A81
:1015800030EE6E0ADDED020A00EEAB0ADDED020A76
:1015900000EE8C0A0EEEA90AB0EE40DAB1EE000AB7
:1015A0002BEE800AD4ED030A20EE200ADDED060AB8
:1015B00000EEC90AF1EE000A6CEE200A94ED031A5F
:1015C00000EE810ADDED050A00EEE80AF0EE40DAF1
:1015D0006FEE0F0A4CEEAC0A4DEE0D0A4DEEAD0A61
:1015E000B0EE600A06F02CFAB0EE408A2FEE080A40
:1015F000B0EE40FA2CEE880AF0EE40CA2DEE080A52
:10160000B0EE40DA2DEE880AF0EE40DA9DED0B0ADE
:101610003F48D0ED000A00EECF0A8DED0B0A9DED9C
:101620000A0AD0ED000A00EEEC0A8DED0A0A9DEDE3
:10163000090AD0ED000A00EECD0A8DED090A9DEDF4
:10164000080AD0ED000A00EEED0A8DED080AD4ED8F
:10165000000A94ED041A9DED0B0A40EE010AC4ED58
:10166000000AD4ED010A94ED041A9DED0A0A40EE39
:10167000010AC4ED010AD4ED020A94ED041A9DEDAD
:10168000090A40EE010AC4ED020AD4ED030A94ED02
:10169000041A9DED080A40EE010AC4ED030AD4EDD8
:1016A000000A60EEA00A94ED011AD4ED011A41EE91
:1016B000210A94ED021AD4ED021A41EE210A94EDAA
:1016C000031AD4ED031A41EE210AB0EE600A06F0C7
:1016D000B7F9B0EE408A94ED000A20EE080A84EDD6
:1016E000000A94ED010A20EE080A84ED010A94ED47
:1016F000020A20EE080A84ED020A94ED030A20EEA5
:10170000080A84ED030A00200CE60000022B073DC6
:10171000B0000020B0EE401AB1EE600AB4EEC01A7C
:10172000F1EE10FA02D2B1EE600A7047B4EEE01AA0
:10173000F1EE10FA02DDB0EE600AF6E7B0EE410A13
:10174000F3E7000010B504210248006809F046FCE8
:1017500010BD0000C000002010B51323034A122161
:10176000002000F0D5F9002010BD0000AC7300206F
:1017700010B54FF0FF320121084609F06FFC10BD93
:101780009FED010A704700000000C84310B5082112
:101790000248006809F022FC10BD0000C0000020D3
:1017A00010B50623034A0221012000F0B1F9002000
:1017B00010BD0000B373002010B54FF0FF320121BF
:1017C000022009F04BFC10BD70B504460D4614B95B
:1017D0006FF0010070BD15B96FF00100FAE74448E1
:1017E000007810B16FF00200F4E709F090FC414975
:1017F000086010B96FF00100ECE7E562B6227E21C7
:10180000002000F0EBF9B6221421012000F0E6F9E7
:101810001E2000F07BFE1E21002000F0A5F9002113
:10182000084600F0A1F91E2802D06FF00300D1E7AE
:101830000021012000F098F90F2802D06FF003007A
:10184000C8E7032000F0F6FC042000F0F3FC2A4A6D
:101850000121002000F022FE2849032000F040FD75
:101860002749042000F03CFDAA224021002000F07E
:10187000B5F901224121002000F0B0F908225321DE
:10188000002000F0ABF904225821002000F0A6F956
:1018900004227D21002000F0A1F9322000F036FE64
:1018A00001220F21104600F099F903221021012096
:1018B00000F094F900221621012000F08FF9012296
:1018C0001821104600F08AF980221521012000F02D
:1018D00085F90A2000F01AFE01200549087003204E
:1018E00000F0C8FC042000F0C5FC002072E70000F6
:1018F000C4000020C0000020C51A000845170008D9
:101900008D1700080EB5014611B96FF001000EBD2C
:101910002B48B0F8010002902948B0F8030001906C
:101920002748B0F805000090BDF9080000EE100A45
:10193000B8EEC00A81ED040ABDF9040000EE100AF9
:10194000B8EEC00A81ED050ABDF9000000EE100AEC
:10195000B8EEC00A81ED060A91ED040ADFED190A1E
:1019600080EE201A81ED041A91ED050ADFED150ACB
:1019700080EE201A81ED051A91ED060ADFED110ABD
:1019800080EE201A81ED061A0D48407CC0000C4BF9
:101990009B7C40EA6312B2F5806F02DBA2F5006027
:1019A00002B200EE102AF8EEC00AB4EE001AB3EE4E
:1019B000070A00EE810A81ED0A0A0020A7E700006D
:1019C000AC73002000A0AA450EB5014611B96FF016
:1019D00001000EBD3848B0F8070002903648B0F854
:1019E000090001903448B0F80B000090BDF90800E0
:1019F00000EE100AB8EEC00A81ED070ABDF9040036
:101A000000EE100AB8EEC00A81ED080ABDF9000028
:101A100000EE100AB8EEC00A81ED090A91ED070A3E
:101A2000DFED260A80EE201A81ED071A91ED080AF3
:101A3000DFED220A80EE201A81ED081A91ED090AE5
:101A4000DFED1E0A80EE201A81ED091A91ED070ADA
:101A5000DFED1B0A20EE200A81ED070A91ED080A4E
:101A6000DFED170A20EE200A81ED080A91ED090A40
:101A7000DFED130A20EE200A81ED090A91ED070A35
:101A8000C86AD0ED000A30EE600A81ED070A91EDD8
:101A9000080AC86AD0ED010A30EE600A81ED080A32
:101AA00091ED090AC86AD0ED020A30EE600A81EDB4
:101AB000090A6FF001008CE7AC7300206F1203423B
:101AC00035FA8E3C10B5012000F0F4FB40B901213D
:101AD000084600F029FC01210848006809F07EFA58
:101AE000022000F0E7FB40B90121022000F01CFCBD
:101AF00002210248006809F071FA10BDC000002000
:101B000010B54FF0FF3201210C2009F0A7FA10BDEB
:101B10002DE9F04105460E4614461F460CB9BDE8B6
:101B2000F08115B1012D0AD104E00021012000F05F
:101B3000FBFB04E00021022000F0F6FB00BF00BF29
:101B400046F080000749087000230122184600F083
:101B5000B3FC01233A462146002000F075FC00BF8B
:101B6000DDE70000BC00002070B504460D460120F2
:101B700000F0CCFC14B1012C0AD104E000210120BA
:101B800000F0D2FB04E00021022000F0CDFB00BFFA
:101B900000BF45F08000104908700023012218465C
:101BA00000F08AFC002302220B49184600F04CFC8E
:101BB00014B1012C0ED106E00121084600F0B4FB5F
:101BC0000548407870BD0121022000F0ADFB0248BD
:101BD0000078F7E700BFF5E7BC00002070B50446C9
:101BE0000E46154606F07F001549087008464570F8
:101BF000012000F08BFC14B1012C0AD104E000217B
:101C0000012000F091FB04E00021022000F08CFB99
:101C100000BF00BF002302220949184600F04CFC17
:101C200014B1012C0AD104E00121084600F07CFB2C
:101C300004E00121022000F077FB00BF00BF70BD6F
:101C4000BC0000202DE9F04107468846164606B93B
:101C50000A2664212348006809F00EF918B16FF0D4
:101C60000400BDE8F081204805680DE02878B842FE
:101C700009D16868404506D11A48006809F086F91C
:101C80004FF0FF30EDE72D69002DEFD1142000F06B
:101C900061FB04462CB91348006809F077F9A81EC7
:101CA000DFE700221C21304609F042F8A060A0685E
:101CB00048B9204600F0B8FA0A48006809F066F909
:101CC0004FF0FF30CDE72770C4F804802673064834
:101CD00000682061044804600248006809F056F971
:101CE0000020BEE7A4000020A000002070470000F4
:101CF00002460B460748016808E00878904204D184
:101D00004868984201D18868704709690029F4D170
:101D10000020F9E7A00000200146C868022806D18B
:101D20008868042801D1032070470220FCE78868F6
:101D3000042801D10120F7E70020F5E70146022938
:101D400001DB0020704711B1012904D101E00348F3
:101D5000F8E70348F6E70020F4E700008C010020D4
:101D6000B40100202DE9F0470746884614469946FD
:101D70001648007818B96FF00200BDE8F08714B972
:101D80006FF00100F9E764211148006809F074F868
:101D900010B16FF00400F0E741463846FFF7A8FFA6
:101DA00005460B48006809F0F1F815B96FF003001B
:101DB000E3E74B4600222146284608F079FF064615
:101DC0000EB90020D9E74FF0FF30D6E7A800002079
:101DD000A400002000B58BB02C48007818B16FF03B
:101DE00002000BB000BD68212948FEF7D5FB294849
:101DF00029490860002009F070F828490860084661
:101E0000006810B94FF0FF30EBE701201F49087060
:101E1000282101A8FEF7C0FB002006900190029047
:101E20000790012008900020039004900120099061
:101E30000E200A900020059001A9194801F09AF897
:101E4000174801F07DFD174A0621002000F044F8F4
:101E50000321134800F0D4FF0E20069001200590C6
:101E600001A9114801F086F80F4801F069FD0F4AF9
:101E70000821012000F030F810210B4800F0C0FFCD
:101E80000120024908700020ABE70000A8000020F4
:101E900058720020ED1C0008AC000020A4000020B7
:101EA0008C010020491F0008B4010020F91F000820
:101EB00070B504460D460748006828B129462046FB
:101EC000044A1268904770BD29462046FFF70EFF6E
:101ED000F9E70000AC00002010B503460F48007879
:101EE00010B96FF0020010BD12B96FF00100FAE7EF
:101EF000022B02DB4FF0FF30F5E70D2902DB4FF03C
:101F0000FF30F0E703EB830000EBC300044C04EB6D
:101F1000800040F821200020E5E70000A800002014
:101F20005872002070B504460D46164605480078E4
:101F300010B96FF0020070BD324629462046FFF707
:101F400081FEF8E7A80000202DE9F04391B00024BD
:101F50004DE0E0B2FFF7F2FE8046B8F1000F00D18D
:101F600044E03CE008AB0AAA0021404601F0C4F876
:101F7000002834D10C9808B90A9800E00B988146E3
:101F80000AA8FFF7C9FE054629464846FFF790FF15
:101F90000646E0B23146FFF7ABFE0746F7B11C211B
:101FA00001A8FEF7F9FA8DF80450CDF808900396D1
:101FB0000E98C0B28DF810000D9828B908A90DF13F
:101FC00011000E9AFEF747FA02F04AF90790002333
:101FD0001A4601A9384608F0F9FE00BF00BF0021EB
:101FE000404601F075F80028BCD100BF641C022CEB
:101FF000AFDB11B0BDE8F0832DE9F04391B00024D0
:102000004DE0E0B2FFF79AFE8046B8F1000F00D134
:1020100044E03CE008AB0AAA0121404601F06CF81C
:10202000002834D10C9808B90A9800E00B98814632
:102030000AA8FFF771FE054629464846FFF738FF14
:102040000646E0B23146FFF753FE0746F7B11C21C2
:1020500001A8FEF7A1FA8DF80450CDF80890039678
:102060000E98C0B28DF810000D9828B908A90DF18E
:1020700011000E9AFEF7EFF902F0F2F80790002334
:102080001A4601A9384608F0A1FE00BF00BF012191
:10209000404601F01DF80028BCD100BF641C022C92
:1020A000AFDB11B0BDE8F0832DE9F04788B0814681
:1020B0000D4614461E46DDF840A02F48007820B992
:1020C0006FF0020008B0BDE8F087B9F1020F02DB43
:1020D0004FF0FF30F6E736B9022D04D0032D02D0C1
:1020E0006FF00100EEE7BAF1080F02DD4FF0FF30AC
:1020F000E8E74846FFF722FE074617B96FF00100F0
:10210000E0E7182102A8FEF747FA35B1012D09D002
:10211000022D0DD0032D17D110E002940020049061
:10212000059014E0039404200490002005900EE034
:102130000294002004900220059008E003940420FB
:1021400004900220059002E04FF0FF30BAE700BF94
:10215000CDF818A000208DF81C0001AB324602A972
:10216000384600F062FE8046B8F1000F02D04FF012
:10217000FF30A7E70020A5E7A800002038B50546F6
:102180000C4614B96FF0010038BD20790090631D32
:10219000002128462268FFF787FFF5E72DE9F04781
:1021A00007460C461F48007818B96FF00200BDE8DA
:1021B000F087022F02DB4FF0FF30F8E73846FFF7D9
:1021C000BDFD054615B96FF00100F0E702F048F8D3
:1021D00006465CB9284601F059F88046B8F1000F70
:1021E00001D00020E3E76FF00400E0E718E02846A4
:1021F00001F04CF88046B8F1000F01D00020D6E77E
:10220000601C48B102F02CF8A0EB0609A14502D3EE
:102210006FF00400CBE700BF012008F072FC00BFA4
:10222000E5E70000A800002010B5044620460AF0AB
:102230001FF810BD10B5044634B1032C08D0042C8F
:102240000AD0052C10D10BE0062002F03FFC0EE076
:102250000A2002F03BFC0AE0172002F037FC06E0FF
:10226000092002F033FC02E04FF0FF3010BD00BF48
:102270000020FBE710B5044634B1032C08D0042C31
:102280000AD0052C10D10BE0062002F035FC0EE040
:102290000A2002F031FC0AE0172002F02DFC06E0D3
:1022A000092002F029FC02E04FF0FF3010BD00BF12
:1022B0000020FBE710B50446072C01DB002010BD11
:1022C000064A32F8341002EBC402506801F0BAFF3B
:1022D000012800D1F3E70020F1E700007CEB0008C3
:1022E00010B5024611B96FF0010010BD072A02DBDC
:1022F0004FF0FF30F9E70A4830F83230002009E0AB
:10230000012484401C401CB1064C44F8201003E01A
:10231000441CE0B21028F3DB00BF0020E5E700001A
:102320007CEB0008C072002070B504460D46072CF7
:1023300002DB4FF0FF3070BD054A32F8341002EB7B
:10234000C40250682A4601F085FF0020F3E7000030
:102350007CEB000810B50446204609F087FC10BD50
:102360000146012902DB4FF0FF307047F7EE000A0B
:10237000B4EEE00AF1EE10FA03DDF7EE000AB0EE7B
:10238000600AB5EEC00AF1EE10FA03D2DFED1E0AC4
:10239000B0EE600A1D4850F831000068C36A581C4E
:1023A00000EE900AF8EE600A60EE200AFCEEE00A09
:1023B00010EE902A154800EBC100808828B9134818
:1023C00050F83100006842631CE0104800EBC10087
:1023D0008088042805D10D4850F8310000688263D8
:1023E00010E00A4800EBC1008088082805D10748A2
:1023F00050F831000068C26304E0044850F831002E
:10240000006802640020B0E700000000B4EB0008A0
:1024100010B50446012C02DB4FF0FF3010BD054A19
:1024200002EBC4029188034A52F8340004F068F8C1
:102430000020F3E7B4EB0008014609B901487047F2
:102440000020FCE7840200202DE9F04105460F46FC
:1024500090461E46022D03DB4FF0FF30BDE8F081B1
:102460002846FFF7E9FF044614B94FF0FF30F5E7BF
:102470004EB142463946204603F05AF908B10120D0
:10248000ECE70020EAE7142342463946204603F0F1
:102490008DF808B10120E1E70020DFE7034612B91B
:1024A0006FF001007047034800EB431040F8212013
:1024B0000020F7E7487300202DE9F04105460F465C
:1024C00090461E46022D03DB4FF0FF30BDE8F08141
:1024D0002846FFF7B1FF044614B94FF0FF30F5E787
:1024E0004EB142463946204603F09CFC08B101201B
:1024F000ECE70020EAE7142342463946204603F081
:10250000DBF908B10120E1E70020DFE770B5044600
:1025100008F047FB4FF47A71B1FBF0F5B4FBF5F628
:1025200008F018FB022816D006DCB0F1FF3F0CD0F3
:10253000C8B101281CD117E0032808D0042807D00F
:102540006FF00041401A13D100E000BF00BF00BF90
:102550004FF0FF3070BD0EB1314600E0012108465A
:1025600008F0CFFA04E000BF204601F037FD00BFBD
:1025700000BF0020EEE72DE9F04108F012FB054610
:102580000BF092F94FF47A71B1FBF5F100FB01F613
:102590004FF0E02087690BF087F94FF47A71B1FBB7
:1025A000F5F100FB01F44FF0E020D0F81880A642CE
:1025B00014D14FF47A7078434FF0E0214969491CF7
:1025C000B0FBF1F004EB4401C1EBC4114FF47A729B
:1025D00002EBC101081A0021BDE8F0814FF47A70C6
:1025E00008FB00F04FF0E0214969491CB0FBF1F015
:1025F00004EB4401C1EBC4114FF47A7202EBC10148
:10260000081A0021E8E7000038B504462068006891
:1026100000F0100010281ED100BF0020009020689C
:102620000068009020684068009000BF00BF20460E
:1026300007F03EF800EBC000074901EB8000006A9C
:1026400048B1204607F034F800EBC000024901EB26
:102650008000056AA84738BD8873002000BFFEE7E8
:1026600010B5024800F02DFE10BD00008C010020C6
:1026700010B5024800F025FE10BD00008C010020BE
:1026800010B5024800F01DFE10BD00008C010020B6
:1026900010B5024800F015FE10BD0000B401002086
:1026A00010B5024800F00DFE10BD0000B40100207E
:1026B000014609B903207047064A0868904201D1D3
:1026C0000020F8E7044A0868904201D10120F2E7AF
:1026D0000320F0E70064004000680040B0EE401ABC
:1026E000D0ED001A71EE811AB0EE610AF5EEC00A63
:1026F000F1EE10FA12DDB4EEE00AF1EE10FA04DBAE
:1027000070EE601AB0EE610A08E0B5EEC00AF1EEB4
:1027100010FA03D270EE201AB0EE610A80ED000AC2
:102720007047F0EE401A31EEE02AB0EE420AB5EE04
:10273000C01AF1EE10FA1BDDF0EE002A81EE223A0B
:10274000B0EE432AB4EEC20AF1EE10FA04DD70EEE8
:10275000412AB0EE620A0AE0F1EE422AB4EEE20A41
:10276000F1EE10FA03D270EE012AB0EE620A00BF59
:102770007047000000487047E400002010B500F0EA
:1027800007F8024801F04AFA10BD000014050020C5
:1027900010B50C48006800F4006088B10A48007861
:1027A0000F2803D0192006F0C3F903E007490648B3
:1027B00009F074FB0348806840F4006001498860B8
:1027C00010BD000000600240D7730020BF730020DE
:1027D00010B5024801F022FA10BD000034030020B9
:1027E00010B5024801F01AFA10BD00009403002051
:1027F0000146087810381823B0FBF3F20848805CD3
:10280000C865032A05D908686FF30900001D8865AB
:1028100003E008686FF309008865886D7047000061
:102820005CEB0008014600208A6A8B69CBB932B1A3
:10283000012A0DD0022A03D0032A10D10EE000BFD6
:10284000CB6A03F08073B3F1807F00D1012007E0F1
:10285000CB6AB3F1C07F00D1012001E000E000BFEE
:1028600034E08B69B3F5005F1AD132B1012A07D089
:10287000022A03D0032A11D10AE000BF01200EE092
:10288000CB6A03F08073B3F1807F00D1012006E0B2
:10289000CB6AB3F1C07F00D1012000E000BF15E09A
:1028A00032B1012A05D0022A04D0032A0CD103E058
:1028B00000BF00BF012008E0CB6A03F08073B3F1D2
:1028C000807F00D1012000E000BF00BF704730B51D
:1028D0000468246824F4802405682C60046863601C
:1028E0008468402C04D10468A2600468E16003E0BD
:1028F0000468A1600468E26030BD704710B5012033
:1029000001F098FB10BD10B5082001F093FB10BD3D
:1029100010B5102001F08EFB10BD10B5202001F085
:1029200089FB10BD72B600BFFEE700002DE9F04143
:102930002DED088B04460D4604B12DB94FF0FF3044
:10294000BDEC088BBDE8F081FFF715FED4E900234C
:10295000861A61EB030130460CF06DF800EE100AA8
:10296000DFED910A80EE201A84ED021AFFF703FED4
:10297000C4E900012978204600F0C8F995ED010A64
:10298000D4ED020A20EE209ADFED880AB0EE490A63
:1029900004F11400FFF7A2FE94ED050ADFED840AAE
:1029A000B4EEE00AF1EE10FA07DD94ED050ADFED72
:1029B0007F0A30EE600A84ED050A95ED020AD4ED37
:1029C000020A60EE208AE06890ED290AB5EEC00A9E
:1029D000F1EE10FA4EDD94ED640AD4ED5E0A30EEAD
:1029E000600AB0EE408A9FED720AB4EEC08AF1EE42
:1029F00010FA05DD9FED6D0A38EE400AB0EE408A10
:102A00009FED6C0AB4EEC08AF1EE10FA05D29FED8C
:102A1000670A38EE000AB0EE408A9FED670A84ED3F
:102A2000460A9FED660A84ED470A94ED061A31EED8
:102A3000081A31EE281AF0EE410A94ED461AB0EE6B
:102A4000410A9FED5A1AFFF76CFEB0EE40BA94EDC2
:102A5000061A31EE081A31EE281AF0EE410A94ED0A
:102A6000471AB0EE410A9FED511AFFF75AFEF0EEF9
:102A700040AA00BF94ED060A30EE280A84ED060A4B
:102A800094ED060A10EE101A08460BF073FF41ECA5
:102A90001B0B9FED4B0B53EC102B0BF03FFE03D2A7
:102AA0009FED450A84ED060A94ED060A10EE101A11
:102AB00008460BF05FFF41EC1B0B9FED430B53EC03
:102AC000102B0BF0F1FC03D29FED3C0A84ED060ABB
:102AD000207C10B1012864D10AE09FED3D0A84ED0D
:102AE000580A9FED3B0A04F5B07084ED590A58E08E
:102AF00094ED021AF0EE411A94ED5D1AF0EE410ADF
:102B000094ED051AB0EE410A9FED311A04F1200050
:102B100005F074FEF0EE409A2E4880ED000A94ED28
:102B2000020AF0EE401A94ED5C0AF0EE400A9FEDC6
:102B3000281AB0EE690A04F15C0005F05FFE84ED2E
:102B4000580A254880ED000A94ED021AF0EE411A69
:102B500094ED5E1AF0EE410A94ED061AB0EE410AC9
:102B60009FED1B1A04F1980005F048FEB0EE40AA54
:102B70001A4880ED000A94ED020AF0EE401A94ED36
:102B80005A0AF0EE400A9FED121AB0EE4A0A04F11A
:102B9000D40005F033FE84ED590A114880ED000A97
:102BA00000BF00BF00BFCBE600247449DB0FC94063
:102BB000DB0F4940DB0F49C0D7A3F03E1F852BBF79
:102BC00014AE47E17A14DE3F713D0AD7A370E5BF2A
:102BD00000000000D8000020DC000020D000002011
:102BE000D400002070B52DED028B04460D46B0EEEA
:102BF000408A24B94FF0FF30BDEC028B70BDE56018
:102C000000202074E06800F13002B0EE480A012193
:102C100004F1200005F0C4FEE06800F11002B0EEFF
:102C2000480A012104F15C0005F0BAFEE06800F1F9
:102C30007002B0EE480A012104F1980005F0B0FEE0
:102C4000E06800F15002B0EE480A012104F1D4001E
:102C500005F0A6FEE06890ED240AF0EE400AB0EE22
:102C6000480A04F5907004F053FFE06890ED240AE0
:102C7000F0EE400AB0EE480A04F5A07004F048FFF8
:102C8000E06890ED260AD0ED280A30EE200A84EDA7
:102C9000440AE06890ED260A84ED450AE06890ED6C
:102CA000270AD0ED290A30EE200A84ED460AE068B2
:102CB00090ED270A84ED470AFFF78CF8E16801F1EF
:102CC000080005F011F9E06805F00EF9002093E71F
:102CD00010B50446D4ED580AB0EE600AE16801F17F
:102CE000080005F061F9D4ED590AF1EE600AB0EE82
:102CF000600AE06805F058F9E06804F0EBFFE1686D
:102D000001F1080004F0E6FF10BD000070B50446B4
:102D10000D4614B94FF0FF3070BD207CA84201D1A0
:102D20000020F9E704F1200005F0A0FE04F15C00AA
:102D300005F09CFE04F1980005F098FE04F1D40023
:102D400005F094FE9FED0D0A04F5907004F06AFF03
:102D50009FED0A0A04F5A07004F064FF04F114006A
:102D6000FDF730FE94ED5E0A84ED060A94ED5D0AEF
:102D700084ED050A25740020CEE700000000000065
:102D80002DE9F04104461CB94FF0FF30BDE8F08159
:102D9000E16801F1080005F060F9E06805F05DF90F
:102DA000E16801F1080005F06CF80646E06805F0FE
:102DB00068F8054605B966B104F5B47006F1080176
:102DC0008EC918308EC0283805F108018EC9283008
:102DD0008EC00020DAE730B5024612B94FF0FF305E
:102DE00030BD02F5807091E83800683038C00C388A
:102DF000D1E90445CB68C0E90445C36000BFEFE7F3
:102E000010B5024692F82030012B01D0022B06D1DA
:102E100010684069084314686061002010BD506A62
:102E200040F4802050620120F8E7F0B504460D46DA
:102E30001E4694F8207020688368A86800B900E0F6
:102E400000BF012F01D0022F7DD103F0806030B987
:102E500003F0006018B903F0805000287ED0C3F35F
:102E60000161012088403060A86860B9B5F800C0F1
:102E7000E86840EA4C5C206800F5C07000EB011087
:102E8000C0F800C00FE0D5E901C040EACC00D5F899
:102E90000CC040EA0C00D4F800C00CF5C07C0CEB70
:102EA000011CCCF80000D5F810C0206800F5C070F7
:102EB00000EB0110C0F804C0287D01280ED1206865
:102EC00000F5C07000EB0110406840F4807C206881
:102ED00000F5C07000EB0110C0F804C0D079000606
:102EE00092F806C040EA0C4092F805C040EA0C2077
:102EF00092F804C040EA0C00D4F800C00CF5C07C85
:102F00000CEB011CCCF80C00D078000692F802C043
:102F100040EA0C4092F801C040EA0C2092F800C050
:102F200040EA0C00D4F800C00CF5C07C0CEB011C8E
:102F3000CCF80800206800F5C07000EB01100068B4
:102F400040F0010C01E00FE008E0206800F5C070DF
:102F500000EB0110C0F800C00020F0BD606A40F432
:102F6000001060620120F8E7606A40F4802060622F
:102F70000120F2E7F0B504460A4694F82050012DEE
:102F800001D0022D7ED1424901F50071086840F060
:102F900001000860086820F47C5008600868566AE0
:102FA00040EA06200860107D00F01F06012000FAAC
:102FB00006F3C8699843C861A1F50071D069C8B922
:102FC000D1F80C029843C1F80C02908880B296891F
:102FD00040EA064601F51070576940F837601088DE
:102FE00080B2168940EA064601F51070576900EB79
:102FF000C7004660D069012819D1D1F80C021843E6
:10300000C1F80C02908880B2168840EA064601F5A5
:103010001070576940F83760908980B2168940EA8D
:10302000064601F51070576900EBC70046609069CD
:1030300028B9D1F804029843C1F8040204E0D1F899
:1030400004021843C1F80402106928B9D1F8140227
:103050009843C1F8140204E0D1F814021843C1F8EF
:103060001402106A012804D1D1F81C021843C1F8D7
:103070001C02D1F8000220F00100C1F8000200207B
:10308000F0BDFFE7606A40F4802060620120F7E74E
:103090000064004070B505462846FFF709FB04466A
:1030A000032C11D004EB840000EBC400074901EBB2
:1030B0008000006B40B104EB840101EBC401034AC2
:1030C00002EB8101086B804770BD00005872002040
:1030D00010B50246002092F82030012B01D0022BBF
:1030E00009D121B91468E46804F0030003E014680E
:1030F000246904F0030010BD70B5044694F8205014
:10310000012D01D0022D7DD151B92068C06800F099
:10311000030080B9606A40F400106062012070BD55
:103120002068006900F0030028B9606A40F40010CC
:1031300060620120F3E7206800F5D87000EB011011
:10314000006800F004009060906840B9206800F5C5
:10315000D87000EB01100068400D106007E0206897
:1031600000F5D87000EB01100068C00850602068BE
:1031700000F5D87000EB0110006800F00200D0608C
:10318000206800F5D87000EB0110406800F00F00D7
:10319000082802D30820106108E0206800F5D870E4
:1031A00000EB0110406800F00F001061206800F58E
:1031B000D87000EB0110406800F47F40000A906175
:1031C000206800F5D87000EB01104068000C5061D9
:1031D000206800F5D87000EB011080681870206836
:1031E00000F5D87000EB0110806800F47F40000A01
:1031F0005870206800F5D87000EB0110806800F46A
:103200007F0000E03CE0000C9870206800F5D8706A
:1032100000EB01108068000ED870206800F5D870AF
:1032200000EB0110C0681871206800F5D87000EB41
:103230000110C06800F47F40000A5871206800F552
:10324000D87000EB0110C06800F47F00000C98718A
:10325000206800F5D87000EB0110C068000ED8712E
:1032600031B92068C06840F020002668F06005E0B1
:103270002068006940F020002668306100204EE799
:10328000606A40F480206062012048E70146002027
:1032900091F82020012A01D0022A11D10B689B68E5
:1032A00003F0806303B1401C0B689B6803F000636C
:1032B00003B1401C0B689B6803F0805303B1401CB2
:1032C00070472DE9F05F04460025206846692068B4
:1032D000D0F80490206887682068D0F80CA0206897
:1032E000D0F810B02068D0F8188006F0010000284F
:1032F00055D007F00100C0B101202168886007F0B7
:10330000020018B1204600F069FB0EE007F004004F
:1033100010B145F4006508E007F0080010B145F46D
:10332000805502E0204600F03BFB07F48070C8B1F6
:103330004FF480702168886007F4007018B120464F
:1033400000F086FB0EE007F4806010B145F40055F4
:1033500008E007F4006010B145F4804502E0204623
:1033600000F058FB07F48030C8B14FF4803021687A
:10337000886007F4003018B1204600F0A5FB0EE08D
:1033800007F4802010B145F4004508E007F4002060
:1033900010B145F4803502E0204600F077FB06F0DE
:1033A000080038B10AF0100020B145F40075102073
:1033B0002168C86006F0040040B10AF0080028B196
:1033C00008202168C860204600F024FA06F00200B8
:1033D00038B12068C06800F0030010B1204600F04A
:1033E00037FA06F0400038B10BF0100020B145F478
:1033F000806510202168086106F0200040B10BF0C4
:10340000080028B1082021680861204600F03EFA33
:1034100006F0100038B12068006900F0030010B118
:10342000204600F051FA06F4003040B109F01000D7
:1034300028B1102021684860204600F063FA06F4A5
:10344000803040B109F0080028B1082021684860A8
:10345000204600F057FB06F4004088B309F0040052
:1034600078B306F4807020B108F0010008B145F08F
:10347000010506F4007020B108F0020008B145F023
:10348000020506F4806020B108F0040008B145F0A0
:10349000040506F40060A0B108F0700088B108F0DF
:1034A0007000402817D006DC10280BD020280CD044
:1034B000302819D10CE0502810D0602814D110E029
:1034C0001DE019E045F008050FE045F010050CE09F
:1034D00045F0200509E045F0400506E045F080058F
:1034E00003E045F4807500E000BF00BF20688069FC
:1034F00020F07000216888610420216848602DB1A7
:10350000606A284360622046FFF7C4FDBDE8F09F73
:1035100070B504460CB9012070BD94F8200010B9B4
:10352000204600F0AFF82068006840F001002168F4
:10353000086000F095FE05460DE000F091FE401B8E
:103540000A2808D9606A40F400306062052084F8D7
:1035500020000120E0E72068406800F0010000281A
:10356000EBD02068006820F002002168086000F0BD
:1035700077FE05460DE000F073FE401B0A2808D9CF
:10358000606A40F400306062052084F82000012069
:10359000C2E72068406800F002000028EBD1207EDE
:1035A000012806D12068006840F08000216808608A
:1035B00005E02068006820F0800021680860607ED7
:1035C000012806D12068006840F0400021680860AA
:1035D00005E02068006820F0400021680860A07EB7
:1035E000012806D12068006840F0200021680860AA
:1035F00005E02068006820F0200021680860E07E77
:10360000012806D12068006820F0100021680860B9
:1036100005E02068006840F0100021680860207F05
:10362000012806D12068006840F008002168086081
:1036300005E02068006820F0080021680860607FCD
:10364000012806D12068006840F004002168086065
:1036500005E02068006820F0040021680860D4E9D3
:103660000201084321690843616908436168491EF2
:1036700008432168C86100206062012084F82000AE
:10368000002049E710B586B00446142101A8FCF7D4
:1036900083FF5A492068884251D159480068401C2C
:1036A000574908600846006801280FD100BF002074
:1036B00000905448006840F0007052490860084685
:1036C000006800F00070009000BF00BF00BF002045
:1036D00000904C481038006840F008004949103903
:1036E00008600846006800F00800009000BF00BFB6
:1036F00003200190022002900020039003200490F8
:103700000920059001A9404800F0A2FC00220521F3
:10371000132001F005FA132001F0EEF90022052133
:10372000142001F0FDF9142001F0E6F90022052132
:10373000152001F0F5F9152001F0DEF95CE03349C0
:103740002068884258D100BF002000902D480068B2
:1037500040F080602B4908600846006800F08060F7
:10376000009000BF00BF26480068401C2449086044
:103770000846006801280FD100BF002000902148B2
:10378000006840F000701F4908600846006800F0BB
:103790000070009000BF00BF00BF002000901948DB
:1037A0001038006840F002001649103908600846D9
:1037B000006800F00200009000BF00BF6020019090
:1037C000022002900020039003200490092005901D
:1037D00001A90F4800F03CFC00220521402001F027
:1037E0009FF9402001F088F900220521412001F0D5
:1037F00097F9412001F080F906B010BD0064004047
:103800000400002040380240000C024000680040E4
:103810000004024070B505462846FEF749FF0446FD
:10382000032C11D004EB840000EBC400074901EB2A
:103830008000C06940B104EB840101EBC401034A7C
:1038400002EB8101C869804770BD000058720020FA
:1038500070B505462846FEF72BFF0446032C11D011
:1038600004EB840000EBC400074901EB8000806991
:1038700040B104EB840101EBC401034A02EB810176
:103880008869804770BD00005872002070B50546F9
:103890002846FEF70DFF0446032C11D004EB8400EC
:1038A00000EBC400074901EB8000406A40B104EB23
:1038B000840101EBC401034A02EB8101486A80479D
:1038C00070BD00005872002070B505462846FEF70E
:1038D000EFFE0446032C11D004EB840000EBC4007F
:1038E000074901EB8000006A40B104EB840101EB61
:1038F000C401034A02EB8101086A804770BD0000E1
:103900005872002070B505462846FEF7D1FE0446E1
:10391000032C11D004EB840000EBC400074901EB39
:103920008000806A40B104EB840101EBC401034ACA
:1039300002EB8101886A804770BD00005872002048
:1039400070B5044694F82000012822D1022084F8A2
:1039500020002068006820F001002168086000F065
:103960007FFC05460DE000F07BFC401B0A2808D9CF
:10397000606A40F400306062052084F82000012075
:1039800070BD2068406800F001000028EBD1606243
:10399000F6E7606A40F4002060620120F0E7000072
:1039A00070B505462846FEF783FE0446032C11D069
:1039B00004EB840000EBC400074901EB8000C06801
:1039C00040B104EB840101EBC401034A02EB810125
:1039D000C868804770BD00005872002070B5054669
:1039E0002846FEF765FE0446032C0FD004EB840046
:1039F00000EBC400064951F8200038B104EB840103
:103A000001EBC401024A52F82100804770BD00005A
:103A10005872002070B505462846FEF749FE044658
:103A2000032C11D004EB840000EBC400074901EB28
:103A30008000006940B104EB840101EBC401034A3A
:103A400002EB81010869804770BD000058720020B8
:103A500070B505462846FEF72BFE0446032C11D010
:103A600004EB840000EBC400074901EB80004068D0
:103A700040B104EB840101EBC401034A02EB810174
:103A80004868804770BD00005872002070B5054638
:103A90002846FEF70DFE0446032C11D004EB8400EB
:103AA00000EBC400074901EB8000406940B104EB22
:103AB000840101EBC401034A02EB8101486980479C
:103AC00070BD00005872002070B505462846FEF70C
:103AD000EFFD0446032C11D004EB840000EBC4007E
:103AE000074901EB8000806840B104EB840101EBE1
:103AF000C401034A02EB81018868804770BD000061
:103B00005872002070B505462846FEF7D1FD0446E0
:103B1000032C11D004EB840000EBC400074901EB37
:103B20008000C06A40B104EB840101EBC401034A88
:103B300002EB8101C86A804770BD00005872002006
:103B400070B50446A56D00F08BFB064694F8350071
:103B5000022808D08020606500BF002084F834006F
:103B600000BF012070BD2068006820F016002168A9
:103B700008602068406920F0800021684861206C5E
:103B800008B9A06C28B12068006820F008002168FE
:103B900008602068006820F001002168086010E0DB
:103BA00000F05EFB801B05280BD9202060650320F8
:103BB00084F8350000BF002084F8340000BF0320E3
:103BC000D0E72068006800F001000028E8D194F8F0
:103BD0005C103F208840A860012084F8350000BFB9
:103BE000002084F8340000BF00BFBBE7014691F815
:103BF0003500022803D08020486501207047052049
:103C000081F835000868006820F001000A6810603B
:103C10000020F3E7014691F835007047F8B50446F7
:103C2000002000908C4800684FF41651B0FBF1F76B
:103C3000A56D2E6894F85C1008208840304098B13B
:103C40002068006800F0040070B12068006820F06F
:103C500004002168086094F85C1008208840A8607F
:103C6000606D40F00100606594F85C1001208840B0
:103C7000304068B12068406900F0800040B194F89D
:103C80005C1001208840A860606D40F00200606513
:103C900094F85C1004208840304068B120680068C7
:103CA00000F0020040B194F85C1004208840A86045
:103CB000606D40F00400606594F85C10102088404E
:103CC000304078B32068006800F0080050B394F8E2
:103CD0005C1010208840A8602068006800F48020F4
:103CE00080B12068006800F4002028B9206CC8B1B9
:103CF0002046216C884715E0A06C98B12046A16C45
:103D000088470FE02068006800F4807028B92068B8
:103D1000006820F0080021680860206C10B120467F
:103D2000216C884794F85C1020208840304000289F
:103D300065D02068006800F0100000285FD094F87B
:103D40005C1020208840A86094F83500052828D110
:103D50002068006820F0160021680860206840692B
:103D600020F0800021684861206C08B9A06C28B15F
:103D70002068006820F008002168086094F85C1052
:103D80003F208840A860012084F8350000BF002053
:103D900084F8340000BF206D10B12046216D8847A3
:103DA000F8BD2068006800F4802080B120680068B9
:103DB00000F4002028B9606C10B12046616C88477F
:103DC0001DE0E06BD8B12046E16B884717E0206822
:103DD000006800F4807068B92068006820F0100066
:103DE00021680860012084F8350000BF002084F8B5
:103DF000340000BFE06B10B12046E16B8847606D76
:103E000038B3606D00F00100F0B1052084F8350092
:103E10002068006820F001002168086000BF009859
:103E2000401C0090B84200D905E02068006800F00E
:103E300001000028F3D100BF012084F8350000BF45
:103E4000002084F8340000BFE06C10B12046E16C23
:103E5000884700BFA4E70000140000202DE9F041CE
:103E60000446002500F0FCF9074614B90120BDE81E
:103E7000F081606A00B100BF022084F8350000BF05
:103E8000002084F8340000BF2068006820F00100A2
:103E9000216808600AE000F0E3F9C01B052805D995
:103EA00020206065032084F83500E0E72068006882
:103EB00000F001000028EED1206805682148054087
:103EC000D4E901010843E1680843216908436169B5
:103ED0000843A1690843E1690843216A084305438F
:103EE000606A042803D1D4E90B0108430543206824
:103EF00005602068456925F00705606A0543606A2A
:103F000004280DD1A06A0543E06A48B12046FEF7B7
:103F100089FC28B140206065012084F83500A6E7BF
:103F2000206845612046FEF763FC064694F85C1065
:103F30003F208840B06000206065012084F8350093
:103F4000002094E73F8010F02DE9F04704460D462D
:103F500016461F464FF00008D4F8589000BF94F85A
:103F60003400012802D10220BDE8F087012084F846
:103F7000340000BF94F83500012825D1022084F8D0
:103F80003500002060653B46324629462046FEF754
:103F90009EFC94F85C103F208840C9F80800206817
:103FA000006840F0160021680860206C28B1206885
:103FB000006840F00800216808602068006840F050
:103FC00001002168086006E000BF002084F834008A
:103FD00000BF4FF002084046C6E7000070B5044637
:103FE00000F03EF906462546681C10B104480078EA
:103FF000054400BF00F034F9801BA842FAD370BD1D
:104000001000002070B5054600240DE00120A040FE
:10401000284038B1064850F8240018B1044951F836
:1040200024008047601CC4B2102CEFDB70BD000080
:10403000C072002010B5044604480068204020B13A
:10404000024804602046FFF7DDFF10BD143C01402C
:10405000F8B502460B460025002400200021D6E0DA
:10406000012606FA01F51E6806EA0504AC4274D181
:104070001E7906F00306012E04D01E7906F0030611
:10408000022E13D190684F000326BE40B0434F006C
:10409000DE68BE4030439060506801268E40B043D9
:1040A0001E79C6F300168E40304350601E7906F02C
:1040B0000306032E09D0D0684F000326BE40B0434C
:1040C0004F009E68BE403043D0601E7906F0030664
:1040D000022E13D1CF0802F1200656F827004E0712
:1040E000F70E0F26BE40B0434F07FF0E1E69BE40BD
:1040F0003043CF0802F1200646F8270010684F0031
:104100000326BE40B0431E7906F003064F00BE40B2
:10411000304310605E6806F44036002E76D000BF53
:10412000002600963C4E366846F480463A4F3E6084
:104130003E46366806F48046009600BF00BF374E04
:104140008F0856F827008E07370F0F26BE40B04362
:10415000334EB24202D1002624E057E0314EB24243
:1041600001D101261EE0304EB24201D1022619E0F3
:104170002E4EB24201D1032614E02D4EB24201D19F
:1041800004260FE02B4EB24201D105260AE02A4E4A
:10419000B24201D1062605E0284EB24201D10726DF
:1041A00000E008268F073F0FBE4030431B4E8F08AC
:1041B00046F82700224E3068A0435E6806F4801659
:1041C00006B120431E4E3060361D3068A0435E6845
:1041D00006F4001606B12043194E361D3060184E05
:1041E000361F3068A0435E6806F4003606B12043EF
:1041F000134E361F3060361F3068A0435E6806F4E9
:10420000803606B120430E4E083E3060491C10290E
:10421000FFF426AFF8BD00004438024008380140E2
:10422000000002400004024000080240000C02406E
:10423000001002400014024000180240001C02401E
:10424000083C0140024613690B400BB1012000E01D
:10425000002070470AB1816101E00B04836170475F
:1042600001480068704700000800002070B505464E
:10427000284602F04FFD0446032C0DD004EBC40089
:10428000064901EB8000006A30B104EBC401034A27
:1042900002EB8101086A804770BD000000730020B6
:1042A00070472DE9F84F0446206847692068D0F828
:1042B0000480002594F83E90C7F3002040B1C8F375
:1042C000002028B145F001056FF480702168486135
:1042D000C7F3402040B1C8F3002028B145F00205E3
:1042E0006FF4007021684861C7F3802070B3C8F391
:1042F000002058B3CA46B4F82AB094F83D60206B49
:104300000090BAF1200F0FD1BBF1000F0CD1212E7C
:1043100006D0292E04D0282E06D10098212803D1BA
:10432000204603F04BFA11E06FF480602168486189
:1043300045F00405B9F1100F02D0B9F1400F05D1D5
:104340002068006840F4007021680860C7F3C0204E
:1043500040B1C8F3002028B145F008056FF40060B3
:10436000216848612DB1206C28432064204602F06A
:10437000E5FCBDE8F88F2DE9F04705464FF0000950
:1043800028684668D5F82CA095F83E7095F83D80D1
:10439000102F01D0402F75D12868D0F818902868C8
:1043A000446904F0010060B9BAF52A0F02D0BAF1ED
:1043B0002A4F01D1012000E00020012801D1BDE8F1
:1043C000F08704F0010048B1C6F3402030B1284620
:1043D00002F00CFC284603F0A6F8B7E0C4F3C000D6
:1043E00030B1C6F3402018B1284602F053FFADE0CB
:1043F000C4F3400030B1C6F3402018B1284602F0A3
:104400005EFFA3E0C9F3800040B32868406800F471
:104410000060B0F5006FE0D0C4F3C01048B1C6F33F
:10442000802030B1C4F3800018B9284602F0C6FEDF
:104430008CE0C4F380000028CFD0C6F340200028D1
:10444000CBD0B8F1210F03D1284602F067FE7DE002
:10445000402F7BD1284603F0B5F877E02868406804
:1044600000F40060B0F5006F70D0C4F3801050B15C
:10447000C6F3802038B1C4F3800020B9284602F08A
:10448000CBFD63E00BE0C4F3800000285ED0C6F3F0
:10449000402000285AD0284602F026FD56E0286C1D
:1044A00010B12868446904E02868D0F8189028689A
:1044B0004469C4F3400060B1C6F3402048B1286CA1
:1044C00010B12868D0F818904946284603F03DF905
:1044D0003CE0C4F3001030B1C6F3402018B12846C8
:1044E00003F0C0F932E0B8F1210F02D0B8F1290F82
:1044F00016D1C4F3C01048B1C6F3802030B1C4F364
:10450000800018B9284603F0FDF81FE0C4F38000CE
:10451000E0B1C6F34020C8B1284603F0E6F815E044
:10452000C4F3801048B1C6F3802030B1C4F38000DA
:1045300018B9284603F0B6F808E0C4F3800028B1A3
:10454000C6F3402010B1284603F09FF800BF36E7BD
:1045500070B50546284602F0DDFB0446032C0DD05D
:1045600004EBC400064901EB8000C06930B104EBE4
:10457000C401034A02EB8101C869804770BD000095
:104580000073002070B504460CB9012070BD94F88A
:104590003D0028B9002084F83C00204600F05AF97C
:1045A000242084F83D002068006820F00100216884
:1045B00008602068006840F40040216808602068B6
:1045C000006820F400402168086000F0C3FB054645
:1045D0005C496068884206D85B48854201D2012068
:1045E00007E0002005E05948854201D2012000E0A3
:1045F0000020012800D1C9E75548B5FBF0F6206836
:10460000406820F03F003043216848604D496068B1
:10461000884201D8701C07E04FF4967070434FF445
:104620007A71B0FBF1F0401C2168096A21F03F016A
:1046300008432168086243496068884214D8681EAC
:1046400061684900B0FBF1F0401CC0F30B00042886
:1046500001D204203DE0681E61684900B0FBF1F022
:10466000401CC0F30B0034E0A06838B9681E6168D4
:1046700001EB4101B0FBF1F0401C0AE0681E6168EB
:1046800001EBC10202EB0111B0FBF1F0401C40F460
:104690008040C0F30B0008B901201AE0A06848B9B7
:1046A000681E616801EB4101B0FBF1F0401CC0F3F2
:1046B0000B000CE0681E616801EBC10202EB011106
:1046C000B0FBF1F0401CC0F30B0040F4804040F41C
:1046D00000402168C9694CF6FF7291430843216884
:1046E000C861D4E9070108432168096821F0C001C5
:1046F000084321680860D4E90310084321688968E9
:1047000048F2FF329143084321688860D4E90501EB
:1047100008432168C96821F0FF0108432168C86087
:104720002068006840F001002168086000202064D3
:10473000202084F83D000020206384F83E0000BF64
:1047400024E70000A086010080841E0000093D00CF
:1047500040420F0070B50546284602F0DBFA0446D9
:10476000032C0DD004EBC400064901EB8000006966
:1047700030B104EBC401034A02EB810108698047B0
:1047800070BD00000073002070B50546284602F099
:10479000C1FA0446032C0DD004EBC400064901EB1A
:1047A0008000406830B104EBC401034A02EB810190
:1047B0004868804770BD00000073002070B5054652
:1047C000284602F0A7FA0446032C0BD004EBC400E1
:1047D000054951F8200028B104EBC401024A52F8FF
:1047E0002100804770BD00000073002070B50546B1
:1047F000284602F08FFA0446032C0DD004EBC400C7
:10480000064901EB8000806930B104EBC401034A22
:1048100002EB81018869804770BD000000730020B1
:1048200070B50546284602F075FA0446032C0DD0F3
:1048300004EBC400064901EB8000406930B104EB91
:10484000C401034A02EB81014869804770BD000042
:104850000073002010B586B00446142101A8FBF7B0
:104860009BFE3E492068884241D100BF0020009055
:104870003B48006840F0020039490860084600687B
:1048800000F00200009000BF00BF4FF440700190A4
:104890001220029000200390032004900420059031
:1048A00001A93048FFF7D4FB00BF002000902C483E
:1048B0001030006840F400102949103108600846A3
:1048C000006800F40010009000BF00BF0022052126
:1048D0001F2000F025F91F2000F00EF9002205210D
:1048E000202000F01DF9202000F006F933E01E49D9
:1048F000206888422FD100BF00200090184800682F
:1049000040F02000164908600846006800F02000CA
:10491000009000BF00BF03200190122002900020F1
:104920000390032004900420059001A90F48FFF78D
:104930008FFB00BF0020009009481030006840F451
:1049400080000749103108600846006800F48000C4
:10495000009000BF00BF06B010BD00000054004032
:104960003038024000040240005800400014024069
:1049700070B50546284602F0CDF90446032C0DD04B
:1049800004EBC400064901EB8000C06830B104EBC1
:10499000C401034A02EB8101C868804770BD000072
:1049A0000073002070B50546284602F0B3F90446AE
:1049B000032C0DD004EBC400064901EB8000806895
:1049C00030B104EBC401034A02EB810188688047DF
:1049D00070BD000000730020034800680349097897
:1049E00008440149086070470800002010000020BA
:1049F00010B50D48006840F400700B490860084687
:104A0000006840F4806008600846006840F48070E8
:104A10000860032000F0C2F80F2000F007F800F053
:104A20002BF8002010BD0000003C024070B5044689
:104A30000E4800784FF47A71B1FBF0F00C49096828
:104A4000B1FBF0F5284601F0D5FA08B1012070BDA0
:104A5000102C07D200222146501E00F061F80548B4
:104A6000046001E00120F2E70020F0E710000020E0
:104A7000140000200C00002008B500BF00200090AA
:104A80001148006840F480400F49086008460068FB
:104A900000F48040009000BF00BF00BF00200090E5
:104AA000081F006840F08050091F08600846006831
:104AB00000F08050009000BF00BF00220F21901E28
:104AC00000F02EF808BD00004438024010B5014641
:104AD000084600280BDB00F01F0301229A40054B1B
:104AE000440943F82420BFF34F8FBFF36F8F00BFFB
:104AF00010BD000080E100E00146084600280DDB03
:104B000000BF00BF00F01F0301229A4043099B0031
:104B100003F1E023C3F8002100BF00BF00BF7047CE
:104B20002DE9F05F80460D461646002704F0DEFFB3
:104B3000074639462A46334601F00700C0F1070A06
:104B4000BAF1040F02D94FF0040A01E0C0F1070ADC
:104B5000D14600F1040ABAF1070F02D24FF0000A61
:104B600001E0A0F1030AD4464FF0010A0AFA09FA5B
:104B7000AAF1010A0AEA020A0AFA0CFA4FF0010B3A
:104B80000BFA0CFBABF1010B0BEA030B4AEA0B042B
:104B90002146404604F0B2FFBDE8F09F00BF00F0A0
:104BA0000702064B19684FF6FF031940044B0B43ED
:104BB00043EA0221014B196000BF70470CED00E091
:104BC0000000FA0570B504460D460CB9012070BD11
:104BD0005848006800F00700A84209D255490D70F6
:104BE0000846006800F00700A84201D00120EEE767
:104BF000207800F0020002281DD1207800F0040087
:104C0000042805D14C48006840F4E0504A49086047
:104C1000207800F00800082805D14748006840F4D3
:104C20006040454908604448006820F0F000A168F1
:104C3000084341490860207800F00100A8B360688B
:104C4000012807D13C4808380068C0F34040B8B993
:104C50000120BCE76068022802D06068032807D101
:104C6000354808380068C0F3406048B90120AEE715
:104C7000314808380068C0F3400008B90120A6E7B1
:104C80002D48006820F00300616808432A49086045
:104C9000FFF7E6FA064609E0FFF7E2FA801B41F269
:104CA0008831884202D9032091E707E02248006852
:104CB00000F00C006168B0EB810FEDD11D48006879
:104CC00000F00700A84209D91A490D70084600688B
:104CD00000F00700A84201D0012078E7207800F01A
:104CE0000400042807D11448006820F4E050E1686B
:104CF000084311490860207800F00800082808D10E
:104D00000D48006820F46040216940EAC1000A496A
:104D1000086000F03FF808490968C1F30311074A29
:104D2000515CC8400649086006480068FFF77EFEEF
:104D300000204CE7003C02400838024064EB0008C9
:104D4000140000200C00002001480068704700009B
:104D50001400002000B5FFF7F7FF04490968C1F30C
:104D60008221034A515CC84000BD0000083802405F
:104D700074EB000800B5FFF7E7FF04490968C1F3C9
:104D80004231034A515CC84000BD0000083802406F
:104D900074EB00082DE9F047002400250026A14609
:104DA0002548006800F00C0020B1042805D0082830
:104DB0003AD105E0DFF8849039E0DFF8849036E0FE
:104DC0001D48001F006800F03F041B48001F0068DA
:104DD00000F4800078B11A481749091F0968C1F327
:104DE0008811A0FB01700146224600233846FBF7DC
:104DF000BBFA05460EE011480F49091F0968C1F3C7
:104E00008811A0FB01700146224600233846FBF7BB
:104E1000ABFA05460848001F0068C0F30140401C7B
:104E20004600B5FBF6F902E0DFF8109000BF00BFC6
:104E30004846BDE8F0870000083802400024F4002E
:104E4000001BB700F8B504460CB90120F8BD207866
:104E500000F00100002874D0F948006800F00C0050
:104E600004280DD0F648006800F00C00082813D183
:104E7000F348001F006800F48000B0F5800F0BD1EC
:104E8000EF4808380068C0F34040002859D06068F7
:104E9000002856D10120D9E700BF6068B0F5803FF7
:104EA00008D1E7480838006840F48030E449083900
:104EB00008601EE06068B0F5A02F0DD1E04808380A
:104EC000006840F48020DE49083908600846006820
:104ED00040F4803008600CE0D9480838006820F4BD
:104EE0008030D749083908600846006820F48020DF
:104EF000086000BF606890B1FFF7B2F9054606E0B0
:104F0000FFF7AEF9401B642801D903209EE7CC4887
:104F100008380068C0F340400028F1D011E0FFF7E6
:104F20009FF9054606E0FFF79BF9401B642801D96D
:104F300003208BE7C24808380068C0F340400028CF
:104F4000F1D1207800F0020002285FD1BC4800684F
:104F500000F00C0058B1BA48006800F00C000828B6
:104F60001CD1B748001F006800F48000B0B9B448F5
:104F700008380068C0F3400020B1E068012801D083
:104F8000012063E7AE480838006820F0F800216986
:104F900040EAC100AA490839086037E0E06800B378
:104FA0000120A8490860FFF75BF9054606E0FFF716
:104FB00057F9401B022801D9032047E7A0480838C9
:104FC0000068C0F340000028F1D09D480838006810
:104FD00020F0F800216940EAC100994908390860C9
:104FE00014E0002097490860FFF73AF9054606E00B
:104FF000FFF736F9401B022801D9032026E7904825
:1050000008380068C0F340000028F1D1207800F093
:10501000080008282CD16069A8B101208A490860DD
:10502000FFF71EF9054606E0FFF71AF9401B0228B4
:1050300001D903200AE782486C300068C0F34000C1
:105040000028F1D014E000207F490860FFF708F93C
:10505000054606E0FFF704F9401B022801D90320AA
:10506000F4E677486C300068C0F340000028F1D1C6
:10507000207800F00400042870D1002770483830F0
:10508000006800F0805090B900BF002000906C488C
:105090003830006840F0805069493831086008466F
:1050A000006800F08050009000BF00BF01276748F3
:1050B000006800F48070B0B96448006840F4807003
:1050C00062490860FFF7CCF8054606E0FFF7C8F82C
:1050D000401B022801D90320B8E65C48006800F4B0
:1050E00080700028F2D000BFA068012808D1544881
:1050F0006830006840F001005149683108601DE0E7
:10510000A06805280DD14E486830006840F00400C2
:105110004B49683108600846006840F001000860AB
:105120000CE047486830006820F0010044496831CD
:1051300008600846006820F00400086000BFA0680E
:10514000A8B1FFF78DF8054609E0FFF789F8401B85
:1051500041F28831884202D9032077E626E03848B8
:1051600068300068C0F340000028EED013E0FFF77D
:1051700077F8054608E0FFF773F8401B41F28831E5
:10518000884201D9032061E62D4868300068C0F3E9
:1051900040000028EFD1012F07D12948383000689E
:1051A00020F0805026493831086000BFA0690028EF
:1051B00045D02348006800F00C0008285DD0A069A5
:1051C000022845D100201F490866FFF749F8054627
:1051D00006E0FFF745F8401B022801D9032035E619
:1051E000174808380068C0F340600028F1D1D4E9BE
:1051F00007010843616A40EA81110122A06AC2EBFB
:10520000500041EA00412C20005D41EA00600C4959
:10521000091F086001200B490866FFF721F80546C1
:1052200006E0FFF71DF8401B022801D903200DE618
:10523000034808380068C0F340600028F1D049E016
:105240000838024000004742800E4742007000408C
:10525000002021490866FFF703F8054606E0FEF73F
:10526000FFFF401B022801D90320EFE51B4800681F
:10527000C0F340600028F2D12CE0A069012800D1E1
:10528000E4E51648001D0668A069012820D006F450
:105290008001E06981421BD106F03F01206A814212
:1052A00016D147F6C0703040616AB0EB811F0FD154
:1052B00006F440310122A06AC2EB5000B1EB004F6E
:1052C00006D106F070612C20005DB1EB006F01D0BB
:1052D0000120BBE50020B9E500004742003802404C
:1052E00070B50446204603F0BBFD0546032D0FD0E4
:1052F000204603F0B5FD074901EB4010806938B145
:10530000204603F0ADFD034901EB40108669B0472C
:1053100070BD00004873002010B504460CB9012090
:1053200010BD606A38B96068B0F5827F00D105E0D1
:105330000021E16102E00021216161610021A1629F
:1053400094F8510028B9002084F85000204600F05D
:1053500047F8022084F851002068006820F04000DF
:1053600021680860A08800F48270218901F404415A
:105370000843A18901F400610843217C01F0020186
:105380000843217D01F001010843218B01F40071E4
:105390000843217F01F0380108432021095D01F015
:1053A00080010843218D01F4005108432168086001
:1053B0000421A06901EA104094F8241001F01001C2
:1053C0000843216848602068C06920F400602168B3
:1053D000C86100206065012084F8510000209FE72B
:1053E00010B586B00446142101A8FBF7D5F866492C
:1053F000206888427ED100BF00200090634800688A
:1054000040F48050614908600846006800F480500C
:10541000009000BF00BF00BF002000905B48143820
:10542000006840F0020059491439086008460068D5
:1054300000F00200009000BF00BF00BF00200090FD
:105440000846006840F0010008600846006800F067
:105450000100009000BF00BF1820019002200290C0
:1054600001200390032004900520059001A94848DD
:10547000FEF7EEFD802001900220029001200390B3
:10548000032004900520059001A94248FEF7E0FDA5
:105490004148424908604FF0C060486000213F48E1
:1054A0008160C1604FF480610161002141618161CF
:1054B000C1614FF44031016200214162FEF7CEFC30
:1054C00008B1FDF72FFA00BF3448E064846300BFE1
:1054D00031481830324908604FF0C06048604021C0
:1054E0002F4881600021C1604FF48061016100217B
:1054F000416100E010E08161C1614FF4003101625F
:1055000000214162FEF7AAFC08B1FDF70BFA00BFCB
:105510002348A064846335E022492068884231D161
:1055200000BF002000901948001F006840F4804030
:105530001649091F08600846006800F48040009082
:1055400000BF00BF00BF0020009010481438006862
:1055500040F480700D49143908600846006800F472
:105560008070009000BF00BF0E20019002200290CA
:1055700001200390032004900520059001A90A480A
:10558000FEF766FD06B010BD003001404438024011
:105590000004024000000240406402403403002046
:1055A0009403002000380040002002402DE9F84319
:1055B0000446884616461D4694F85100012802D03C
:1055C0000220BDE8F883B8F1000F00D00EB9012029
:1055D000F7E76068B0F5827F0CD1A06850B904206D
:1055E00084F851003346424641462046009500F07B
:1055F00042FAE6E7FEF734FE074600BF94F8500093
:10560000012801D10220DCE7012084F8500000BF0E
:10561000042084F8510000206065C4F83880A68713
:10562000E6872063A086E08620646064A068B0F509
:10563000004F0BD12068006820F04000216808600E
:105640002068006820F480402168086020680068B5
:1056500000F04000402805D02068006840F040007D
:1056600021680860E06830BB21E02068806800F0B5
:10567000010050B12068007BA16B0870A06B401C3A
:10568000A063E08F401EE08711E0FEF7E9FDC01B3C
:10569000A84201D3681C00B94DB9012084F851001B
:1056A00000BF002084F8500000BF032089E7E08F8E
:1056B0000028DAD125E021E02068806800F00100B0
:1056C00050B12068C068A16B0880A06B801CA063EB
:1056D000E08F401EE08711E0FEF7C2FDC01BA8422C
:1056E00001D3681C00B94DB9012084F8510000BFF6
:1056F000002084F8500000BF032062E7E08F0028FC
:10570000DAD13A462946204603F01BFB08B1202097
:105710006065012084F8510000BF002084F850002B
:1057200000BF606D08B101204BE7002049E7000091
:105730002DE9F04104460E46154694F85100012823
:1057400002D00220BDE8F08106B10DB90120F9E7D1
:10575000A06868B96068B0F5827F09D1042084F838
:1057600051002B4632463146204600F0A9FAE9E7BF
:1057700000BF94F85000012801D10220E2E7012087
:1057800084F8500000BF042084F8510000206065B8
:10579000A663A587E58720646064A086E086A0688C
:1057A000B0F5004F0BD12068006820F04000216860
:1057B00008602068006820F48040216808601F4865
:1057C000E16C08641E48E16CC8631E48E16CC86463
:1057D0000020E16C0865E38F276807F10C01A26BDC
:1057E000E06CFEF7B1FB50B1606D40F010006065F9
:1057F00000BF002084F8500000BF0120A2E720680D
:10580000006800F04000402805D02068006840F0A3
:1058100040002168086000BF002084F8500000BFED
:105820002068406840F02000216848602068406897
:1058300040F0010021684860002083E7B58B000834
:10584000DF8B00088D8B000870B50446204603F0FE
:1058500007FB0546032D0FD0204603F001FB074947
:1058600001EB4010406838B1204603F0F9FA0349D3
:1058700001EB40104668B04770BD0000487300203F
:1058800070B50446204603F0EBFA0546032D0FD011
:10589000204603F0E5FA074901EB4010006938B1F2
:1058A000204603F0DDFA034901EB40100669B047DA
:1058B00070BD0000487300202DE9F84304460F46F0
:1058C00016461D46FEF7CCFC8046B14694F85100C2
:1058D000012802D00220BDE8F88307B10EB90120EB
:1058E000F9E700BF94F85000012801D10220F2E747
:1058F000012084F8500000BF032084F851000020EC
:1059000060652763A686E686A063A087E08760645B
:105910002064A068B0F5004F0BD12068006820F02B
:105920004000216808602068006840F480402168D9
:1059300008602068006800F04000402805D020681A
:10594000006840F0400021680860E068B0F5006F32
:1059500037D1606810B1B9F1010F09D1206B00880F
:105960002168C860206B801C2063E08E401EE086AA
:1059700023E02068806800F0020002280AD1206B32
:1059800000882168C860206B801C2063E08E401E68
:10599000E08612E0FEF764FCA0EB0800A84201D309
:1059A000681C00B94DB9012084F8510000BF0020E7
:1059B00084F8500000BF03208DE7E08E0028D8D186
:1059C00036E0606810B1B9F1010F09D1206B0078A1
:1059D00021680873206B401C2063E08E401EE08627
:1059E00023E02068806800F0020002280AD1206BC2
:1059F000007821680873206B401C2063E08E401EF5
:105A0000E08612E0FEF72CFCA0EB0800A84201D3D0
:105A1000681C00B94DB9012084F8510000BF002076
:105A200084F8500000BF032055E7E08E0028D8D14D
:105A300042462946204603F0CFF908B12020606590
:105A4000A06850B900BF002000902068C068009096
:105A500020688068009000BF00BF012084F85100DA
:105A600000BF002084F8500000BF606D08B1012025
:105A700031E700202FE72DE9FE4F04460F46904600
:105A80001D460C9E01200190FEF7EAFB814694F82A
:105A900051B060680290AA46BBF1010F0BD002988A
:105AA000B0F5827F04D1A06810B9BBF1040F02D019
:105AB0000220BDE8FE8F1FB1B8F1000F00D00DB974
:105AC0000120F6E700BF94F85000012801D1022020
:105AD000EFE7012084F8500000BF94F8510004283B
:105AE00002D0052084F8510000206065C4F8388099
:105AF000E587A5872763E586A5862064606420681E
:105B0000006800F04000402805D02068006840F0A0
:105B1000400021680860E068B0F5006F52D160680D
:105B200010B1BAF1010F09D1206B00882168C8605B
:105B3000206B801C2063E08E401EE0863BE02068E6
:105B4000806800F00200022810D1E08E70B1019848
:105B500001280BD1206B00882168C860206B801C55
:105B60002063E08E401EE08600200190206880685F
:105B700000F0010068B1E08F58B12068C068A16BE7
:105B80000880A06B801CA063E08F401EE08701208E
:105B90000190FEF765FBA0EB0900B0420BD3701C2F
:105BA00048B1012084F8510000BF002084F8500063
:105BB00000BF03207DE7E08E0028C0D1E08F0028E1
:105BC000BDD152E0606810B1BAF1010F09D1206B6C
:105BD000007821680873206B401C2063E08E401E13
:105BE000E0863CE02068806800F00200022810D1C6
:105BF000E08E70B1019801280BD1206B00782168EC
:105C00000873206B401C2063E08E401EE08600205D
:105C100001902068806800F0010068B1E08F58B101
:105C20002068C068A16B0870A06B401CA063E08F67
:105C3000401EE08701200190FEF712FBA0EB090057
:105C4000B04201D3701C00B94EB9012084F8510054
:105C500000BF002084F8500000BF032029E7E08E39
:105C60000028BFD1E08F0028BCD14A4631462046EB
:105C700003F0B2F840B12020606500BF002084F836
:105C8000500000BF012014E7A06850B900BF0020F9
:105C900000902068C068009020688068009000BF75
:105CA00000BF012084F8510000BF002084F850009C
:105CB00000BF606D08B10120FBE60020F9E600009E
:105CC0002DE9F04704460E4617461D4694F85180CC
:105CD000D4F80490B8F1010F0AD0B9F5827F04D14D
:105CE000A06810B9B8F1040F02D00220BDE8F08717
:105CF0000EB107B10DB90120F8E700BF94F85000CC
:105D0000012801D10220F1E7012084F8500000BFF2
:105D100094F85100042802D0052084F85100002096
:105D200060652663A586E586A763A587E587206469
:105D3000606494F85100042806D13548E16C086489
:105D40003448E16CC86305E03348E16C08643348CB
:105D5000E16CC8633248E16CC8640020E16C0865FE
:105D6000E38FD4F800C00CF10C01A26BE06CFEF7DD
:105D7000EBF850B1606D40F01000606500BF00208E
:105D800084F8500000BF0120B0E72068406840F070
:105D90000100216848600020A16C0864A16CC86300
:105DA000A16CC864A16C0865E38ED4F800C00CF146
:105DB0000C02216BA06CFEF7C7F850B1606D40F08B
:105DC0001000606500BF002084F8500000BF012073
:105DD0008CE72068006800F04000402805D020686B
:105DE000006840F040002168086000BF002084F88F
:105DF000500000BF2068406840F0200021684860E3
:105E00002068406840F002002168486000206DE78B
:105E1000B58B0008DF8B0008D18B0008DB8C0008F5
:105E20008D8B00082DE9F04104460E46154694F886
:105E30005100012802D00220BDE8F08106B10DB961
:105E40000120F9E700BF94F85000012801D1022099
:105E5000F2E7012084F8500000BF032084F85100CD
:105E6000002060652663A586E586A06360642064E3
:105E7000A087E087A068B0F5004F0BD120680068CC
:105E800020F04000216808602068006840F48040ED
:105E9000216808601F48A16C08641F48A16CC86392
:105EA0001E48A16CC8640020A16C0865E38E2768B9
:105EB00007F10C02216BA06CFEF746F850B1606D43
:105EC00040F01000606500BF002084F8500000BF63
:105ED0000120B1E72068006800F04000402805D0AC
:105EE0002068006840F040002168086000BF002082
:105EF00084F8500000BF2068406840F0200021680E
:105F000048602068406840F0020021684860002036
:105F100092E70000C38B00085B8C00088D8B0008A3
:105F200070B50546284602F09BFF0446032C09D0B5
:105F3000054800EB4410006820B1034901EB44110F
:105F40000868804770BD00004873002070B50446A3
:105F5000204602F085FF0546032D0FD0204602F0B3
:105F60007FFF074901EB4010C06838B1204602F0BE
:105F700077FF034901EB4010C668B04770BD0000D1
:105F80004873002070B50446204602F069FF0546BC
:105F9000032D0FD0204602F063FF074901EB4010AC
:105FA000806838B1204602F05BFF034901EB4010E6
:105FB0008668B04770BD00004873002070B5044685
:105FC000204602F04DFF0546032D0FD0204602F07B
:105FD00047FF074901EB4010406938B1204602F005
:105FE0003FFF034901EB40104669B04770BD000018
:105FF0004873002070B504462546681EB0F1807FC6
:1060000001D301200FE0681E4FF0E02148610F210D
:106010004FF0FF3003F072FD00204FF0E021886167
:1060200007200861002070BD7047704730B50246F8
:106030000B4600BF92F83C00012801D1022030BD80
:10604000012082F83C0000BF022082F83D00106869
:1060500044681068816824F070041868044310686C
:106060004460184D1068A8421BD01068B0F1804FF2
:1060700017D0154D1068A84213D0144D1068A842CF
:106080000FD0134D1068A8420BD0124D1068A842D3
:1060900007D0114D1068A84203D0104D1068A842D7
:1060A00005D121F08001586801431068816001200A
:1060B00082F83D0000BF002082F83C0000BF00BF16
:1060C000BDE700000000014000040040000800405F
:1060D000000C004000040140004001400018004056
:1060E00010B504460CB9012010BD94F83D0028B944
:1060F000002084F83C00204600F026F8022084F8B6
:106100003D00211D206802F0A1FF012084F8460017
:1061100000BF84F83E0001213F2001554020015579
:106120004120015500BF00BF012084F842004320F8
:106130000155442001554520015500BF012084F838
:106140003D000020D0E7000038B50446194920681A
:10615000884218D100BF002000901748006840F026
:106160002000154908600846006800F020000090F3
:1061700000BF00BF002205213720FEF7D1FC3720E9
:10618000FEF7BAFC15E00D492068884211D100BF26
:10619000002000900848001D006840F400300649C7
:1061A000091D08600846006800F40030009000BF38
:1061B00000BF38BD00140040403802400044014098
:1061C000704770B504462068C5682068066906F007
:1061D0000200022819D105F00200022815D1401F43
:1061E00021680861012020772068806900F00300A1
:1061F00018B12046FFF7E4FF05E0204600F0C8F89C
:10620000204600F07CF90020207706F004000428E6
:1062100019D105F00400042815D1C0432168086194
:10622000022020772068806900F4407018B1204671
:10623000FFF7C6FF05E0204600F0AAF8204600F070
:106240005EF90020207706F00800082819D105F033
:106250000800082815D1C043216808610420207770
:106260002068C06900F0030018B12046FFF7A8FFBE
:1062700005E0204600F08CF8204600F040F90020B0
:10628000207706F01000102819D105F01000102812
:1062900015D1C04321680861082020772068C069B3
:1062A00000F4407018B12046FFF78AFF05E0204651
:1062B00000F06EF8204600F022F90020207706F06A
:1062C000010048B105F0010030B16FF00100216814
:1062D0000861204600F09AF906F08000802809D174
:1062E00005F08000802805D1C04321680861204660
:1062F000FFF79AFE06F04000402809D105F0400063
:10630000402805D1C04321680861204600F07FF98C
:1063100006F02000202809D105F02000202805D112
:10632000C043216808612046FFF77FFE70BD000072
:1063300010B586B00446142101A8FAF72DF91149C9
:10634000206888421CD100BF002000900E480068E1
:1063500040F020000C4908600846006800F020006A
:10636000009000BF00BF402001900220029000205A
:10637000039004900320059001A90448FDF768FEEE
:1063800006B010BD00440140303802400014024005
:1063900070472DE9F04104460D461646002700BF20
:1063A00094F83C00012802D10220BDE8F0810120D0
:1063B00084F83C0000BF36B1042E1BD0082E31D02B
:1063C0000C2E5ED145E02946206802F0C1FE20680F
:1063D000806940F00800216888612068806920F0A9
:1063E0000400216888612068806929690843216860
:1063F000886148E02946206802F0E2FE2068806952
:1064000040F40060216888612068806920F4806021
:106410002168886120688069296940EA0120216833
:10642000886130E02946206802F008FF2068C069D2
:1064300040F008002168C8612068C06920F00400AD
:106440002168C8612068C069296908432168C8615A
:1064500019E02946206802F02DFF2068C06940F449
:1064600000602168C8612068C06920F480602168EC
:10647000C8612068C069296940EA01202168C861B3
:1064800001E0012700BF00BF00BF002084F83C00EE
:1064900000BF384689E710B504460CB9012010BD8D
:1064A00094F83D0028B9002084F83C00204600F014
:1064B00025F8022084F83D00211D206802F0C6FD69
:1064C000012084F8460000BF84F83E0001213F20EF
:1064D0000155402001554120015500BF00BF01205A
:1064E00084F84200432001554420015545200155C0
:1064F00000BF012084F83D000020D0E770477047BE
:1065000070B504460D4615B994F83E000BE0042D15
:1065100002D13F20005D06E0082D02D14020005D41
:1065200001E04120005D012801D0012070BD1DB9AE
:10653000022084F83E000EE0042D03D102213F200A
:10654000015508E0082D03D102214020015502E049
:1065500002214120015501222946206802F0E6FD72
:1065600023492068884203D022492068884201D10B
:10657000012000E0002028B12068406C40F4004079
:10658000216848641A49206888421BD02068B0F10D
:10659000804F17D018492068884213D017492068C7
:1065A00088420FD01649206888420BD011492068D4
:1065B000884207D013492068884203D012492068D6
:1065C00088420CD12068806800F00706062E0CD0A7
:1065D0002068006840F001002168086005E020683C
:1065E000006840F001002168086000209EE700007C
:1065F0000000014000040140000400400008004089
:10660000000C0040004001400018004070477047F7
:106610007047000070B50546284603F049F8044667
:10662000022C0DD004EBC400064901EB8000006988
:1066300030B104EBC401034A02EB810108698047D1
:1066400070BD0000887300202DE9F84F04462068D3
:1066500005682068C668206847694FF00009CA4687
:1066600005F00F09B9F1000F0AD105F0200038B18B
:1066700006F0200020B1204603F026F8BDE8F88F90
:10668000B9F1000F7CD007F0010018B906F4907042
:10669000002875D005F0010030B106F4807018B103
:1066A000606C40F00100606405F0040030B107F058
:1066B000010018B1606C40F00200606405F0020057
:1066C00030B107F0010018B1606C40F00400606464
:1066D00005F0080048B106F0200010B907F00100ED
:1066E00018B1606C40F008006064606C002846D00F
:1066F00005F0200028B106F0200010B1204602F07D
:10670000E3FF20684069C0F3801A606C00F0080065
:1067100010B9BAF1000F2DD0204602F082FF206898
:10672000406900F04000402820D100BF00BF216830
:10673000143151E8001F21F040002168143141E874
:106740000002002AF3D100BFE06B50B17F48E16B3B
:106750000865E06BFDF74AFA88B1E06B016D884788
:106760000DE02046FFF756FF09E009E02046FFF75D
:1067700051FF04E02046FFF74DFF002060647DE7F5
:10678000206B012878D105F01000002874D006F0A5
:1067900010000028FAD000BF002000902068006898
:1067A000009020684068009000BF00BF20684069EA
:1067B00000F04000402870D1E06B006840681FFA8C
:1067C00080F8B8F1000F58D0A08D404555DDA4F8F1
:1067D0002E80E06BC069B0F5807F43D000BF00BF62
:1067E00021680C3151E8001F21F4807021680C31C0
:1067F00041E80002002AF3D100BF00BF00BF2168BA
:10680000143151E8001F21F001002168143141E8E2
:106810000002002AF3D100BF00BF00BF216814317D
:1068200051E8001F21F040002168143141E80002C6
:10683000002AF3D100BF202084F84200002020630A
:1068400000BF00BF21680C3151E8001F21F010008B
:1068500021680C3141E80002002AF3D100BFE06B4F
:10686000FDF76EF902206063A08DE28D801A81B27F
:106870002046FFF7CDFE0EE052E0A08D40450AD144
:10688000E06BC069B0F5807F05D102206063A18D07
:106890002046FFF7BDFEF1E6FFE7A08DE18D401A2F
:1068A0001FFA80F8E08DD0B3B8F1000F37D000BFE9
:1068B00000BF21680C3151E8001F21F4907021685D
:1068C0000C3141E80002002AF3D100BF00BF00BF35
:1068D0002168143151E8001F21F0010021681431B2
:1068E00041E80002002AF3D100BF202084F84200D2
:1068F0000020206300BF00BF21680C3151E8001F59
:1069000021F0100021680C3141E80002002AF3D187
:1069100000BF0220606341462046FFF779FEADE6E6
:1069200005F0800030B106F0800018B1204603F079
:106930005FF8A3E605F0400030B106F0400018B162
:10694000204602F0A4FE99E600BF97E611960008E3
:1069500010B504460CB9012010BDA06900B100E0DB
:1069600000BF94F8410028B9002084F84000204678
:1069700000F02AF8242084F841002068C06820F440
:1069800000502168C860204602F01CFF20680069A2
:1069900020F49040216808612068406920F02A00B6
:1069A000216848612068C06840F400502168C860D0
:1069B00000206064202084F8410084F84200002018
:1069C000606300BFC8E7000010B586B0044614211C
:1069D00001A8F9F7E1FD5A49206888424ED100BF6D
:1069E000002000905748006840F0100055490860AA
:1069F0000846006800F01000009000BF00BF00BF14
:106A0000002000904F481438006840F002004D49C3
:106A1000143908600846006800F00200009000BFCA
:106A200000BF00BF002000900846006840F0010051
:106A300008600846006800F00100009000BF00BF39
:106A400080200190022002900020039003200490F7
:106A50000720059001A93C48FDF7FAFA4FF40070B1
:106A60000190022002900020039003200490072050
:106A7000059001A93548FDF7EBFA5EE0344920683E
:106A800088425AD100BF002000902E48001F0068A5
:106A900040F480202B49091F08600846006800F474
:106AA0008020009000BF00BF00BF0020009025485C
:106AB0001438006840F00400224914390860084680
:106AC000006800F00400009000BF00BF4FF4406079
:106AD00001900220029000200390032004900720E0
:106AE000059001A91B48FDF7B3FA1B481B49086034
:106AF0004FF000604860002118488160C1604FF489
:106B0000806101610021416181614FF48071C16147
:106B1000002101624162FDF7A1F908B1FBF702FF14
:106B200000BF0E48E063846300BF002205212720D8
:106B3000FDF7F6FF2720FDF7DFFF06B010BD0000D0
:106B400000100140443802400004024000000240AE
:106B50000048004000080240286002401405002060
:106B600070B50546284602F0A3FD0446022C0DD060
:106B700004EBC400064901EB8000C06830B104EBAF
:106B8000C401034A02EB8101C868804770BD000060
:106B90008873002070B50546284602F089FD04463A
:106BA000022C0DD004EBC400064901EB80004068C4
:106BB00030B104EBC401034A02EB8101486880470D
:106BC00070BD00008873002000BFFEE710B50248CA
:106BD000FDF767FB10BD0000DC01002010B5024886
:106BE000FDF7C9FB10BD0000DC010020C16AB1F552
:106BF0002A0F02D10121C16205E0C16AB1F12A4F19
:106C000001D10821C1627047F8B505460020009007
:106C1000AC6B94F83D60394800681921B0FBF1F085
:106C20004FF47A71B0FBF1F0C0EBC00000EB8000D4
:106C3000009000BF009820B9206C40F02000206434
:106C400009E00098401E00902068006800F4007081
:106C5000B0F5007FEED000BF606B10B10020616B1B
:106C6000C863A06B10B10020A16BC86320680068E6
:106C700020F480602168086000206085606B10B19E
:106C80000020616B0865A06B10B10020A16B086546
:106C90002068006820F001002168086094F83D0039
:106CA00060280AD1202084F83D00002084F83E00AE
:106CB00020642046FDF7DAFA1EE006F028002828B6
:106CC00011D12068006840F0010021680860206848
:106CD000006840F48060216808600020206328205C
:106CE00084F83D0005E0202084F83D00002084F871
:106CF0003E002046FDF72CFCF8BD000014000020EB
:106D000001684969C1F3C01111B100210268116124
:106D1000704700000146074A0868904201D10020F0
:106D20007047054A0868904201D10120F8E7032026
:106D3000F6E7000000540040005800402DE9F04103
:106D4000044694F83D6094F83E70102F01D0402F17
:106D500007D1222E05D12068006820F40060216848
:106D6000086006F02800282805D10020206328208C
:106D700084F83D0010E02068406800F40060B0F541
:106D8000006F07D0602E05D0202084F83D00002041
:106D900084F83E00002020632068406800F4006012
:106DA000B0F5006F40D12068406820F40060216891
:106DB0004860606B90F83500012814D04848616B3A
:106DC0000865606BFCF712FF00285BD02068006844
:106DD00020F0010021680860202084F83D00606BED
:106DE000016D88474EE03E48A16B0865A06BFCF73B
:106DF000FDFE002846D020684069C0F3801030B105
:106E000020680069616A0870606A401C60622068DE
:106E1000006820F0010021680860202084F83D000F
:106E2000A06B016D88472DE094F83D0060281AD1D1
:106E3000202084F83D000020206420684069C0F3D1
:106E4000801030B120680069616A0870606A401C77
:106E500060622068006820F0010021680860204618
:106E6000FDF704FA0EE020684069C0F3801030B1ED
:106E700020680069616A0870606A401C6062204690
:106E8000FDF766FB256C05F0010058B905F002001E
:106E9000022807D005F00400042803D005F00800FC
:106EA000082805D12068406820F4E0602168486027
:106EB00094F83D60206C00F0040004280ED1282EC8
:106EC0000CD10848E06200202063202084F83D00B7
:106ED000002084F83E002046FDF73CFCBDE8F08130
:106EE000096C00080000FFFF70B50446E56A608D7C
:106EF000042810D12068406820F480602168486030
:106F000020680069616A0870606A401C6062608D78
:106F1000401E60857FE0608D03281AD1206840689C
:106F200020F4806021684860042D07D0022D05D030
:106F30002068006820F4806021680860206800698B
:106F4000616A0870606A401C6062608D401E6085E6
:106F500061E0608D022854D1012D01D0102D06D1A1
:106F60002068006820F480602168086010E0042D2B
:106F700001D0022D06D12068006840F480602168AD
:106F8000086005E02068006840F40070216808602F
:106F900020680069616A0870606A401C6062608DE8
:106FA000401E608520680069616A0870606A401C44
:106FB0006062608D401E60852068406820F44070EB
:106FC00021684860202084F83D0094F83E00402865
:106FD00007D1002084F83E0020632046FDF706FC20
:106FE00019E0002084F83E00082D01D0202D02D1A8
:106FF0000020206301E0122020632046FDF7C4FB3F
:1070000009E020680069616A0870606A401C60627B
:10701000608D401E608570BD70B5044694F83D00DB
:1070200022287AD1E66A658D032D13D9206800697C
:10703000616A0870606A401C6062608D401E6085F5
:10704000608D032868D12068406820F48060216842
:10705000486061E0E06A022858D0012D01D0002D7F
:1070600054D1204600F0C4FCA0BB2068006820F486
:107070008060216808602068406820F4E060216832
:10708000486020680069616A0870606A401C60623C
:10709000608D401E6085202084F83D0094F83E00FD
:1070A000402807D1002084F83E0020632046FDF7E9
:1070B0009DFB31E0002084F83E00082E01D0202EF8
:1070C00002D10020206301E0122020632046FDF75A
:1070D0005BFB21E0FFE72068406820F4E060216866
:1070E000486020680069616A0870606A401C6062DC
:1070F000608D401E6085202084F83D00002084F8CB
:107100003E002046FDF724FA06E006E020684068CD
:1071100020F480602168486000BF70BD70B50446EF
:10712000E56A94F83D00212847D1608D50B1606A2E
:10713000007821680861606A401C6062608D401EB2
:1071400060853AE0082D16D0202D14D015F5803F2B
:1071500011D02068406820F4E06021684860112068
:107160002063002084F83E00202084F83D00204663
:10717000FDF724FB21E02068406820F4E0602168EE
:1071800048602068006840F40070216808600020B2
:107190002063202084F83D0094F83E00402806D16A
:1071A000002084F83E002046FDF73AFB05E0002071
:1071B00084F83E002046FDF701FB70BD2DE9F0414B
:1071C000044694F83D5094F83E70E66A208DB0BBBA
:1071D000212D3CD1082E16D0202E14D016F5803F3C
:1071E00011D02068406820F4E060216848601120D8
:1071F0002063002084F83E00202084F83D002046D3
:10720000FDF7DCFA44E02068406820F4E060216883
:1072100048602068006840F4007021680860002021
:107220002063202084F83D0094F83E00402807D1D8
:10723000002084F83E002046FDF7F2FA28E006E040
:10724000002084F83E002046FDF7B8FA20E0212D0A
:1072500003D0402F1CD1222D1AD1608D30B9206867
:10726000406820F480602168486011E094F83E0096
:10727000402803D1204600F0A5F909E0606A0078B3
:1072800021680861606A401C6062608D401E6085F4
:10729000BDE8F081416CC9B202681161416B11B166
:1072A000416BC96B21B9816B41B1816BC96B29B14C
:1072B0000168496841F4006102685160704738B55F
:1072C00090F83E20C16A036B90F83D40222C73D1A8
:1072D000046D64B9402A0AD100BF002400940468F8
:1072E000646900940468A469009400BF1AE1046D05
:1072F000C4B90469B4F5404F14D100BF0024009410
:107300000468646900940468A469009400BF00BF25
:107310000468246844F4807405682C60046D641C5F
:107320000465FFE0448D8CB900BF0024009404681C
:10733000646900940468A469009400BF00BF0468F5
:10734000246844F4007405682C60DDE0448D012C51
:1073500072D111F5803F30D10468246824F4806430
:1073600005682C600468646804F40064B4F5006F78
:1073700010D10468246824F4806405682C6000BF80
:10738000002400940468646900940468A46900946B
:1073900000BFB9E000BF0024009404686469009451
:1073A0000468A469009400BF00BF0468246844F422
:1073B000007405682C60A7E0A9E0082923D02029E3
:1073C00021D0122B01D101291DD104290AD0022973
:1073D00008D0102906D00468246824F48064056865
:1073E0002C6005E00468246844F4806405682C601F
:1073F00000BF002400940468646900940468A469D0
:10740000009400BF80E00468246824F48064056868
:107410002C6000BF00240094046864690094046830
:10742000A469009400BF00BF0468246844F4007499
:1074300005682C6068E0FFE7448D022C3BD10429ED
:1074400010D002290ED010290CD00468246824F42E
:10745000806405682C600468246844F4006405684E
:107460002C6005E00468246844F4806405682C609E
:107470000468646804F40064B4F5006F10D111F579
:10748000803F07D0012905D0082903D0102901D059
:10749000202905D10468646844F4805405686C6050
:1074A00000BF002400940468646900940468A4691F
:1074B000009400BF28E00468246844F480640568F0
:1074C0002C600468646804F40064B4F5006F10D1A3
:1074D00011F5803F07D0012905D0082903D01029D4
:1074E00001D0202905D10468646844F480540568FB
:1074F0006C6000BF00240094046864690094046810
:10750000A469009400BF00BF002404650AE000BF26
:10751000002400940468646900940468A4690094D9
:1075200000BF00BF38BD90F83E1040290ED1016D5C
:1075300029B9416C01F0FE010268116141E0416C22
:10754000C9B241F00101026811613AE00169B1F587
:10755000804F20D190F83D10212905D1416C01F0D8
:10756000FE010268116105E0416CC9B241F0010100
:1075700002681161416B11B1416BC96B21B9816B1B
:10758000F9B1816BC96BE1B10168496841F40061EF
:107590000268516015E0016D41B9416C01F4407120
:1075A000F02242EAE111026811610AE0016D01294D
:1075B00007D1416C01F44071F12242EAE111026805
:1075C0001161704770B5044694F83D50206D98B92C
:1075D000E06C012807D1A06CC0B221680861206D61
:1075E000801C206550E0A06CC0F307202168086172
:1075F000206D401C206547E0206D012807D1A06C5C
:10760000C0B221680861206D401C20653CE0206DFF
:10761000022836D1222D09D12068006840F48070FC
:1076200021680860206D401C20652DE0608D60B1F0
:10763000212D0AD1606A007821680861606A401CC7
:107640006062608D401E60851EE0608DE0B9212D76
:107650001AD12068406820F4E06021684860206802
:10766000006840F40070216808600020206320203A
:1076700084F83D00002084F83E002046FDF7D0F855
:1076800002E02046FFF73CFB70BD418D49B1016827
:107690000969426A1170416A491C4162418D491E63
:1076A0004185704770B5044694F83D50608DD8B15F
:1076B00020680069616A0870606A401C6062608DC1
:1076C000401E6085608D78B92A2D0DD120684068F4
:1076D00020F480602168486022202063282084F8FC
:1076E0003D002046FDF744F970BD418D49B1416A26
:1076F000097802681161416A491C4162418D491E45
:107700004185704770B5044694F83D50608DD8B1FE
:10771000606A007821680861606A401C6062608D60
:10772000401E6085608D78B9292D0DD12068406894
:1077300020F480602168486021202063282084F89C
:107740003D002046FDF72EF970BDF8B504460D4604
:10775000002794F83D0000F0280028281CD120685C
:10776000406820F4806021684860C5F3800000B95B
:107770000127C5F3C01010B9A08986B201E0208BA3
:1077800086B200BF002084F83C0000BF3246394674
:107790002046FCF785FD0FE000BF00200090206828
:1077A0004069009020688069009000BF00BF00BF62
:1077B000002084F83C0000BFF8BD000070B504460E
:1077C00094F83D50E66A082E01D0202E1FD1282DB6
:1077D0001DD12348E0622068406820F4E060216801
:1077E00048606FF48060216848612068006820F478
:1077F00080602168086000202063202084F83D001C
:10780000002084F83E002046FCF7A4FF26E0212D4E
:1078100020D11348E06221202063202084F83D001D
:10782000002084F83E002068406820F4E060216871
:1078300048606FF48060216848612068006820F427
:107840008060216808602046FFF75AFA2046FDF75D
:10785000A9F803E06FF480602168486170BD000002
:107860000000FFFF38B5044694F83D50206840689A
:1078700020F4E0602168486000BF0020009020688C
:10788000406900902068006840F0010021680860AD
:1078900000BF00BF2068006820F480602168086095
:1078A0002068406800F40060B0F5006F42D1222DDE
:1078B00001D02A2D1FD1A06B006840686085608DC3
:1078C00018B1206C40F0040020642068406820F467
:1078D000006021684860A06BFCF79CF9012829D062
:1078E0004148A16B0865A06BFCF780F910B3A06B51
:1078F000016D88471EE0606B006840686085608DA0
:1079000018B1206C40F0040020642068406820F426
:10791000006021684860606BFCF77CF9012809D0A1
:107920003148616B0865606BFCF760F910B1606B02
:10793000016D8847608D18B320684069C0F38000EE
:1079400048B120680069616A0870606A401C606222
:10795000608D401E608520684069C0F3801048B18A
:1079600020680069616A0870606A401C6062608D0E
:10797000401E6085608D18B1206C40F004002064CA
:10798000206C18B12046FFF7D9F92BE02A2D07D13A
:1079900000202063282084F83D002046FCF7E8FF03
:1079A00094F83D0028280DD11048E06200202063A3
:1079B000202084F83D00002084F83E002046FCF79B
:1079C000C9FE0FE0206B222801D0222D0AD1002011
:1079D0002063202084F83D00002084F83E002046EB
:1079E000FCF7C6FF38BD0000096C00080000FFFF6F
:1079F00008B5014600200090104800681922B0FB2D
:107A0000F2F04FF47A72B0FBF2F000EB80000090DD
:107A100000BF0098401E0090009828B9086C40F004
:107A200020000864012008BD0868006800F40070A8
:107A3000B0F5007FEDD00020F5E700001400002035
:107A4000F0EE400AF6EE001A60EEA11AB0EE611AEE
:107A5000B0EE600A10EE100A0C49A1EB600000EED7
:107A6000100A21EE002AF7EE081A42EE401A61EEE3
:107A7000801AB0EE610A21EE002AF7EE081A42EEF3
:107A8000401A61EE801AB0EE610A7047DF59375F25
:107A9000B0EE401A10B99FED1D0A704790ED062A0E
:107AA000D0ED012AB0EE410A02EE620A90ED072AFB
:107AB000D0ED022AF0EE400A42EE620A10EE901A71
:107AC0004FF07F42B2EB410F01D1012200E00022D2
:107AD0000AB1F0EE410A90ED060A90ED042A20EE7C
:107AE000020A90ED032A00EE820A90ED072AD0EDFB
:107AF000052AF0EE401A42EE221A90ED060A80EDB9
:107B0000070AC0ED060AB0EE610AC6E700000000F1
:107B100010B52DED068B0446B0EE409AF0EE609A5B
:107B200014B9BDEC068B10BDC4ED009A9FED3A0A66
:107B300084ED060A9FED380A84ED070A94ED000AE9
:107B4000B5EEC00AF1EE10FA14D8B7EE000A84EDD3
:107B5000030A9FED310A84ED040A9FED2F0A84ED9C
:107B6000050A9FED2D0A84ED010A9FED2B0A84ED95
:107B7000020AD6E794ED000A89EE00AA9FED270AD3
:107B8000C0EE0A0AF0EE60AAB0EE6A0A02F0F2FC59
:107B9000B0EE408A9FED220A02F020FCF0EE000ACF
:107BA00060EE200AB7EE000A00EE880AF0EE408A86
:107BB00048EE088A28EE080AC0EE280AC4ED030A37
:107BC00094ED030AF0EE000A20EE200A84ED040A88
:107BD00094ED030A84ED050AB7EE000A18EE080AD0
:107BE000F0EE000A20EE200AC0EE280AC4ED010AD9
:107BF0009FED0B0A02F0F2FBF0EE000A60EE200AA5
:107C0000B7EE000A00EEC80A08EE080AC0EE280A1D
:107C1000C4ED020A00BF84E700000000DB0F49400A
:107C2000DB0F493F00B50346F0EE403A13B99FED34
:107C3000140A00BD93ED030AD3ED040A30EE200AC6
:107C4000D3ED050A30EE200A83EE803A13EE100AD7
:107C5000C0F3C751FF2901D0012100E0002121B16B
:107C600083ED063A83ED073A03E0C3ED063AC3ED30
:107C7000073AB0EE630A1846FFF70AFFD9E700009B
:107C80000000000010B50446022C02DB4FF0FF306C
:107C900010BD0F4850F8240008B10020F8E7482034
:107CA000FAF758FB0A4941F82400084650F8240026
:107CB00010B94FF0FF30EBE7054951F82400482197
:107CC000F8F76AFC024850F8240004700020DFE74F
:107CD000C80000202DE9FF41054625B96FF00100DD
:107CE00004B0BDE8F081287800F08AF8064616B99D
:107CF0006FF00300F4E7B41C6F88A7F201200B2893
:107D00006BD2DFE800F0060708092526272845463C
:107D1000470000BF00BF00BF4FF400700090082074
:107D20008DF80400002010E034F81010C1F3072291
:107D30000DF1050101F8102014F81020012101EBCC
:107D400040030DF10501CA54401C0428ECDB47E058
:107D500000BF00BF00BF40F2FF10009008208DF868
:107D60000400042011E034F81010C1F30723011FB0
:107D70000DF1050202F8113014F81020012303EB75
:107D800041030DF10501CA54401C0828EBDB27E034
:107D900000BF00BF40F2FF20009008208DF80400D3
:107DA00000BF12E034F81010C1F30723A0F108015E
:107DB0000DF1050202F8113014F81020012303EB35
:107DC00041030DF10501CA54401C0B28EADB0021D8
:107DD0008DF80B108DF80C1002E04FF0FF307FE7AC
:107DE00000BF28780121FAF7D9F928786946FAF70F
:107DF000C5F908B9002073E74FF0FF3070E70000C5
:107E00000146022901DB00207047024850F821009A
:107E1000FAE70000C8000020014621B1012905D081
:107E2000022909D105E042F2107070474FF48040FA
:107E3000FBE747F23050F8E74FF0FF30F5E7024636
:107E400021B1012903D0022916D10AE000BFB2F501
:107E5000007F05DDB2F5027F02DA501E40B27047A6
:107E60000BE0B2F5017F06DD40F20B20824202DA20
:107E7000501E40B2F3E700E000BF00BF4FF0FF30FC
:107E8000EDE770B505460DB9002070BD2878FFF705
:107E9000B7FF04460CB90020F7E700210AE004F11F
:107EA000180252F8210020B142886B889A4200D112
:107EB000EBE7491C94F844008842F0DC0020E4E73A
:107EC00020B1012805D0022809D105E09FED050A5F
:107ED0007047B3EE030AFBE7B7EE000AF8E7B7EE28
:107EE000000AF5E70000104270B5054615B96FF0BD
:107EF000010070BD2878FFF7C5FE10B14FF0FF30CC
:107F0000F7E72878FFF77CFF044614B94FF0FF30FD
:107F1000EFE7002110E004F1180050F8210050B103
:107F200004F1180050F8210040886A88904202D17C
:107F30006FF00200DDE7491C94F844008842EADC57
:107F400094F844000B2802DB4FF0FF30D1E75020BB
:107F5000FAF700FA064616B94FF0FF30C9E728686D
:107F6000306068687060282106F11800F8F714FB8B
:107F7000697928208155698828780322F9F7D2FF8A
:107F800028B13046FAF750F94FF0FF30B1E794F8D6
:107F9000441004F1180040F8216094F84400401C9B
:107FA00084F844000020A4E72DE9F0472DED028B72
:107FB0000446B0EE408A2CB96FF00100BDEC028B94
:107FC000BDE8F0872078FFF71BFF054615B96FF075
:107FD0000300F3E7B7EE000AB4EEC08AF1EE10FA40
:107FE00003DDB7EE000AB0EE408ABFEE000AB4EE41
:107FF000C08AF1EE10FA03D2BFEE000AB0EE408A5A
:10800000607918B1B1EE480AB0EE408A2046FFF719
:1080100038FF074617B96FF00300CFE72179608872
:10802000FFF70DFF0646002E02DA4FF0FF30C5E7DE
:1080300005F102082079FFF7EFFE00EE100AB8EE16
:10804000C00A20EE080ABDEEC00A10EE100A0FFAB0
:1080500080F928F816900020B0E72DE9F04387B0AA
:10806000054625B96FF0010007B0BDE8F083287818
:10807000FFF7C6FE064616B96FF00300F4E74FF0AF
:1080800000093AE006F1180050F8294094B36088DE
:10809000698888422FD16988287800236A46F9F7D1
:1080A00061FEA8B1FAF767FA07468846D4E90831B5
:1080B000FA1A68EB01004FF47A7300219A1A814191
:1080C00003D200202076001FCEE74FF0FF30CBE731
:1080D00001202076FAF74FFAC4E9080169462046E4
:1080E00000F0C2FA04F108018EC904F12C008EC020
:1080F0000020B9E7FFE709F1010996F84400484577
:10810000C0DC6FF00300AFE710B50F480F490860FF
:108110000320486000210D488160C1604FF41021A8
:1081200001614FF4001141610021017641768176B1
:108130000121C176002101774177FBF7E9F908B108
:10814000FAF7F0FB10BD0000006400408C01002035
:1081500010B50E480E4908600320486000210C4805
:108160008160C1604FF4102101614FF40011416141
:108170000021017641768176C17601774177FBF760
:10818000C7F908B1FAF7CEFB10BD00000068004047
:10819000B401002008B500BF002000901A48006814
:1081A00040F40010184908600846006800F4001008
:1081B000009000BF00BF00BF00200090084600688C
:1081C00040F4800008600846006800F480000090D9
:1081D00000BF00BF002207210C20FCF7A1FC0C20EF
:1081E000FCF78AFC002205213A20FCF799FC3A2092
:1081F000FCF782FC002205213B20FCF791FC3B2090
:10820000FCF77AFC08BD00003038024010B5064A81
:108210000021064802F081FF05490860054A002157
:10822000054802F07AFF10BD38EB0008518F0008B6
:1082300000000020DCEB00080993000800B587B0BF
:10824000142102A8F8F7A8F900BF00200190724895
:10825000006840F00200704908600846006800F0BD
:108260000200019000BF00BF00BF0020019008463F
:10827000006840F0010008600846006800F0010056
:10828000019000BF00BF00BF0020019008460068B9
:1082900040F0080008600846006800F008000190FF
:1082A00000BF00BF00BF002001900846006840F0FA
:1082B000040008600846006800F00400019000BF58
:1082C00000BF00BF002001900846006840F48070A5
:1082D00008600846006800F48070019000BF00BF8D
:1082E00000BF002001900846006840F020000860B0
:1082F0000846006800F02000019000BF00BF00BFEA
:10830000002001900846006840F0800008600846A0
:10831000006800F08000019000BF00BF00BF002097
:1083200001900846006840F0400008600846006878
:1083300000F04000019000BF00BF002240213748FC
:10834000FBF788FF012210213548FBF783FF01224C
:1083500011463448FBF77EFF402002900120039035
:108360000490059002A92D48FBF772FE08200290A8
:108370004FF4041003900120049002A92748FBF752
:1083800067FE012002904FF4041003900120049036
:1083900002A92348FBF75CFE102002900120039005
:1083A0000490059002A91E48FBF752FE302002906F
:1083B0004FF4041003900120049002A91A48FBF71F
:1083C00047FE0120029003900490059002A91548F1
:1083D000FBF73EFE002205210620FCF7A1FB06204C
:1083E000FCF78AFB002205210920FCF799FB0920F4
:1083F000FCF782FB002206210A20FCF791FB0A20F1
:10840000FCF77AFB002206211720FCF789FB1720D6
:10841000FCF772FB07B000BD303802400018024084
:1084200000000240000402400008024010B50B4862
:108430000B4908600B484860002109488160C16011
:108440004FF480410161002141618161C16101629C
:10845000FCF798F808B1FAF765FA10BD005400402F
:10846000DC010020A086010010B50B480B49086014
:108470000B484860002109488160C1604FF4804189
:108480000161002141618161C1610162FCF77AF8FB
:1084900008B1FAF747FA10BD00580040300200203A
:1084A000A086010010B50F480F4908604FF4827094
:1084B000486000210C488160C160022101610121F6
:1084C0004161490281611821C1610021016241625B
:1084D00081620A21C162FCF71FFF08B1FAF722FA94
:1084E00010BD0000003001408402002010B50F488C
:1084F0000F4908604FF48270486000210C48816089
:108500004FF40061C1600221016101214161490212
:1085100081610021C1610162416281620A21C162FF
:10852000FCF7FAFE08B1FAF7FDF910BD003800407B
:10853000DC02002000B587B01C216846F8F72CF853
:1085400015481649086000204860002113488160E2
:1085500041F28831C160002101618161FDF7C0FDF8
:1085600008B1FAF7DFF90D48FDF795FF08B1FAF702
:10857000D9F9602000900020019002900490002220
:1085800069460648FDF705FF08B1FAF7CBF903483D
:10859000FDF7CEFE07B000BD004401403C040020C2
:1085A0001CB50020009001900E480F490860002083
:1085B000486000210C48816040F2E731C160002131
:1085C0008161FDF78DFD08B1FAF7ACF9002000904C
:1085D000019069460448FDF729FD08B1FAF7A2F9B0
:1085E0001CBD000000140040F403002010B50B482F
:1085F0000B4908604FF4E130486000210848816071
:10860000C16001610C21416100218161C161FEF7FE
:108610009FF908B1FAF786F910BD0000001001407B
:108620008404002010B50C480C4908600C484860D0
:1086300000210A4881604FF40051C160C9100161F6
:108640000C21416100218161C161FEF781F908B10E
:10865000FAF768F910BD000000480040CC04002083
:10866000A086010000BFFEE72DE9F0412DED068B4D
:1086700004460D46A87B697B40EA0126297CE87BFD
:1086800041EA002000B209EE100AA97C687C41EAA8
:10869000002007B22079FFF7BFFB80462079FFF763
:1086A0000FFCB0EE408A00EE106AB8EE400A9FED73
:1086B0004E1AC0EE010A9FED4D0A20EE800AF0EE40
:1086C000408AB8EEC90AF0EE409A17FB08F000EEB7
:1086D000100AB8EEC00ADFED460A80EE201AB0EEAE
:1086E00041AAA07970B3B4F84010701AB0F5805F59
:1086F00003DD616C491E616405E010F5805F02DAFC
:10870000616C491C6164A4F84060B0EE680AD4ED65
:10871000110AB8EEE01ADFED351AF0EE400A41EE2C
:10872000210A80EE881A84ED121AD4ED120AC4EDE3
:10873000020AC9EE880AC4ED030A6AEE080AC4ED0B
:10874000040A0DE000206064A4F840609FED290A4F
:1087500084ED120AC4ED028AC4ED039A84ED04AAE2
:108760002820005DA8B307E094ED020ADFED1F0AA0
:1087700030EE200A84ED020A94ED020AB5EEC00A3A
:10878000F1EE10FAF0D307E094ED020ADFED170ADC
:1087900030EE600A84ED020A94ED020ADFED130A5E
:1087A000B4EEE00AF1EE10FAEEDA94ED020ADFED33
:1087B0000F0A30EEC00A84ED020A94ED030AB1EE0E
:1087C000400A84ED030A94ED040AB1EE400A84EDF8
:1087D000040AE87C00EE100AB8EE400A84ED050AAF
:1087E000BDEC068BBDE8F08100000046DB0FC94000
:1087F000000080460000000000BFFEE710B52DED30
:108800000C8B0446B0EE40DAF0EE60AAB0EE41BA4E
:10881000F0EE619A1DEE100A01F05FF970B11AEEE8
:10882000900A01F05AF948B11BEE100A01F055F90F
:1088300020B119EE900A01F050F920B994ED060A22
:10884000BDEC0C8B10BD606890ED070AB0EE401ACD
:10885000F0EE6A0AB0EE4D0AF9F763FFF0EE40BAA7
:10886000606890ED000A20EE2BCA606890ED000A67
:1088700060EE2ADAB0EE6D0A04F11C00FFF708F989
:10888000B0EE40AA2078B0B1012802D0022815D15C
:108890000EE094ED020AF0EE400AB0EE690A01F033
:1088A00045FED4ED050A7AEE600AC0EE808A05E046
:1088B000F0EE4B8A02E0DFED388A00BF00BFC4ED66
:1088C00004BA84ED05AA18EE900A01F006F918B969
:1088D0009FED310AF0EE408A606890ED010A20EECB
:1088E0000C0AD0ED030AB0EE408A08EEE08A94ED5F
:1088F000030AB0EE409A0CEE299A606890ED020AE5
:1089000060EE09CA606890ED020ADFED240AB4EE59
:10891000E00AF1EE10FA1CDD19EE100A01F0DDF8A4
:10892000B8B138EE2C0AB0EEC00A6068D0ED050A86
:10893000B4EEE00AF1EE10FA0BD8B0EEC90A6068A6
:10894000D0ED040AB4EEE00AF1EE10FA01D884ED9D
:10895000039A38EE2C0AB0EE408A18EE100A01F0A5
:10896000BCF8B0B1606890ED050ADFED0C0AB4EE1A
:10897000E00AF1EE10FA0ADD606890ED050AF0EE0B
:10898000400AB0EE480AF8F7C5FEB0EE408A84ED22
:10899000068A94ED060A53E700000000BD378635CD
:1089A00070B52DED028B04460E46F0EE408A15465A
:1089B00024B94FF0FF30BDEC028B70BD95ED010A7C
:1089C00010EE101A084601F088F810B94FF0FF3089
:1089D000F1E795ED020A10EE101A084601F07DF855
:1089E00010B94FF0FF30E6E795ED030A10EE101ACC
:1089F000084601F072F810B94FF0FF30DBE795ED53
:108A0000040A10EE101A084601F067F810B94FF08A
:108A1000FF30D0E795ED050A10EE101A084601F078
:108A20005CF810B94FF0FF30C5E76560B7EE000A9B
:108A300080EE288A18EE100A01F04FF810B184ED8C
:108A4000028A02E04FF0FF30B5E7606890ED060A59
:108A5000F0EE400AB0EE680A04F11C00FFF758F887
:108A60002670204600F002F80020A4E710B5044666
:108A700014B94FF0FF3010BD9FED0B0A84ED030ACF
:108A80009FED090A84ED040A9FED070A84ED050AAB
:108A90009FED050A84ED060A9FED030A04F11C0010
:108AA000FFF7C0F80020E6E7000000001C4A12684B
:108AB000526942F040021A4B1B685A61194A926A85
:108AC00042F01002174B9A62174A1268126822F09D
:108AD0000102154B1B681A6007E0134A12681268FE
:108AE00022F00102104B1B681A600F4A12681268CC
:108AF00002F00102002AF0D10C4A0B4B1B689A606D
:108B0000094A1268D060084A12685160064A126821
:108B1000126842F00102044B1B681A6070470000A3
:108B2000CC040020006002401405002004480040EE
:108B300010B5044613480068C06820F4005011497D
:108B40000968C86010480068006820F001000E49FC
:108B5000096808600C4800684460032003F0C3FA09
:108B600009480068006840F001000749096808608A
:108B700004480068C06840F4005002490968C860B1
:108B800010BD0000CC0400201405002070B505467F
:108B9000AC6B2068406820F0030021684860606D7D
:108BA00040F010006065012084F851002046FCF779
:108BB00097FB70BD70B50446A56B2846FCF760FEB8
:108BC00070BD70B50446A56B2846FDF7BFF970BDB2
:108BD00070B50446A56B2846FDF7F0F970BD70B579
:108BE0000546AC6BFBF73CFB06462868006800F4C2
:108BF0008070B0F5807F2BD02068406820F0200086
:108C000021684860A06850B96068B0F5827F06D1DD
:108C10002068406820F003002168486005E0206873
:108C2000406820F0010021684860324664212046F7
:108C300000F087F808B1202060650020E08701205F
:108C400084F85100606D18B12046FCF749FB70BDF7
:108C50002046FCF7F9FD00BFF9E7F8B50546AC6B17
:108C6000FBF7FEFA06462868006800F48070B0F54D
:108C7000807F2DD02068406820F020002168486067
:108C80002068406820F00200216848603246642174
:108C9000204600F0A1F818B1606D40F0200060653A
:108CA000A06850B900BF002000902068C068009004
:108CB00020688068009000BF00BF0020E08601208F
:108CC00084F85100606D18B12046FCF709FBF8BD2F
:108CD0002046FDF725F900BFF9E770B50546AC6BF6
:108CE000FBF7BEFA06462868006800F48070B0F50D
:108CF000807F21D02068406820F0200021684860F3
:108D000032466421204600F067F818B1606D40F0EB
:108D1000200060652068406820F0030021684860FA
:108D20000020E086E087012084F85100606D18B1D2
:108D30002046FCF7D5FA70BD2046FDF723F900BFA9
:108D4000F9E7F8B504460E4615466068B0F5827F2F
:108D50000DD1A068B0F5004F03D0A068B0F5806FCA
:108D600005D12068006820F0400021680860606834
:108D7000B0F5827F1FD1A068B0F5806F0DD033466B
:108D8000002280212046009500F076F808B3606D3F
:108D900040F0200060650320F8BD33460022012129
:108DA0002046009500F068F898B1606D40F0200012
:108DB00060650320F0E7334600220121204600953C
:108DC00000F05AF828B1606D40F020006065032083
:108DD000E2E70020E0E700007CB504460E461546B9
:108DE0003346012202212046009500F045F828B1C3
:108DF000606D40F02000606503207CBD164800686F
:108E00001821B0FBF1F01549B0FBF1F04FF47A7185
:108E1000484301906068B0F5827F0DD1334600224F
:108E200080212046009500F027F898B1606D40F051
:108E3000200060650320E0E700BF019800B908E06A
:108E40000198401E019020688068C0F3C01000287F
:108E5000F3D100BF0020D0E71400002040420F00F3
:108E60000146044A0868904201D10020704703205F
:108E7000FCE70000003001402DE9F84F04460D46A4
:108E800090461E46DDF82890FBF7EAF9A0EB0900B2
:108E9000371AFBF7E5F982462C480068C0F3CB305F
:108EA0007843009046E0701C002843D0FBF7D8F9C7
:108EB000A0EB0A00B84200D2A7BB2068406820F0AF
:108EC000E000216848606068B0F5827F0DD1A0683D
:108ED000B0F5004F03D0A068B0F5806F05D12068D1
:108EE000006820F0400021680860A06AB0F5005FCB
:108EF0000DD100BF2068006820F400502168086090
:108F00002068006840F400502168086000BF01201C
:108F100084F8510000BF002084F8500000BF0320F7
:108F2000BDE8F88FFFE7009808B9002702E0009835
:108F3000401E0090206880682840A84201D101208E
:108F400000E000204045AED10020E9E714000020F9
:108F500070B5054602F0DBF8044602F03AF970BD40
:108F600010B5FBF739FD04F08FFC012801D003F0A8
:108F7000ABFD10BD00B593B0302107A8F7F70CFB8F
:108F8000142102A8F7F708FB00BF00200190244835
:108F9000006840F08050224908600846006800F0F0
:108FA0008050019000BF00BF00BF002001901D480D
:108FB000006840F480401B4908600846006800F4DF
:108FC0008040019000BF00BF01200790000408907E
:108FD00002200D9041050E9106210F91A8211091BC
:108FE000022111910421129107A8FBF72BFF08B170
:108FF000F9F798FC0F2002900220039000200490C3
:109000004FF4A05005904FF480500690052102A81F
:10901000FBF7D8FD08B1F9F785FC13B000BD0000DF
:1090200040380240007000400348006840F470007F
:10903000014908607047000088ED00E010B5024863
:10904000FDF7BFF810BD0000F403002010B5026862
:109050002B4B98420ED0B0F1804F0BD0294B984249
:1090600008D0294B984205D0284B984202D0284B73
:10907000984203D122F070024B681A43204B984269
:1090800020D0B0F1804F1DD01E4B98421AD01E4BFD
:10909000984217D01D4B984214D01D4B984211D0C6
:1090A0001C4B98420ED01C4B98420BD01B4B984245
:1090B00008D01B4B984205D01A4B984202D01A4B4D
:1090C000984203D122F44072CB681A4322F0800305
:1090D0004C6943EA04028B68C3620B688362084BE5
:1090E000984202D00A4B984201D10B69036303688E
:1090F00043F00403036001234361026010BD0000DC
:10910000000001400004004000080040000C004046
:10911000000401400040014000440140004801407B
:1091200000180040001C00400020004030B501F055
:109130001F05012404FA05F3046A9C430462046ACF
:1091400001F01F0502FA05F52C43046230BD000052
:1091500030B5026A056A25F0010505624368846935
:1091600024F0700424F003040D682C4322F0020262
:109170008D682A43104DA84200D103E00F4DA8424C
:1091800006D100BF22F00802CD682A4322F0040273
:10919000094DA84202D0094DA84207D123F480739B
:1091A00023F400734D692B438D692B434360846125
:1091B0004D684563026230BD00000140000401407B
:1091C00030B5026A056A25F01005056243688469B6
:1091D00024F4E04424F440740D6844EA052422F0A9
:1091E00020028D6842EA0512124DA84200D103E028
:1091F000114DA84207D100BF22F08002CD6842EA9B
:10920000051222F040020B4DA84202D00A4DA8429E
:1092100009D123F4806323F400634D6943EA850395
:109220008D6943EA8503436084614D68856302620A
:1092300030BD0000000001400004014030B5026A6A
:10924000056A25F4807505624368C46924F07004DA
:1092500024F003040D682C4322F400728D6842EA66
:109260000522124DA84200D103E0114DA84207D1BA
:1092700000BF22F40062CD6842EA052222F4806237
:109280000A4DA84202D00A4DA84209D123F48053C6
:1092900023F400534D6943EA05138D6943EA05132E
:1092A0004360C4614D68C563026230BD0000014087
:1092B0000004014030B5036A056A25F48055056253
:1092C0004468C26922F4E04222F440720D6842EA26
:1092D000052223F400538D6843EA0533084DA84264
:1092E00002D0084DA84204D124F480444D6944EAD8
:1092F00085144460C2614D680564036230BD00009E
:10930000000001400004014070B5054601F062FC18
:109310001D4A00211D4801F000FF1D4908601D4A3B
:1093200000211D4801F0F9FE194948601B4A00213F
:109330001B4801F0F2FE1649886000220A21022033
:1093400001F0F6FC1249C86000223021022001F031
:10935000EFFC0F49486100220C21022001F0E8FCDB
:1093600001460B48816100221821022001F0E0FC37
:1093700001460748C16101F079FC01F0C8FE0446CE
:1093800001F027FF70BD000000EC0008A593000865
:10939000B476002024EC0008E994000848EC0008AA
:1093A000919500082DED048B01F0FBFB064605F0BE
:1093B00067F841EC190B9FED3F0B53EC102B04F0B9
:1093C00057FE41EC180B05F017F80546002001F098
:1093D00098FB01F0D9FB044638493948F8F7F4F90D
:1093E0003748F8F7CDF9B0EE408A36493648F7F7F6
:1093F000DFF93348F8F7C4F9F7EE000A80EE801A77
:10940000B0EE418A314AB0EE480A00213048FFF7F9
:10941000C7FA0020F8F7FCFF4BE02C44F8F770FB8C
:10942000F8F79AF9F8F7A4F9F8F7BAF9F8F7C4F9E0
:1094300001F0D0FB2248F8F765FA2148F8F7C4FAA2
:10944000204B1F4A1C32A2F10C011F48F7F7C0FA4B
:109450001D492048F7F714F901F008FC184890ED71
:109460000A0AF0EE400ADFED1C1A9FED1B1A9FED71
:109470001B0A1748FFF7C2F9B0EE408A0020F8F740
:109480006FFF1748134B0ECB0C300EC018380C4B27
:109490001C330ECB0EC01349486901F0D9FC1149A9
:1094A00000231A4648690E4901F090FC204601F05D
:1094B00037FBB2E70000000000407F40C07400208E
:1094C000F07300205474002040740020BCEB0008AE
:1094D0006C74002060740020000000000000204236
:1094E000A8740020B47600202DED048B01F059FB08
:1094F000064604F0C5FF41EC190B9FED1E0B53EC23
:10950000102B04F0B5FD41EC180B04F075FF054677
:10951000002001F0F6FA01F037FB0446F9F72AF9CA
:1095200006469FED160A31461548F9F75BFB1FE02A
:109530002C44144900231A464869134901F0B8FB2A
:1095400011490F48F9F747FC0E4900231A4688696C
:109550000E4901F0ADFB0A48F9F712FC0B49084827
:10956000F9F7E4F90648F9F7B3FB204601F0D8FA19
:10957000DEE700000000000000407F400000FA43EA
:10958000F0740020B476002090760020A8760020A9
:109590002DED048B01F005FB064604F071FF41EC54
:1095A000190B9FED150B53EC102B04F061FD41ECF2
:1095B000180B04F021FF0546002001F0A2FA01F08B
:1095C000E3FA044601F0FEF902F060FC13E02C44DB
:1095D0000B4A0C490C4802F015FC0C49886901F053
:1095E00037FC0A4900231A468869074901F0EEFB57
:1095F000204601F095FAEAE70000000000407F40B5
:10960000D8740020BF730020CC740020B4760020F2
:1096100070B50446A56B0020E8852846FCF7FAFFE4
:1096200070BD00BF00BF02680C3252E8002F22F468
:10963000907102680C3242E80013002BF3D100BF96
:1096400000BF00BF0268143252E8002F22F001016F
:109650000268143242E80013002BF3D100BF016B03
:1096600001290ED100BF00BF02680C3252E8002F62
:1096700022F0100102680C3242E80013002BF3D1F3
:1096800000BF202180F8421000210163704710B50F
:1096900004462068C06820F040002168C86020208F
:1096A00084F841002046FDF775FA002010BD000047
:1096B0000146044A0868904201D100207047022008
:1096C000FCE7000000480040F8B5044600250026ED
:1096D00094F84200222873D1A068B0F5805F0BD1C6
:1096E000206948B9A66A20684068C0F30800308045
:1096F000A06A801CA06214E0A56AA068B0F5805F33
:1097000003D0A06828B9206918B92068406828707B
:1097100004E02068406800F07F002870A06A401CC8
:10972000A062E08D401E80B2E085002846D120680E
:10973000C06820F020002168C8602068C06820F45C
:1097400080702168C8602068406920F001002168AD
:109750004861202084F8420000206063206B0128CB
:1097600026D10020206300BF00BF21680C3151E8E2
:10977000001F21F0100021680C3141E80002002A8E
:10978000F3D100BF2068006800F0100010280AD153
:1097900000BF0020009020680068009020684068AA
:1097A000009000BF00BFA18D2046FCF731FF02E012
:1097B0002046FDF7D5F90020F8BD01E00020FBE7C9
:1097C0000220F9E72DE9F84F04462068006920F4EB
:1097D0004050E1680843216808612169A068084396
:1097E00061690843E169084300902068C06849F254
:1097F0000C618843009908432168C860206840696B
:1098000020F44070A16908432168486176492068C6
:10981000884203D075492068884203D1FBF7AAFA31
:10982000814602E0FBF796FA8146E069B0F5004F09
:109830006CD102206168A0FB015003461920A9FBEE
:10984000007001462A463846F6F78EFD6421B0FBCB
:10985000F1F04FEA001A02206168A0FB01510B46AB
:109860001920A9FB00712A463846F6F77DFD83468C
:1098700002206168A0FB015003461920A9FB00717A
:109880002A463846F6F770FD6421B0FBF1F000EB94
:10989000C00101EB0010ABEB8000322101EBC000F6
:1098A0006421B0FBF1F000F0F8000AEB400A02205E
:1098B0006168A0FB015003461920A9FB0070014616
:1098C0002A463846F6F750FD834602206168A0FB21
:1098D000015003461920A9FB00712A463846F6F7C5
:1098E00043FD6421B0FBF1F000EBC00101EB00107F
:1098F000ABEB8000322101EBC0006421B0FBF1F042
:1099000000F007005044216888606AE00420616824
:10991000A0FB015003461920A9FB007001462A460E
:109920003846F6F721FD824604206168A0FB01500D
:1099300003461920A9FB007001462A463846F6F76F
:1099400013FD6421B0FBF1F000EBC00101EB00104E
:10995000AAEB8000322101EB00106421B0FBF1F092
:1099600000F0F00A04206168A0FB01700346192092
:10997000A9FB00513A462846F6F7F6FC6421B0FBF5
:10998000F1F00AEB001A04206168A0FB01510B46BC
:109990001920A9FB00712A463846F6F7E5FC8346F4
:1099A00004206168A0FB015003461920A9FB007048
:1099B00001462A463846F6F7D7FC6421B0FBF1F0A1
:1099C00000EBC00101EB0010ABEB8000322101EB9A
:1099D00000106421B0FBF1F000F00F00504421684A
:1099E0008860BDE8F88F00000010014000140140BD
:1099F000014691F84100212828D18868B0F5805FA0
:109A00000BD1086948B90A6A1088C0F308000B68CE
:109A10005860086A801C086205E00B6A581C0862DE
:109A200018780B685860C88C401E80B2C88458B93A
:109A30000868C06820F080000B68D8600868C068BB
:109A400040F040000B68D860002070470220FCE71F
:109A500010B500F009F80348FCF7F6FD0148F8F7E7
:109A6000D3FD10BDCC0400200448006800F02000A5
:109A700018B102480068014908607047004800407A
:109A800000BFFEE703B401984100009850EAC120EE
:109A900018BF04204A0D18BF40F0010040F2FF72C9
:109AA000B2EB515F08BF40F00200012808BF05205B
:109AB00002B070474100080218BF04200A0E18BF08
:109AC00040F001004FF07F4232EA010108BF40F050
:109AD0000200012808BF052070470146C1F3C750A6
:109AE000FF2801D0012070470020FCE702480068F1
:109AF000C0F30220704700000CED00E010B5002814
:109B000004DB0A07130E054A135406E00A07140E75
:109B1000034A00F00F031B1FD45410BD00E400E003
:109B200018ED00E0EFF305807047000010B54FF02E
:109B30000E402DED028BB0EE408A18EE104A00EB7D
:109B40004400B0F1506F4AD84FF0FC40B0EB440FE6
:109B500022D2B0EEC80AF7EE000A30EEC00AF6EEE6
:109B6000000A60EE208A18EE900A02F09DFA01EEDB
:109B7000100A14F0004F1DBFDFED2D0A9FED2D0AD6
:109B8000B1EE411ADFED2C0A08BF9FED2C0AF8EE6A
:109B9000001A21EE218A05E0DFED290A68EE088A25
:109BA000B0EE600A9FED271ADFED271A30EE080AA3
:109BB00048EE811A9FED251A08EEA11ADFED241A4E
:109BC00048EE811A9FED231A08EEA11A68EE281AB2
:109BD000BDEC028B01EE810A30EE200A10BD4FF081
:109BE000E440B0EB440F0CD918EE100AFFF762FF07
:109BF000042808BF00F02AFEB0EE480ABDEC028B34
:109C000010BD4FF07F40B0EB440F07D2B0EE480AD2
:109C1000BDEC028BBDE8104000F00ABE0120F6F753
:109C2000EAFCBDEC028BBDE8104000F007BE00006E
:109C30000000C9BF22AAFDB90000C93F22AAFD3910
:109C40000000000024FE1C3DC78AD83C1E67383D3A
:109C50001B93993DAFAA2A3E70B59B482DED020B90
:109C60002DED068B079D25F00044A04218DC974897
:109C7000844202DC0AD1069840B19DED060BBDEC92
:109C8000068B02B0BDE8704000F0AEBD002DCCBF29
:109C90009FED8F0B9FED900BBDEC068B02B070BD5E
:109CA0008F48A04215DD8F48A042D8BF4FF0FF3447
:109CB00058DD9DED060B51EC100BFFF7E3FE042879
:109CC00008BF00F0A5FD9DED060BBDEC068B02B0B4
:109CD00070BD9DED060B51EC100B00F0D5FECDE9EB
:109CE000060181489FED828BA0423CDD8248A04264
:109CF0001FDD00249FED82AB9DED060B53EC1A2B6C
:109D000051EC100B04F000F99DED060B41EC190B22
:109D100053EC1A2B51EC100B04F002FC53EC182BF3
:109D200004F03EFD53EC192B04F0A2F9CDE9060135
:109D300049E09DED060B012453EC182B51EC100B60
:109D400004F0E2F89DED060B41EC190B53EC182BD7
:109D500051EC100B04F024FD53EC192B04F088F99E
:109D6000CDE906012FE06848A0421FDD02249FEDE7
:109D7000689B9DED060B53EC192B51EC100B04F076
:109D8000CFFB53EC182B04F0BFF89DED060B41EC14
:109D9000180B53EC192B51EC100B04F001FD53EC94
:109DA000182B04F065F9CDE906010CE09DED060BDA
:109DB000032453EC102B9FED580B51EC100B04F0C7
:109DC00057F9CDE906019DED060B53EC102B51EC34
:109DD000100B04F0A5FB41EC180B53EC182B04F00E
:109DE0009FFB41EC190B4E480621B0EE490AF0EEFC
:109DF000690A784400F07CFC53EC182B51EC100BF2
:109E000004F08EFB41EC180B4648B0EE490AF0EE28
:109E1000690A0521784400F06BFC53EC192B51ECD6
:109E2000100B04F07DFB41EC100B51EC180B53ECC4
:109E3000102B002C0EDA04F067F89DED061B53EC96
:109E4000112B04F06DFB9DED061B53EC112B04F060
:109E50009BFC35E004F058F89DED061B53EC112BEC
:109E600004F05EFB41EC100B2F48784400EBC4007B
:109E700090ED001B51EC100B53EC112B04F090FCF7
:109E80009DED061B53EC112B04F08AFC41EC100BEA
:109E90002648784400EBC40090ED001B51EC100BF9
:109EA00053EC112B04F070FC41EC100B002DA2BF01
:109EB000BDEC068B02B070BD51EC100B03F0E6FF59
:109EC00041EC100B01E70000000010440000F07F9F
:109ED000182D4454FB21F93F182D4454FB21F9BFA0
:109EE0000000DC3F0000203E0000F33F00000000C7
:109EF000000000000000F03F0000E63F000000000E
:109F0000000000000000004000800340000000004E
:109F1000000000000000F83F000000000000F0BF5B
:109F2000E24E0000984E0000224E0000DA4D000084
:109F300070B56F4E2DED040B2DED048B82B0DDF866
:109F400024C0DDE907235C422CF000411C4341EAB8
:109F5000D474069D22F00040B44205D86C422C43D4
:109F600040EAD474B4420BD99DED081B9DED060B5D
:109F700002B0BDEC048B04B0BDE8704000F03EBC04
:109F8000ACF14054A4F17F641C430BD0022404EADA
:109F9000AC7444EAD27405439FED578B9FED582B68
:109FA00007D015E09DED060B51EC100B00F000FD05
:109FB00042E0002C11BF012C9DED060B02B0BDEC60
:109FC000048B04BF04B070BD022C38D0032C3BD0EE
:109FD0000B439FED4D1B9FED4E0B0AD0B14218D1A4
:109FE000B04209D121F0804120F0804009910790D2
:109FF0000FE0002A15DA10E0474B7B44002C08BF25
:10A0000093ED000B0DD0012C10D0022C17D0032C97
:10A010001AD0B0421DD1002A03DAB0EE410AF0EEA8
:10A02000610A02B0BDEC048B04B070BD93ED000B6F
:10A0300051EC100B03F02AFF41EC100BF1E7B0EEEE
:10A04000480AF0EE680AECE7B0EE420AF0EE620A67
:10A05000E7E7401A00159FED329B3C28C8BF8DED05
:10A06000000B17DCBCF1000FBCBF10F13C0F8DEDF5
:10A07000009B0FDB9DED080B53EC102B9DED060BA9
:10A0800051EC100B03F0F4FF00F0FEFC00F090FC2C
:10A09000CDE90001B4B1012C10D0022C9FED220BB0
:10A0A00053EC102B9DED000B51EC100B19D004F06C
:10A0B00077FB53EC182B04F073FBBDE7019880F09D
:10A0C000004001909DED000B53EC192B51EC100B4F
:10A0D00004F026F904BF0220F6F78DFA9DED000B7F
:10A0E0009FE704F05DFB53EC182B04F04DFBA3E756
:10A0F0000000F07F00000000182D4454FB210940AF
:10A10000182D4454FB2109C0182D4454FB21F9BFDC
:10A11000182D4454FB21F93F0A4D000000000000B7
:10A120000000000000000000075C143326A6A13CDC
:10A1300070B54FF068422DED048BF0EE408A18EEBA
:10A14000900AB0EE608A18EE101A02EB4003B3F1E9
:10A15000654F3CBF02EB4102B2F1654F7DD200BFBB
:10A16000C0F3C753C1F3C7529A1A1B2A09DD10F076
:10A17000004F14BF9FED830A9FED830ABDEC048B53
:10A1800070BD12F11A0F36DA11F0004F09D010F03D
:10A19000004F0CBF9FED7D0A9FED7D0ABDEC048B47
:10A1A00070BD88EE889A19EE100AFFF783FC042828
:10A1B00008BF00F04BFB18EE900AFFF77BFC05464A
:10A1C00018EE100AFFF776FC044619EE100AFFF7A6
:10A1D00071FC042D18BF052D08D1042C18BF052CC7
:10A1E00004D1002804BF0220F6F705FAB0EE490AB0
:10A1F000BDEC048B70BD4200B2EB410F3AD910F0B8
:10A20000004F19BFDFED630A9FED630ADFED630ABC
:10A210009FED630AB0EE481A0A46B1EE688A80F0F4
:10A220000041F0EE418A10460A1A5200B2F1807FD6
:10A2300034D2484010F0004FDFED5A1A9FED5A2AF1
:10A240001DBFBEEE001A70EEE10A30EE420AB6EE15
:10A25000001A08BF70EEA10A00E040E008BF30EE2F
:10A26000020AB0EE682A01EE482A08EE818AC2EEA0
:10A27000081A15E011F0004F04BF9FED4C0AF0EEF4
:10A28000400AD1D010F0004F19BFDFED490A9FED11
:10A29000490ADFED490A9FED490AC5E7C8EE881A69
:10A2A00021EEA11A9FED462ADFED462A41EE022A51
:10A2B0009FED452A01EE222ADFED442A41EE022AD3
:10A2C0009FED432ABDEC048B01EE222A21EE811A78
:10A2D00001EE020A30EE210A30EE200A70BD4FF086
:10A2E0007F42B2EB400F28BFB2EB410F09D2F0EE34
:10A2F000480AB0EE680ABDEC048BBDE8704000F07F
:10A300009ABA40EA01035B0008BF41F0FF410BD05D
:10A31000B2EB400F08BFB2EB410F08D120F08040F4
:10A3200008EE900A21F0804108EE101A18E7B2EB0F
:10A33000400F12BF5FEA410340F0FF4001F00041CF
:10A340003FF40EAFB2EB410F12BF5FEA400200F0E4
:10A35000004041F0FF413FF403AF4A0092EA40035E
:10A360003FF5FEAE002AACBF9FED1A0A9FED1A0A18
:10A3700068EE808A28EE008A18EE900A18EE101A0D
:10A38000EEE60000DB0FC9BFDB0FC93FDB0F494022
:10A39000DB0F49C00000C9BF22AAFDB90000C93FB8
:10A3A00022AAFD390060ED3EC30ACE37000000004E
:10A3B000000049C022AA7DBA0000494022AA7D3A85
:10A3C0002DAD65BD8FB8D53D0FB511BE61C84C3EF2
:10A3D000A8AAAABE0000804F0000802F10EE101A1D
:10A3E00008B5444A6846B2EB410F28D94FF0E64021
:10A3F000B0EB410F94BF00204FF0FF300090009869
:10A40000002861DB60EE000A10F0010F45D010F06B
:10A41000020FDFED391A9FED391A00EEE11ADFED78
:10A42000381A40EE811A21EEA01AF0EE400A40EEF2
:10A43000010A08BFF1EE600AB0EE600A08BD314BB8
:10A4400021F0004293423CD911F0004FDFED2E0A7B
:10A4500020EE201ADFED2D0A19BF31EE601A71EEE1
:10A46000200A31EE201A71EE600ABDEEE01A11EEFC
:10A47000100A9FED271A00F0030000EEC10A9FEDBD
:10A48000251A009000EEC10A9FED231A00EEC10AC2
:10A490009FED221A00EEC10AB1E79FED211A9FED50
:10A4A000210A10F0020F00EE810A9FED1F1A00EE44
:10A4B000801AB7EE000A00EE810A18BFB1EE400A1A
:10A4C00008BD00F0CBF99AE710EE100A4000B0F199
:10A4D0007F4F3CBFB7EE000A08BD07D14FF0010027
:10A4E000F6F789F8BDE8084000F0A8B9BDE80840D3
:10A4F00000F09EB9B61F927E336D4C39DA82083C6B
:10A50000A0AA2ABE490E494683F9223F0000004B0B
:10A510000000C93F00A0FD390020A2331A61342C8D
:10A52000B93AB2BACA9F2A3DDDFFFFBE10B52DED84
:10A53000028BB0EE608AF0EE408A18EE101A18EE28
:10A54000900A04F04FFA00F07040B0F1005F0CD0B8
:10A5500018EE100A20F00040C0F1FF40C00F02BF0B
:10A56000B0EE480ABDEC028B10BDB0EE680ABDEC3F
:10A57000028B10BD00B510EE101A2DED028B81B0CC
:10A580004D4A6846B2EB410F3CD94FF0E640B0EB84
:10A59000410F94BF00204FF0FF3000900098B0EEC4
:10A5A000408A00285FDB28EE080ADFED440A9FEDB1
:10A5B000441A00EE201ADFED430A40EE010A9FED37
:10A5C000421A00EE201ADFED410A10F0010F40EEB2
:10A5D000010A9FED3F1A00EE201A61EE000AB0EE6C
:10A5E000480A08EE200A02BF01B0BDEC028B00BD94
:10A5F000BFEE001A01B0C1EE000ABDEC028BB0EE56
:10A60000600A00BD334B21F00042934228D911F07B
:10A61000004FDFED310A20EE201ADFED300A19BFBE
:10A6200031EE601A71EE200A31EE201A71EE600AE6
:10A63000BDEEE01A11EE100A9FED291A00F003009A
:10A6400000EEC10A9FED271A009000EEC10A9FEDAF
:10A65000261A00EEC10A9FED251A00EEC10A9DE7F9
:10A6600000F0FCF89AE718EE100A4000B0F17F4FB6
:10A670000DD218EE100AFFF71DFA042808BF00F0EB
:10A68000E5F8B0EE480A01B0BDEC028B00BD09D17F
:10A690000120F5F7B0FF01B0BDEC028B5DF804EBD3
:10A6A00000F0CCB801B0B0EE480ABDEC028B5DF80A
:10A6B00004EB00F0BDB80000B61F927EBBE9223C5F
:10A6C0000C6D063B8A76CE3CACB5593D35A1083EB3
:10A6D00029AAAA3E490E494683F9223F0000004BB1
:10A6E0000000C93F00A0FD390020A2331A61342CBC
:10A6F00070B504462DED028B4D1E00EBC500B0EE8B
:10A70000408AF0EE608A90ED000B35F0060017D01D
:10A7100053EC182B51EC100B03F002FF41EC100B23
:10A720006D1E04EBC50090ED001B51EC100B53ECBB
:10A73000112B03F0E9FB41EC100B35F00600E7D1DB
:10A74000022D36D0042D1CD0062D1CBFBDEC028B73
:10A7500070BD53EC182B51EC100B03F0E1FE94ED9F
:10A760000A1B53EC112B03F0CFFB53EC182B03F017
:10A77000D7FE94ED081B53EC112B03F0C5FB41EC05
:10A78000100B53EC182B51EC100B03F0C9FE94ED99
:10A79000061B53EC112B03F0B7FB53EC182B03F003
:10A7A000BFFE94ED040B53EC102B03F0ADFB41EC1A
:10A7B000100B53EC182B51EC100B03F0B1FE94ED81
:10A7C000021B53EC112B03F09FFB53EC182B03F0EF
:10A7D000A7FE94ED001B53EC112B03F095FBBDEC91
:10A7E000028B41EC100B70BD10B553EC102B51ECEB
:10A7F000100B03F089FB41EC100B10BD10B553ECAE
:10A80000112B51EC100B03F07FFB41EC100B10BD32
:10A810009FED050B10B553EC102B51EC100B03F012
:10A820007FFE41EC100B10BD000000000000001086
:10A8300030EE000A704730EE200A7047DFED020A62
:10A8400080EEA00A70470000000000009FED020AA1
:10A8500020EE000A70470000000000102DE9F00112
:10A860004FF07F42B2EB410F9FBF4FF0FF310160CD
:10A87000BDE8F00170474FF0004242EA0123C1F306
:10A88000C752783A551112F01F0C434CCCF12006F8
:10A890007C44C1F3C752A2F178024FEA621204EB82
:10A8A000820254F8254008BFD2E9015612D05568FB
:10A8B00004FA0CF425FA06F73C43976805FA0CF500
:10A8C00027FA06F8D26807FA0CFCF24045EA0805B8
:10A8D0004CEA0206A4FB034CA5FB0352A6FB036350
:10A8E0001D449D4234BF012600261319334416B17E
:10A8F000934202D903E0934201D2012200E00022F8
:10A90000624402F1200C9206DC0C42EA443200EE72
:10A91000102A5B03DFED210AF8EEC01A00EE103AB0
:10A920004FEA9C1C11F0004FB8EE400AC0F800C07E
:10A9300020EE201A00EE105ADFED190AB8EE400A98
:10A9400020EE200A71EE810A70EE800A10EE902A45
:10A9500002F500626FF30B0200EE902A70EEE11A2E
:10A9600031EEC11ADFED101A30EE411A9FED0D0ADB
:10A9700020EE800A01EE210A9FED0C1A00EE810AFA
:10A9800004BFBDE8F0017047CCF180510160BDE823
:10A99000F001B1EE400A70477C4400000000003630
:10A9A0000000802C22AAFD29DB0FC92F0000C92F2F
:10A9B00010B541EC100BFFF74FF951EC100B10BD27
:10A9C00070470000074800680749B0FBF1F00749ED
:10A9D0000870044800684FF47A71B0FBF1F0044944
:10A9E000086070471400002040420F00B4000020AF
:10A9F000B80000202DE9F04707463E4656B900BF93
:10AA0000502080F31188BFF34F8FBFF36F8F00BFCB
:10AA100000BFFEE717480068864201D1002426E007
:10AA200001F0DEFB75691448D0F800801348D0F8B7
:10AA3000009001F0FFFB454501D04D4501D10224B6
:10AA400015E00F4885420BD1B06A38B996F860001E
:10AA5000012801D102240AE0032408E0022406E0D0
:10AA60000848854200D00DB9042400E001242046A6
:10AA7000BDE8F087180000201C0000202000002006
:10AA8000640A0020500A002082B0CDE9000121F0C4
:10AA9000004001909DED000B02B051EC100B70478F
:10AAA00000207047F9F7A4FFFEF764FAFDF7C6FB34
:10AAB000FDF770FBFDF728FBFDF74AFBFDF7F2FC05
:10AAC000FDF714FDFDF76CFDFDF7ACFDFDF732FD64
:10AAD000FDF7ACFCFDF7C8FCFDF788FD00F064F85D
:10AAE000FDF794FB00F092F800BFFEE770B5044656
:10AAF000049D601AEE1A7043561A90FBF6F0184443
:10AB000070BD70B50546FFF70DF810B16FF0050484
:10AB100004E0002415B1284601F088FC204670BDF1
:10AB2000F8B50646FEF7FEFF10B16FF005050FE021
:10AB3000002502F0B9FE00900098341A34B1E00FFD
:10AB400020B92146684601F09FFC01E06FF0030543
:10AB50002846F8BD10B502F097FE28B1012806D0AE
:10AB6000022803D102240AE0032408E000BF0548BC
:10AB70000068012801D1012400E0002400BF00BFCB
:10AB8000204610BD7000002010B5FEF7CBFF18B1B5
:10AB900002F090FE044602E002F086FE04462046E3
:10ABA00010BD4FF47A70704710B5FEF7BBFF10B1BF
:10ABB0006FF0050409E00648006820B90120044947
:10ABC0000860002401E04FF0FF34204610BD000073
:10ABD0007000002010B5FEF7A5FF10B16FF005045E
:10ABE00012E002F051FE20B1012809D0022806D15E
:10ABF00001E0012407E001F029FE002403E000BF8A
:10AC00004FF0FF3400BF00BF204610BD70B5FEF707
:10AC100089FF10B16FF005041FE01148006801289A
:10AC200019D100BF801F0021002804DB0A07130E82
:10AC30000C4A135406E00A07150E0B4A00F00F03E6
:10AC40001B1FD55400BF00BF02200549086001F05A
:10AC50009FFD002401E04FF0FF34204670BD00004E
:10AC60007000002000E400E018ED00E010B5FEF7F1
:10AC700059FF10B16FF0050418E002F005FE20B195
:10AC800001280FD002280CD109E0012402F0FEFFB8
:10AC9000012803D002F0F8FD00B9A41E05E000244D
:10ACA00003E000BF4FF0FF3400BF00BF204610BDDF
:10ACB0002DE9F84307460D4691461C463E464FF0A7
:10ACC0000008FEF72FFFE0B10EB105B114B16FF02F
:10ACD000030828E0002000906A462946304602F02A
:10ACE00047FA012802D06FF002081CE00098D0B1AA
:10ACF0004FF080500D490860BFF34F8FBFF36F8F47
:10AD000011E006B115B96FF003080CE022462946A0
:10AD1000304602F079F9012805D014B16FF001082E
:10AD200001E06FF002084046BDE8F88304ED00E062
:10AD30002DE9F84305460E4614464FF00009FEF78C
:10AD4000F1FE00283ED1002D3CD0002E3AD0471E07
:10AD5000BCB1A06858B1E068502808D3206930B170
:10AD600005FB06F06169814201D301270AE0A06872
:10AD700040B9E06830B9206920B9606910B900278E
:10AD800000E00027012F09D100200090314628461D
:10AD9000A368226901F005FF814606E02FB9002271
:10ADA0003146284601F0D0FE8146B9F1000F09D0A6
:10ADB00014B1D4F8008001E04FF000084146484645
:10ADC00001F0F8FA4846BDE8F88300002DE9F843A1
:10ADD00007460D4691461C463E464FF00008FEF7DA
:10ADE000A1FEE8B10EB105B114B16FF003082AE07D
:10ADF0000020009000236A462946304602F062F89F
:10AE0000012802D06FF002081DE00098D8B14FF081
:10AE100080500E490860BFF34F8FBFF36F8F12E071
:10AE200006B115B96FF003080DE00023224629464C
:10AE3000304601F073FF012805D014B16FF001080E
:10AE400001E06FF002084046BDE8F88304ED00E041
:10AE500070B505462E46FEF765FE10B16FF005048D
:10AE600008E016B96FF0030404E000240021304626
:10AE700001F008FF204670BD2DE9F04104460D4663
:10AE800024F0010604F001080027FEF74BFE08B18C
:10AE9000BF1F1FE016B96FF003071BE0B8F1000FEA
:10AEA0000CD02946304602F0A5FA012812D015B17F
:10AEB0006FF001070EE06FF002070BE02946304605
:10AEC00002F0BCF9012805D015B16FF0010701E0CF
:10AED0006FF002073846BDE8F0812DE9F0470446DF
:10AEE0000026FEF71FFE00284DD10CB1676800E078
:10AEF000002707F0010008B1012500E0002507F058
:10AF0000080008283FD04FF0FF3874B1A06828B17E
:10AF1000E068502802D34FF0010808E0A06830B97B
:10AF2000E06820B94FF0000801E04FF00008B8F1E8
:10AF3000010F0CD12DB10420A16801F0F0FD0646EF
:10AF400012E00120A16801F0EAFD06460CE0B8F12C
:10AF5000000F09D125B1042001F0D0FD064603E021
:10AF6000012001F0CBFD06464EB114B1D4F800909B
:10AF700001E04FF000094946304601F01BFA16B1D6
:10AF80000DB146F001063046BDE8F0872DE9F041ED
:10AF9000044624F0010504F001070026FEF7C2FD77
:10AFA00008B1B61F16E015B96FF0030612E03FB105
:10AFB000284602F005F801280CD06FF0020609E0DF
:10AFC00000231A461946284601F0A8FE012801D0A0
:10AFD0006FF002063046BDE8F0810000FEB5044681
:10AFE0000D46264616B105F0004018B16FF003007B
:10AFF00002902EE04FF0FF300290FEF793FDE0B19B
:10B000000020019001A8002301222946009030462B
:10B0100002F082FB002002AB02460146009030465F
:10B0200002F07AFB0198A0B14FF080500A49086005
:10B03000BFF34F8FBFF36F8F0BE000230122294630
:10B04000304602F0D5FA02AB00221146304602F03B
:10B05000CFFA0298FEBD000004ED00E02DE9FC5F90
:10B06000054689461646FEF75DFD10B16FF00504F2
:10B070004AE005F0004010B16FF0030444E009F02D
:10B080000200022802D14FF0000A00E0AA46002484
:10B09000374602F009FC009000BF3B4601AA51462A
:10B0A000002002F0B3FC8046B8F1010F22D12C4001
:10B0B0000198044309F0010040B105EA0400A842E8
:10B0C00000D120E056B96FF002041CE005EA04004C
:10B0D00000B118E016B96FF0020414E002F0E4FBCE
:10B0E0000099A0EB010BBB4501D9002708E0A7EBB5
:10B0F0000B0705E016B96FF0020401E06FF00104E0
:10B10000B8F1000FC9D100BF2046BDE8FC9F10B5C3
:10B1100002F0B4FB0446204610BD2DE9FF478046EF
:10B120008946144600200390FEF7FCFC00284ED10F
:10B13000B8F1000F4BD0802618258246471E44B335
:10B14000206808B1D4F800A0A06900B1A5692DB1AC
:10B15000382D03D8207900F0010018B1002004B088
:10B16000BDE8F087606908B160698608A06840B1F1
:10B17000E068642805D3206918B1606908B1012727
:10B1800008E0A06830B9E06820B9206910B900274C
:10B1900000E00027012F0CD12169A0684B46324600
:10B1A000CDE9005102905146404602F0C3F90390A8
:10B1B0000DE067B903A8B2B24B465146CDE9005045
:10B1C000404602F085F9012801D000200390039841
:10B1D000C5E72DE9F04106463746FEF7A3FC10B15E
:10B1E0006FF0050410E017B96FF003040CE0384667
:10B1F000FFF700FC0546042D04D00024384601F07A
:10B20000ADF901E06FF002042046BDE8F0810000D6
:10B210002DE9F04105460E461648076816480068B5
:10B22000001D00F078FF681C38B936B1124801687B
:10B23000091D124800F0C7FF1AE07C190E4800688B
:10B240004460BC4207D20C480168091D0C480068E4
:10B2500000F09FFF0CE008480168091D09480068DC
:10B2600000F097FF08480068844201D20648046055
:10B27000BDE8F0812C00002018000020640A0020A6
:10B28000200000201C0000204800002010B50446CB
:10B2900000F0A6FF24480068401C234908602348AA
:10B2A000006840B9214804600846006801280DD1B3
:10B2B00000F018FA0AE01E48006838B91B48006818
:10B2C000C06AE16A884201D81848046019480068D9
:10B2D000401C1849086008460068A0641649E06AE6
:10B2E0000968884202D91449E06A0860E16A01EB02
:10B2F0008101124A02EB8100211D00F064FF00F081
:10B3000099FF0B48006868B108480068C06AE16AA4
:10B31000884207D24FF0805009490860BFF34F8F31
:10B32000BFF36F8F10BD0000280000201800002020
:10B33000340000204400002030000020B40500202C
:10B3400004ED00E008B500F04BFF12480068E8B9D2
:10B35000114800F00EFF114800F00BFF0E48104995
:10B3600008600E480F49086000200F4B0F4A10215B
:10B3700000900A2001F015FC0649086008460068A4
:10B3800020B10BA10348006801F014F800F052FF4F
:10B3900008BD000064000020780A00208C0A00200C
:10B3A0005C00002060000020A00A0020F00A0020BD
:10B3B000546D72510000000010B516E000F010FF4F
:10B3C0000C48C068C468201D00F0A5FE0A4800684B
:10B3D000401E0949086009480068401E0749086086
:10B3E00000F028FF204600F05FF8044800680028BD
:10B3F000E4D110BD500A00202800002024000020C5
:10B4000070B504460D46206C70B1216CE0680144B3
:10B41000E160D4E90210884201D32168E160284646
:10B42000226CE168F5F717F870BD2DE9F04104468C
:10B430000F4615464FF00008A66B206C48B92068EF
:10B4400000282CD1A06802F031FB80460020A060CB
:10B4500025E07DB93946226C6068F4F7FCFF216C69
:10B46000606808446060D4E90101884217D320680D
:10B47000606014E03946226CE068F4F7ECFF216C60
:10B48000E068411AE1602168E068884203D2216CDB
:10B49000A068411AE160022D01D106B1761E701C30
:10B4A000A0634046BDE8F08110B5044694F8610001
:10B4B00030B9206B00F0DCFE204600F0D9FE1AE027
:10B4C00094F86100012803D1204600F0D1FE12E07B
:10B4D00094F86100022801D1012000E0002050B959
:10B4E00000BF502080F31188BFF34F8FBFF36F8FE1
:10B4F00000BF00BFFEE710BD01464A6A22B10A6BD9
:10B500001268C2F1380000E0002070470146084A86
:10B51000126812680AB9012200E000220A600A6873
:10B5200022B9034A1268D268106800E00020704710
:10B530005C00002030B54FF4C043174800F007040A
:10B540002CB1C01D20F00700134C041B1B1B02462E
:10B55000124C22600024114D6C60D018083820F085
:10B5600007000F4C206000240D4D2D686C600C4DC1
:10B570002D682C601146441A4C60094C24680C60FC
:10B58000084D4C682C60084D4C682C604FF000440E
:10B59000064D2C6030BD00005812002074000020C1
:10B5A0007C0000208400002080000020900000200B
:10B5B00000BFFFF701FF064800680128F9D94FF0E6
:10B5C000805004490860BFF34F8FBFF36F8FF0E7DF
:10B5D000B405002004ED00E010B5044654B100208D
:10B5E000A06020600021E16000231A461946204631
:10B5F00001F094FB10BD2DE9F04106460D461746BB
:10B600009846069C0DB9246000E02760E663256437
:10B610000121204601F036FB84F84C80BDE8F08122
:10B620002DE9F05F82460E4691469B460A9F0C9C90
:10B630004FEA8901A522206BF4F784FFA9F10100EC
:10B64000216B01EB800828F0070808F0070008B913
:10B65000012000E0002050B900BF502080F3118885
:10B66000BFF34F8FBFF36F8F00BF00BFFEE7C4F87B
:10B67000448086B1002507E0715D04F13400415536
:10B68000705D00B902E06D1C102DF5D300BF0021E4
:10B690004320015502E0002084F83400382F00D305
:10B6A0003727E762276500206065201D00F06EFDEA
:10B6B00004F1180000F06AFD2461C7F13800A061B0
:10B6C00064620020A065E06584F860005A46514637
:10B6D000404600F081FB20600B9808B10B98046095
:10B6E000BDE8F09F10B5002407E004EB84010F4A89
:10B6F00002EB810000F03DFD641C382CF5D30C48B2
:10B7000000F037FD0B4800F034FD0B4800F031FD30
:10B710000A4800F02EFD0A4800F02BFD04480949B4
:10B72000086004480849086010BD0000B405002006
:10B73000140A0020280A00203C0A0020500A002099
:10B74000640A00201C0000202000002010B50146E3
:10B75000164800E0006803688B42FBD3024643684A
:10B7600013448B4204D143684C6823444360014630
:10B770000A464B6813440468A34211D10C4C036879
:10B780002468A34208D04B680468646823444B6073
:10B7900003681B680B6005E0054B1B680B6001E04C
:10B7A00003680B60884200D0016010BD7400002067
:10B7B0007C0000202DE9F04104460D4616461F4648
:10B7C0004FF0000865602461B5420CD8F01BA169F8
:10B7D000884202D34FF0010811E0211D094800689A
:10B7E00000F0D7FC0BE0BE4204D2BD4202D34FF0C2
:10B7F000010804E0211D0448006800F0CAFC40462E
:10B80000BDE8F081600000205C00002070B50546B6
:10B8100000F0E6FCA86B08B9012400E0002400F069
:10B8200009FD204670BD70B5054600F0D9FCA86B37
:10B83000E96B884201D1012400E0002400F0FAFC09
:10B84000204670BDF8B505460F461A480068C06826
:10B85000C468201D00F05FFC94F8280000F004008C
:10B86000E8B1A06941192B463A462046FFF7A2FFEE
:10B87000D8B1002003462A4601460090204602F037
:10B88000C3FA064656B900BF502080F31188BFF3B3
:10B890004F8FBFF36F8F00BF00BFFEE705E094F846
:10B8A000280020F0010084F828002046216A8847FB
:10B8B000F8BD00005C000020F0B587B0A0E0039860
:10B8C000002811DA04AE56B900BF502080F3118869
:10B8D000BFF34F8FBFF36F8F00BF00BFFEE7D6E906
:10B8E0000020B168904700BF03980028E6DB059C64
:10B8F000606908B9012000E0002010B9201D00F0A7
:10B900000AFC02A800F0DEF8054603980A2875D262
:10B91000DFE800F009050739416306083A4200BF35
:10B9200000BF00BF00BF94F8280040F0010084F879
:10B9300028000498A269811803462A462046FFF78A
:10B9400039FFF8B12046216A884794F8280000F0B2
:10B950000400B8B1002000900498A16942180023A7
:10B960001946204602F050FA074657B900BF50204A
:10B9700080F31188BFF34F8FBFF36F8F00BF00BFFD
:10B98000FEE700BF3BE000BF94F8280020F0010074
:10B9900084F8280033E000BF94F8280040F001004C
:10B9A00084F828000498A061A06908B1012000E093
:10B9B000002050B900BF502080F31188BFF34F8F93
:10B9C000BFF36F8F00BF00BFFEE7A06941192B4690
:10B9D0002A462046FFF7EEFE11E094F8280000F01A
:10B9E000020018B9204600F043FC05E094F8280056
:10B9F00020F0010084F8280001E0FFE700BF00BF4D
:10BA0000002203A90448006801F0FEFA00287FF430
:10BA100056AF07B0F0BD000064000020F8B5054641
:10BA20000C4600F013FF684600F04CF806460098FC
:10BA300020BB44B9B54206D802F028F93146284661
:10BA4000FFF700FF1CE03CB10E480068006808B931
:10BA5000012000E000200446A91B22460A48006895
:10BA600000F0BEFC02F012F950B94FF080500749C7
:10BA70000860BFF34F8FBFF36F8F01E002F006F94C
:10BA8000F8BD0000600000206400002004ED00E02C
:10BA90000A490968096809B9012100E0002121B1BA
:10BAA0004FF0FF31064A116006E004490968C96891
:10BAB000C868034A41681160704700001C000020FC
:10BAC0004800002070B5044601F0EEFE0546074828
:10BAD0000068854204D200F00BF80120206001E0EC
:10BAE0000020206001480560284670BD6C000020E1
:10BAF0002DE9F84334E025480068C068056823480C
:10BB00000068C068C468201D00F005FB2046216A5B
:10BB1000884794F8280000F0040008B3A06946198B
:10BB2000AE4207D966602461211D1848006800F004
:10BB300030FB15E0002003462A46014600902046CF
:10BB400002F062F9074657B900BF502080F3118810
:10BB5000BFF34F8FBFF36F8F00BF00BFFEE700BF83
:10BB60000A480068006808B9012000E000200028A9
:10BB7000C1D00648D0F80080054800680349086035
:10BB80000348C0F80080BDE8F88300005C00002096
:10BB9000600000200E480068401C08B9012000E049
:10BBA000002050B900BF502080F31188BFF34F8FA1
:10BBB000BFF36F8F00BF00BFFEE700BF502080F3D0
:10BBC0001188BFF34F8FBFF36F8F00BF00BFFEE739
:10BBD0009400002008B500BF6846FFF797FC0446B4
:10BBE00020460099FFF71AFFFFF766FEF4E770B5ED
:10BBF000044600F0F5FA94F9455010E0606A08B97F
:10BC0000012000E0002038B904F1240001F0F2FF27
:10BC100018B100F013FD00E003E0681E45B2002DEE
:10BC2000ECDC00BFFF2084F8450000F003FB00F0CF
:10BC3000D7FA94F9445010E0206908B9012000E0D7
:10BC4000002048B904F1100001F0D4FF08B100F061
:10BC5000F5FC681E45B200E001E0002DECDC00BF01
:10BC6000FF2084F8440000F0E5FA70BD2DE9F041B2
:10BC700004464FF0000800F0E9FD4948006808B9A3
:10BC8000FFF758FC474800682040002870D1D4B125
:10BC9000083404F00700B0B104F00700C0F1080058
:10BCA000044404F0070008B9012000E0002050B966
:10BCB00000BF502080F31188BFF34F8FBFF36F8F09
:10BCC00000BF00BFFEE7002C52D037480068844216
:10BCD0004ED8364E3046056801E02E462D6868681D
:10BCE000A04202D228680028F7D12D48006885427A
:10BCF0003ED0306800F10808286830606868001B92
:10BD0000102819D92F1907F0070008B9012000E001
:10BD1000002050B900BF502080F31188BFF34F8F2F
:10BD2000BFF36F8F00BF00BFFEE76868001B78603D
:10BD30006C603846FFF70AFD1B4968680968081AF5
:10BD4000194908600846006819490968884203D201
:10BD50001548006816490860124968680968084370
:10BD600068600020286013480068401C1149086082
:10BD700001F08CFF08F0070008B9012000E0002066
:10BD800050B900BF502080F31188BFF34F8FBFF32D
:10BD90006F8F00BF00BFFEE74046BDE8F0810000A6
:10BDA0007C00002090000020800000207400002013
:10BDB00084000020880000200648006830B1054952
:10BDC000096801F15400496D491C0160014800688F
:10BDD0007047000018000020001F4FF080730360C0
:10BDE000001F21F001030360001F054B036014389E
:10BDF0000260001F6FF002030360203870470000EC
:10BE000095BB000870B52DED048B04460D46164613
:10BE1000B5F90C00B0F5E16F26D101202070B5F91D
:10BE20000410A1F5437002F014FB41EC190B9FEDD7
:10BE3000130B53EC102B02F073FB41EC180B02F0C8
:10BE400031F8A060B5F9000002F003FB41EC190BDA
:10BE50009FED0C0B53EC102B02F062FB41EC180B26
:10BE600002F020F8606005E0B5F90C00C82801D1A7
:10BE700000202070BDEC048B70BD0000EE42B24A81
:10BE80000ADB483FFA6B43132A55583F10B5192176
:10BE90000148FCF70BFE10BDD773002030B52DED27
:10BEA000048B81B005460C4605B11CB901B0BDEC50
:10BEB000048B30BD6878A97840EA0120C0F30A00FD
:10BEC0002080A878C010E97840EA4110C0F30A0049
:10BED0006080E8788011297940EA8100697940EA38
:10BEE0008120C0F30A00A08068794010A97940EA57
:10BEF000C110C0F30A00E080A8790011E97940EA96
:10BF00000110C0F30A002081E879C011297A40EAC3
:10BF10004100697A40EA4120C0F30A0104F10800B7
:10BF20006181687A8010A97A40EA8110C0F30A0121
:10BF300004F10800A181A87A4011E97A40EAC10021
:10BF400004F10801E081287B697B40EA0120C0F30D
:10BF50000A0104F108002182687BC010A97B40EA35
:10BF60004110C0F30A0104F108006182A87B80112E
:10BF7000E97B40EA8100297C40EA8120C0F30A0184
:10BF800004F10800A182287C4010697C40EAC110BD
:10BF9000C0F30A0104F10800E1822088A0F5806066
:10BFA00000B220806088A0F5806000B26080A08828
:10BFB000A0F5806000B2A080E088A0F5806000B2AB
:10BFC000E0802088183000B2208060884042183815
:10BFD00000B26080A088C0F53F7000B2A080E08809
:10BFE000183000B2E0804FF42F700090B4F90200D6
:10BFF0002A4B40F2B622D91DFEF778FD00B26080D0
:10C000004FF42F700090B4F90000244B40F2B52299
:10C01000991DFEF76BFD00B22080B4F9060002F016
:10C0200018FA41EC190B9FED1E0B53EC102B02F08C
:10C0300077FA41EC180B02F0AFF900B2E080B4F9E6
:10C04000000010F11E0F05DDB4F900001E2801DA12
:10C0500000202080B4F9020010F11E0F05DDB4F9B4
:10C0600002001E2801DA00206080B4F9040010F1FB
:10C070001E0F05DDB4F904001E2801DA0020A0809F
:10C08000B4F9060010F11E0F05DDB4F906001E28F4
:10C0900001DA0020E08000BF08E7000044FDFFFF58
:10C0A000000000000000E03F10B500EE100A2DED8A
:10C0B000028BB1EEC08A18EE100A20F00040C0F1E9
:10C0C000FF40C00F0AD010EE100A20F00040C0F16F
:10C0D000FF40C00F04BF0120F4F78DFA18EE100ADC
:10C0E000BDEC028B10BD00B5034605E04FF47A703D
:10C0F00000F005F8581E83B2002BF7DC00BD07E006
:10C10000322101E04A1ED1B20029FBDC411E88B277
:10C110000028F5DC704701460A69D1E901309860D2
:10C12000D1E9010358605068884201D188685060A5
:10C13000002008611068401E106010687047000001
:10C14000034B0360034B0B608023136070470000B8
:10C15000900B0020F40B0020034B0360034B0B609B
:10C160004FF4807313607047F40D0020580E0020C8
:10C17000704700F1080141604FF0FF31816000F12C
:10C180000801C16001610021016070470021016167
:10C19000704710B502460B685C1C0CB9106907E0CB
:10C1A00002F1080000E04068446824689C42FAD923
:10C1B00044684C604C68A160886041600A61146802
:10C1C000641C146010BD42684A6093688B60936879
:10C1D00059609160086103685B1C03607047000050
:10C1E00000BF502080F31188BFF34F8FBFF36F8FD4
:10C1F00000BF0E480068401C0C49086008460068F3
:10C20000012812D10A480068C0B208B9012000E034
:10C21000002050B900BF502080F31188BFF34F8F2A
:10C22000BFF36F8F00BF00BFFEE770479400002090
:10C2300004ED00E00D48006850B900BF502080F3C5
:10C240001188BFF34F8FBFF36F8F00BF00BFFEE7B2
:10C2500006480068401E054908600846006820B985
:10C26000002080F3118800BF00BF704794000020B9
:10C2700070B506463546002E44D0083D2C4622496E
:10C2800060680968084008B1012000E0002050B94A
:10C2900000BF502080F31188BFF34F8FBFF36F8F23
:10C2A00000BF00BFFEE7206808B9012000E00020C1
:10C2B00050B900BF502080F31188BFF34F8FBFF3F8
:10C2C0006F8F00BF00BFFEE70F4960680968084034
:10C2D000C0B12068B0B90C496068096888436060E3
:10C2E00000F0B4FA09496068096808440749086021
:10C2F0002046FFF72BFA06480068401C04490860F6
:10C3000001F0C4FC70BD00009000002080000020FF
:10C310008C00002000204FF0E02108618861064871
:10C3200000684FF47A71B0FBF1F0401E4FF0E0214D
:10C3300048610720086170471400002070B5F3F7CA
:10C34000EFFF0446102C16D304F1E02090F8F053D0
:10C3500015480078854201DB012000E0002050B93B
:10C3600000BF502080F31188BFF34F8FBFF36F8F52
:10C3700000BF00BFFEE70D48006800F4E0600C4914
:10C380000968884201D8012000E0002050B900BFB0
:10C39000502080F31188BFF34F8FBFF36F8F00BF22
:10C3A00000BFFEE770BD0000980000200CED00E02B
:10C3B0009C000020024600200BE0084B53F8303070
:10C3C00033B9064B43F8301003EBC0035A6002E068
:10C3D000401C0828F1D300BF7047000074050020FE
:10C3E0002DE9F04105460E4617462C46FFF7F8FEAC
:10C3F00094F94400401C10B9002084F8440094F9DA
:10C400004500401C10B9002084F84500FFF712FFDA
:10C41000A06B28B93A46314604F1240000F030F907
:10C420002046FFF7E4FBBDE8F081000070B504464C
:10C430000025D4B11248006808B9012000E00020AE
:10C4400050B900BF502080F31188BFF34F8FBFF366
:10C450006F8F00BF00BFFEE700F0F8F90021204613
:10C46000FEF7D6FE01F012FC05463DB94FF08050B4
:10C4700004490860BFF34F8FBFF36F8F70BD00009A
:10C480005000002004ED00E02DE9F04704460F467F
:10C490004FF0000954B900BF502080F31188BFF35A
:10C4A0004F8FBFF36F8F00BF00BFFEE70FB10120BA
:10C4B00000E0002050B900BF502080F31188BFF386
:10C4C0004F8FBFF36F8F00BF00BFFEE720480068AB
:10C4D00008B9012000E0002050B900BF502080F3CF
:10C4E0001188BFF34F8FBFF36F8F00BF00BFFEE710
:10C4F00000F0ACF9174806682068C5192068B042FA
:10C5000007D92068A8420BD9B54209D94FF00109D3
:10C5100006E02068A84201D8B54201D94FF00109D0
:10C520002560B9F1000F03D0A81B0021FEF770FEB3
:10C5300001F0ACFB8046B8F1000F07D14FF08050FE
:10C5400005490860BFF34F8FBFF36F8FBDE8F087D9
:10C55000500000202C00002004ED00E070B50546DE
:10C56000FFF73EFE15B92748006800E0284604465C
:10C57000201DFFF7D0FDA06A18B104F11800FFF7E5
:10C58000CAFD21480068401C1F4908601D4800681A
:10C59000844209D1211D1D48FFF715FE1C48006883
:10C5A000401C1B49086009E01A480068401E1949F0
:10C5B00008602046FEF778FFFFF76AFAFFF73AFEB9
:10C5C00015480068E8B10F480068844219D1134843
:10C5D000006808B9012000E0002050B900BF5020D9
:10C5E00080F31188BFF34F8FBFF36F8F00BF00BF81
:10C5F000FEE74FF080500A490860BFF34F8FBFF34A
:10C600006F8F70BD1800002044000020500A0020E9
:10C6100024000020280000203400002050000020CA
:10C6200004ED00E0034909680160034909684160BD
:10C6300070470000400000202C000020012001492C
:10C64000086070473C00002070B504460D4654B9A0
:10C6500000BF502080F31188BFF34F8FBFF36F8F5F
:10C6600000BF00BFFEE70548016818312046FFF70C
:10C6700090FD01212846FEF7CBFD70BD180000207B
:10C6800070B505460E46144655B900BF502080F3DC
:10C690001188BFF34F8FBFF36F8F00BF00BFFEE75E
:10C6A0000648016818312846FFF78DFD0CB14FF0A0
:10C6B000FF3621463046FEF7ABFD70BD1800002066
:10C6C0002DE9F04706460F4634464FF00109002E8B
:10C6D00055D0606D50B900BF502080F31188BFF372
:10C6E0004F8FBFF36F8F00BF00BFFEE7206DB842D2
:10C6F00001D23D4600E0256DE06AA8423FD0606D62
:10C7000001283CD11F480068844201D0012000E08C
:10C71000002050B900BF502080F31188BFF34F8F25
:10C72000BFF36F8F00BF00BFFEE7D4F82C80E56237
:10C73000A06900F0004010B9C5F13800A06108EB15
:10C740008801114A02EB81016069884201D1012010
:10C7500000E0002098B1201DFFF7DDFC0B49E06AE6
:10C760000968884202D90949E06A0860E16A01EB78
:10C770008101054A02EB8100211DFFF724FDBDE880
:10C78000F087000018000020B405002030000020D1
:10C7900010B586B000200590049003AA04A905A84E
:10C7A000FFF7CEFC0022DDE904101346CDE900219D
:10C7B00002901FA12048039A00F0BCFE1F490860A8
:10C7C0000846006808B1012400E00024012C02D1D1
:10C7D00001F0DEFA0446012C17D100BF502080F38F
:10C7E0001188BFF34F8FBFF36F8F00BF4FF0FF3043
:10C7F00013490860012013490860002012490860AD
:10C80000FEF7DEF800F0ACF810E0601C08B1012083
:10C8100000E0002050B900BF502080F31188BFF322
:10C820004F8FBFF36F8F00BF00BFFEE706B010BD94
:10C8300049444C4500000000B1B500084C00002000
:10C8400048000020340000202C000020024800682E
:10C85000401C0149086070475000002070B53948FD
:10C86000006818B101203849086069E000203649A5
:10C870000860FEF715F93549086008460068344934
:10C88000096888420BD93349096801F15800896D5C
:10C890002E4A12682E4B1B68D21A114401602B4895
:10C8A00000682B4908602B480068046B4FF0A535E1
:10C8B0002068B0F1A53F0BD16068B0F1A53F07D16A
:10C8C000A068B0F1A53F03D1E068B0F1A53F05D065
:10C8D0002048016834310068FFF74AFC1E480168AF
:10C8E0000CE051B900BF502080F31188BFF34F8F87
:10C8F000BFF36F8F00BF00BFFEE7491E01EB810051
:10C90000164A52F8200008B9012000E00020002853
:10C91000E7D101EB8102114B03EB820042685268C0
:10C92000426000F108024368934202D142685268B3
:10C9300042604268D268074B1A600748016000BF36
:10C9400070BD0000500000203C0000205800002076
:10C95000540000201800002030000020B405002002
:10C960001CB5524800685249884201D0012000E0BD
:10C97000002050B900BF502080F31188BFF34F8FC3
:10C98000BFF36F8F00BF00BFFEE74848006848490B
:10C99000491E884201D0012000E0002050B900BFAC
:10C9A000502080F31188BFF34F8FBFF36F8F00BF0C
:10C9B00000BFFEE73F49084600780190FF200A4685
:10C9C00010700846007800909DF8000000F0F0001C
:10C9D0009DF80020904201D1012000E0002050B9D4
:10C9E00000BF502080F31188BFF34F8FBFF36F8FCC
:10C9F00000BF00BFFEE79DF8000000F050002E4A87
:10CA0000107007202D4A106009E02C480068401E75
:10CA10002A4A10609DF800004006000E00909DF824
:10CA2000000000F080008028EFD024480068C0F1AA
:10CA30000700042801D1012000E0002050B900BF08
:10CA4000502080F31188BFF34F8FBFF36F8F00BF6B
:10CA500000BFFEE7194800680002184A106010463F
:10CA6000008800F4E0601060124A019810700F48CE
:10CA70002030006840F470000C49203108600846FE
:10CA8000006840F070400860FFF744FC00200C494B
:10CA90000860F3F70DFC0B48006840F0404009497E
:10CAA0000860F3F7F1FB00201CBD000000ED00E082
:10CAB00071C20F4100E400E0980000209C000020BB
:10CAC0009400002034EF00E010B500BF502080F348
:10CAD0001188BFF34F8FBFF36F8F00BF00F0F4FEDC
:10CAE00018B14FF080500449086000BF002080F367
:10CAF000118800BF10BD000004ED00E02DE9F041F9
:10CB000004460126002722460021012000F01CF8DF
:10CB100005462846FEF760FD2846BDE8F0812DE970
:10CB2000F84304460D4601274FF000082B4600222B
:10CB300011460120009400F034F806463046FEF716
:10CB40004BFD3046BDE8F8832DE9F84305460E4617
:10CB500017460DB1012000E0002050B900BF502061
:10CB600080F31188BFF34F8FBFF36F8F00BF00BFFB
:10CB7000FEE705FB06F808F15000FFF777F80446DA
:10CB800064B1A14609F15009002084F846003B46F3
:10CB90004A46314628460094FEF72DFD2046BDE862
:10CBA000F8832DE9F84380460E4617461D46DDF80A
:10CBB0002090B8F1000F01D0012000E0002050B912
:10CBC00000BF502080F31188BFF34F8FBFF36F8FEA
:10CBD00000BF00BFFEE70DB1012000E0002050B90A
:10CBE00000BF502080F31188BFF34F8FBFF36F8FCA
:10CBF00000BF00BFFEE707B10EB1012000E000203A
:10CC000050B900BF502080F31188BFF34F8FBFF39E
:10CC10006F8F00BF00BFFEE707B90EB9012000E02B
:10CC2000002050B900BF502080F31188BFF34F8F10
:10CC3000BFF36F8F00BF00BFFEE750200090009849
:10CC4000502801D1012000E0002050B900BF502041
:10CC500080F31188BFF34F8FBFF36F8F00BF00BF0A
:10CC6000FEE700BF2C464CB1012084F846004B463D
:10CC70003A46314640460094FEF7BDFC2046BDE8EA
:10CC8000F883000070B505460E462C4654B900BF27
:10CC9000502080F31188BFF34F8FBFF36F8F00BF19
:10CCA00000BFFEE7FFF79CFAD4E90F12206801FBF2
:10CCB0000200A0600020A06320686060E06B401E5E
:10CCC000226C216800FB0211E160FF2084F844001F
:10CCD00084F845009EB9206908B9012000E00020D1
:10CCE000A8B904F1100000F085FF80B14FF080502A
:10CCF00009490860BFF34F8FBFF36F8F07E004F15E
:10CD00001000FFF736FA04F12400FFF732FAFFF7BC
:10CD100091FA012070BD000004ED00E02DE9FF4311
:10CD200083B0064688461D464FF00009344654B984
:10CD300000BF502080F31188BFF34F8FBFF36F8F78
:10CD400000BF00BFFEE7B8F1000F01D1206C08B9A9
:10CD5000012000E0002050B900BF502080F311886E
:10CD6000BFF34F8FBFF36F8F00BF00BFFEE7022DF1
:10CD700002D1E06B012801D1012000E0002050B970
:10CD800000BF502080F31188BFF34F8FBFF36F8F28
:10CD900000BF00BFFEE700F077FD08B9059808B9AD
:10CDA000012000E0002050B900BF502080F311881E
:10CDB000BFF34F8FBFF36F8F00BF00BFFEE700BF11
:10CDC000FFF70EFAA06BE16B884201D3022D28D148
:10CDD0002A4641462046FEF728FB0746606A08B906
:10CDE000012000E0002068B904F1240000F002FFF7
:10CDF00088B14FF0805032490860BFF34F8FBFF3C6
:10CE00006F8F08E03FB14FF080502D490860BFF3AD
:10CE10004F8FBFF36F8FFFF70DFA012007B0BDE80A
:10CE2000F083059818B9FFF705FA0020F6E7B9F185
:10CE3000000F04D101A8FFF7F5FB4FF00109FFF740
:10CE4000F9F9FFF703FDFFF7CBF994F94400401C13
:10CE500010B9002084F8440094F94500401C10B932
:10CE6000002084F84500FFF7E5F905A901A800F0C6
:10CE7000E9FAF0B92046FEF7D6FCA0B104F11000A3
:10CE80000599FFF7E1FB2046FEF7B1FE00F0FEFE3C
:10CE9000002895D14FF0805009490860BFF34F8FAB
:10CEA000BFF36F8F8CE72046FEF7A1FE00F0EEFE89
:10CEB00086E72046FEF79BFE00F0E8FE0020ADE787
:10CEC00004ED00E02DE9F84F07468A4690461E46DD
:10CED0003C4654B900BF502080F31188BFF34F8FF8
:10CEE000BFF36F8F00BF00BFFEE7BAF1000F01D1A3
:10CEF000206C08B9012000E0002050B900BF50208C
:10CF000080F31188BFF34F8FBFF36F8F00BF00BF57
:10CF1000FEE7022E02D1E06B012801D1012000E0E2
:10CF2000002050B900BF502080F31188BFF34F8F0D
:10CF3000BFF36F8F00BF00BFFEE7FFF7FFF900BF31
:10CF40005021EFF3118081F31188BFF34F8FBFF3AE
:10CF50006F8F00BF0546A06BE16B884201D3022EA4
:10CF600025D194F945B0A06B009032465146204639
:10CF7000FEF75BFA0BF1010088B9606A08B901207D
:10CF800000E0002050B904F1240000F033FE28B185
:10CF9000B8F1000F02D00120C8F8000004E00BF146
:10CFA000010040B284F845004FF0010901E04FF064
:10CFB000000900BF85F3118800BF4846BDE8F88F1F
:10CFC00070B505462C4654B900BF502080F3118837
:10CFD000BFF34F8FBFF36F8F00BF00BFFEE700F0BE
:10CFE0004DFCA16888420CD1E068401EE060E0681A
:10CFF00028B900231A4619462046FFF78FFE01265E
:10D0000000E00026304670BD2DE9F74183B00546AB
:10D010000E464FF000082C4654B900BF502080F354
:10D020001188BFF34F8FBFF36F8F00BF00BFFEE7C4
:10D030000EB9206C08B9012000E0002050B900BFF3
:10D04000502080F31188BFF34F8FBFF36F8F00BF65
:10D0500000BFFEE700F018FC08B9059808B90120E8
:10D0600000E0002050B900BF502080F31188BFF3CA
:10D070004F8FBFF36F8F00BF00BFFEE700BFFFF70A
:10D08000AFF8A76BF7B131462046FEF7B9F9781E25
:10D09000A063206908B9012000E0002060B904F114
:10D0A000100000F0A7FD38B14FF080502F49086004
:10D0B000BFF34F8FBFF36F8FFFF7BCF8012006B0AF
:10D0C000BDE8F081059818B9FFF7B4F80020F6E73D
:10D0D000B8F1000F04D101A8FFF7A4FA4FF001083E
:10D0E000FFF7A8F8FFF7B2FBFFF77AF894F94400CE
:10D0F000401C10B9002084F8440094F94500401CFD
:10D1000010B9002084F84500FFF794F805A901A89C
:10D1100000F098F9F0B92046FEF778FBA0B104F1D1
:10D1200024000599FFF790FA2046FEF760FD00F015
:10D13000ADFD0028A3D14FF080500C490860BFF32B
:10D140004F8FBFF36F8F9AE72046FEF750FD00F038
:10D150009DFD94E72046FEF74AFD00F097FD20462E
:10D16000FEF754FB00288AD00020A8E704ED00E079
:10D170002DE9F05F064689461746344654B900BF8C
:10D18000502080F31188BFF34F8FBFF36F8F00BF24
:10D1900000BFFEE7B9F1000F01D1206C08B90120F2
:10D1A00000E0002050B900BF502080F31188BFF389
:10D1B0004F8FBFF36F8F00BF00BFFEE7FFF7BEF8D2
:10D1C00000BF5021EFF3118081F31188BFF34F8F1F
:10D1D000BFF36F8F00BF0546D4F838A0BAF1000F37
:10D1E00022D094F944B049462046FEF709F9AAF145
:10D1F0000100A0630BF1010070B9206908B901209A
:10D2000000E0002068B904F1100000F0F3FC40B128
:10D210003FB10120386004E00BF1010040B284F816
:10D2200044004FF0010801E04FF0000800BF85F313
:10D23000118800BF4046BDE8F09F00002DE9F34192
:10D2400082B005464FF000082C46002654B900BFB6
:10D25000502080F31188BFF34F8FBFF36F8F00BF53
:10D2600000BFFEE7206C08B9012000E0002050B9A3
:10D2700000BF502080F31188BFF34F8FBFF36F8F33
:10D2800000BF00BFFEE700F0FFFA08B9039808B935
:10D29000012000E0002050B900BF502080F3118829
:10D2A000BFF34F8FBFF36F8F00BF00BFFEE700BF1C
:10D2B000FEF796FFA76BFFB1781EA063206810B938
:10D2C000FEF77AFDA060206908B9012000E0002087
:10D2D00060B904F1100000F08DFC38B14FF08050BF
:10D2E00043490860BFF34F8FBFF36F8FFEF7A2FF74
:10D2F000012004B0BDE8F081039898B90EB901206F
:10D3000000E0002050B900BF502080F31188BFF327
:10D310004F8FBFF36F8F00BF00BFFEE7FEF78AFF9E
:10D320000020E6E7B8F1000F04D16846FFF77AF96C
:10D330004FF00108FEF77EFFFFF788FAFEF750FF77
:10D3400094F94400401C10B9002084F8440094F97A
:10D350004500401C10B9002084F84500FEF76AFF24
:10D3600003A9684600F06EF840BB2046FEF74EFA6F
:10D37000F0B1206838B9FEF733FFA06800F0E8FB91
:10D380000646FEF757FF04F124000399FFF75CF906
:10D390002046FEF72CFC00F079FC002888D14FF0E5
:10D3A000805013490860BFF34F8FBFF36F8F7FE743
:10D3B0002046FEF71CFC00F069FC79E72046FEF7EA
:10D3C00016FC00F063FC2046FEF720FA0028EED0A1
:10D3D0005EB1FEF705FF2046FEF78EF80746394698
:10D3E000A068FFF76DF9FEF725FF002081E7000038
:10D3F00004ED00E02DE9F04106460F46344654B9ED
:10D4000000BF502080F31188BFF34F8FBFF36F8FA1
:10D4100000BF00BFFEE700F031FAA168884204D1E6
:10D42000E068401CE060012508E039462046FFF72F
:10D4300005FF054615B1E068401CE0602846BDE8E0
:10D44000F081000070B505460C4655B900BF50206C
:10D4500080F31188BFF34F8FBFF36F8F00BF00BF02
:10D46000FEE754B900BF502080F31188BFF34F8FFF
:10D47000BFF36F8F00BF00BFFEE7FEF7B1FE12489B
:10D4800002686868131A2068401C08B9002617E073
:10D490000E4928680968884204D06868904201D81B
:10D4A00001260DE02068984207D92068C01A206044
:10D4B0002846FFF7B7F8002602E00020206001268A
:10D4C000FEF7B8FE304670BD2C0000204000002062
:10D4D0002DE9FF4F85B0804689461746DDE912AB3E
:10D4E000B800FEF7C3FB064656B16420FEF7BEFB4C
:10D4F00004460CB1266304E03046FEF7B9FE00E0B6
:10D5000000248CB1002084F86100CDE900ABCDE9A6
:10D5100002403A4649464046089BFEF781F82046BD
:10D52000FDF7B4FE012501E04FF0FF35284609B0B4
:10D53000BDE8F08F2DE9F04F85B00746884691464B
:10D540009A46DDE90EB6109C0EB1012000E00020E5
:10D5500050B900BF502080F31188BFF34F8FBFF345
:10D560006F8F00BF00BFFEE70CB1012000E000207C
:10D5700050B900BF502080F31188BFF34F8FBFF325
:10D580006F8F00BF00BFFEE76420039003986428FC
:10D5900001D1012000E0002050B900BF502080F3ED
:10D5A0001188BFF34F8FBFF36F8F00BF00BFFEE73F
:10D5B00000BFB4B1AEB125462C462E63022085F8DB
:10D5C0006100002004A953464A46CDE900B1CDE9E7
:10D5D000025041463846FEF723F82846FDF756FE2E
:10D5E00001E000200490049805B0BDE8F08F000031
:10D5F0002DE9F04706460D46174698464FF0010ABA
:10D6000056B900BF502080F31188BFF34F8FBFF38E
:10D610006F8F00BF00BFFEE73446FEF7E1FDB8F1B3
:10D62000000F02D0E06DC8F8000094F8609002206E
:10D6300084F86000052F17D2DFE807F01503070B09
:10D640000D00E06D2843E06521E0E06D401CE065E1
:10D650001DE0E5651BE0B9F1020F01D0E56501E0D1
:10D660004FF0000A13E012E0E06D401C08B9012001
:10D6700000E0002050B900BF502080F31188BFF3B4
:10D680004F8FBFF36F8F00BF00BFFEE700BF00BF2B
:10D69000B9F1010F32D1201DFEF73DFD1A49E06AB4
:10D6A0000968884202D91849E06A0860E16A01EB1A
:10D6B0008101164A02EB8100211DFEF784FDA06A5C
:10D6C00008B9012000E0002050B900BF502080F3CD
:10D6D0001188BFF34F8FBFF36F8F00BF00BFFEE70E
:10D6E0000B49E06A0968C96A884207D94FF080503F
:10D6F00008490860BFF34F8FBFF36F8FFEF79AFDA5
:10D700005046BDE8F087000030000020B40500203E
:10D710001800002004ED00E02DE9F84F07460E4602
:10D7200090469946DDF828B00120009057B900BF17
:10D73000502080F31188BFF34F8FBFF36F8F00BF6E
:10D7400000BFFEE7FEF7FAFD3C4600BF5021EFF3B5
:10D75000118081F31188BFF34F8FBFF36F8F00BF2C
:10D760000546B9F1000F02D0E06DC9F8000094F849
:10D7700060A0022084F86000B8F1050F17D2DFE83E
:10D7800008F01503070B0D00E06D3043E06521E064
:10D79000E06D401CE0651DE0E6651BE0BAF1020F9C
:10D7A00001D0E66501E00020009013E012E0E06D9A
:10D7B000401C08B9012000E0002050B900BF5020F3
:10D7C00080F31188BFF34F8FBFF36F8F00BF00BF8F
:10D7D000FEE700BF00BFBAF1010F3CD1A06A08B953
:10D7E000012000E0002050B900BF502080F31188D4
:10D7F000BFF34F8FBFF36F8F00BF00BFFEE7194825
:10D800000068A0B9201DFEF786FC1749E06A096888
:10D81000884202D91449E06A0860E16A01EB81019B
:10D82000124A02EB8100211DFEF7CDFC04E004F159
:10D8300018010F48FEF7C7FC0E49E06A0968C96A7B
:10D84000884208D9BBF1000F02D00120CBF80000BC
:10D8500001200949086000BF85F3118800BF0098C6
:10D86000BDE8F88F5000002030000020B4050020F3
:10D870003C0A0020180000203C00002001490868F4
:10D8800070470000180000200549096809B9012007
:10D8900005E00449096809B9022000E0002070474A
:10D8A0003400002050000020014908687047000043
:10D8B0002C00002070B5FEF741FD002501480468EA
:10D8C000204670BD2C0000202DE9F0414FF00008EB
:10D8D0004348006800287BD142480068451C414805
:10D8E000056015BB40480068006808B9012000E0E9
:10D8F000002050B900BF502080F31188BFF34F8F34
:10D90000BFF36F8F00BF00BFFEE737480768374897
:10D910000068354908603548076035480068401C94
:10D9200033490860FEF7B4F800BF3248006885420A
:10D930003BD300BF2C480068006808B9012000E014
:10D94000002020B14FF0FF302A4908602CE0264823
:10D950000068C068C4686668B54202D2254806609F
:10D9600022E0201DFEF7D7FBA06A18B104F11800D1
:10D97000FEF7D1FB2049E06A0968884202D91E49B6
:10D98000E06A0860E16A01EB81011C4A02EB810058
:10D99000211DFEF718FC1A49E06A0968C96A884225
:10D9A000C8D34FF00108C5E700BF15480068C06A3A
:10D9B00000EB8000114951F82000012801D94FF0F7
:10D9C00001081048006808B14FF0010805E0FFE7C2
:10D9D0000D480068401C0C4908604046BDE8F081D5
:10D9E000500000202C0000201C00002020000020FF
:10D9F000400000204800002030000020B405002036
:10DA0000180000203C000020380000202DE9F041E3
:10DA10000746884614461D46FEF7E2FB214800688B
:10DA200090F86000022818D01E49096801F15C00D6
:10DA3000C96DB943016001201A49096881F8600085
:10DA40005DB101212846FDF7E3FB4FF080501649F8
:10DA50000860BFF34F8FBFF36F8FFEF7EBFBFEF74E
:10DA6000BFFB1CB10F480068C06D20600D48006806
:10DA700090F86000022801D0002608E009490968F2
:10DA800001F15C00C96D21EA080101600126002056
:10DA90000449096881F86000FEF7CCFB3046BDE818
:10DAA000F08100001800002004ED00E070B505468C
:10DAB0002C460026002D43D022480068844201D124
:10DAC000012000E0002050B900BF502080F31188F1
:10DAD000BFF34F8FBFF36F8F00BF00BFFEE7606DD6
:10DAE00050B900BF502080F31188BFF34F8FBFF3B0
:10DAF0006F8F00BF00BFFEE7606D401E6065216D47
:10DB0000E06A88421CD0606DD0B9201DFEF703FB8F
:10DB1000206DE062E06AC0F13800A0610A49E06A65
:10DB20000968884202D90849E06A0860E16A01EBA5
:10DB30008101064A02EB8100211DFEF744FB01260C
:10DB4000304670BD1800002030000020B4050020D1
:10DB500070B505462C460026002D42D02249E06AC9
:10DB60000968C96A884235D2A06900F0004028B926
:10DB70001D480068C06AC0F13800A061E16A01EB8D
:10DB800081011A4A02EB81016069884201D10120BA
:10DB900000E00020C0B1201DFEF7BDFA1248006869
:10DBA000C06AE0621249E06A0968884202D91049F5
:10DBB000E06A0860E16A01EB81010C4A02EB810036
:10DBC000211DFEF700FB03E007480068C06AE06221
:10DBD000012606E00449206D0968C96A884200D21E
:10DBE0000126304670BD000018000020B40500205A
:10DBF0003000002070B50646F068C46854B900BF14
:10DC0000502080F31188BFF34F8FBFF36F8F00BF99
:10DC100000BFFEE704F11800FEF77DFA1548006822
:10DC2000A0B9201DFEF777FA1349E06A0968884217
:10DC300002D91149E06A0860E16A01EB81010F4AEB
:10DC400002EB8100211DFEF7BEFA04E004F1180189
:10DC50000B48FEF7B8FA0B49E06A0968C96A8842BE
:10DC600004D9012501200849086000E00025284664
:10DC700070BD00005000002030000020B4050020DE
:10DC80003C0A0020180000203C00002070B5002451
:10DC900000263648006850B900BF502080F3118834
:10DCA000BFF34F8FBFF36F8F00BF00BFFEE7FEF7DC
:10DCB00097FA2E480068401E2C4908600846006804
:10DCC00000284ED12A48006800284AD023E029487D
:10DCD000C068C46804F11800FEF71DFA201DFEF7A5
:10DCE0001AFA2549E06A0968884202D92249E06A9D
:10DCF0000860E16A01EB8101204A02EB8100211DED
:10DD0000FEF761FA1E49E06A0968C96A884202D3CF
:10DD100001201C4908601748006808B9012000E08C
:10DD200000200028D3D00CB1FDF7B2FE16480568DC
:10DD300065B100BFFFF7C8FD10B1012011490860AF
:10DD40006D1E002DF6D100200F4908600D480068B7
:10DD500038B1012630070D490860BFF34F8FBFF37C
:10DD60006F8FFEF767FA304670BD0000500000204C
:10DD7000280000203C0A002030000020B4050020CC
:10DD8000180000203C0000203800002004ED00E0D6
:10DD900010B586B00024FDF7D5FA16480068D0B15A
:10DDA00000200590049003AA04A905A8FEF7D4F961
:10DDB0000222DDE904100023CDE9002102900EA12A
:10DDC0000F48039AFFF7B6FB0E4908600846006843
:10DDD00000B1012400BF54B900BF502080F3118866
:10DDE000BFF34F8FBFF36F8F00BF00BFFEE720462A
:10DDF00006B010BD64000020546D7220537663009D
:10DE0000D5BB0008680000202DE9FF4704460D46F9
:10DE100016461F46DDF830804FF0000954B900BFA8
:10DE2000502080F31188BFF34F8FBFF36F8F00BF77
:10DE300000BFFEE71448006810B3009501960294F5
:10DE4000062D15DAFFF720FD022808D100234246EF
:10DE500069460D480068FEF761FF814610E0002327
:10DE60001A46694608480068FEF758FF814607E0F1
:10DE700000233A46694604480068FFF723F88146C4
:10DE8000484604B0BDE8F0876400002081F00041FE
:10DE9000704780F00040704721F00041704720F04B
:10DEA0000040704721F00042A2F16052B2F5801F9D
:10DEB00001F0004328BFD2F17F6C0BD95FEA001C50
:10DEC00043EAC20242EB507018BF704728BF20F0EF
:10DED00001007047B2F5801FBCBF184670474FEA7B
:10DEE000410C1CF5001F02D2084600F01FBE70B5A1
:10DEF00000F0C0FB00000089FFF7F6BF4FF00040C4
:10DF0000A0F580007047000010B591EA030F48BFEC
:10DF100083F0004300F14C84841A71EB030C05D2AA
:10DF2000121943EB0C03001B61EB0C01DFF824E139
:10DF30004FEA1154A4EB135C1EEA430F18BF9EEA8C
:10DF4000445F73D023EA0E03DCF1200E21EA045172
:10DF500043F4801332D322FA0CFE10EB0E0023FAA6
:10DF60000CFE41EB0E01CCF1200E03FA0EFE10EB7D
:10DF70000E0051F10001B1F5801FCCF1200E32D21C
:10DF800001EB045112FA0EF2BDE8104058BF704781
:10DF9000401C38BF5FEA420218BF7047002814BF18
:10DFA00020F0010041F100014FEA410313F5001F89
:10DFB00038BF7047A1F1C04100F0AABB012A43EB72
:10DFC0000302ACF1200CDCF11F0E32BF4FF0000E4B
:10DFD00023FA0CF310EB030041EB0451B4EB115F97
:10DFE000D0D0A1EB045101F5801149085FEA30005F
:10DFF00001EB04510ED350F1000038BF12FA0EFEAF
:10E0000008D1BDE81040C9E7401C38BF5FEA4202B2
:10E01000CAD1C3E7BDE810404FEA410313F5001F22
:10E0200038BF7047A1F1C04100F072BB9EEA445F67
:10E0300008D011EA5E0FBDE8104004BF01F00041B6
:10E0400000207047BDE8104070B500F013FB00BF22
:10E0500064FBBE3E0000E0FF491058BFC1F14041E3
:10E060005B1058BFC3F140438B42EFF30080704711
:10E070002DE9C04130B4DFF8A0C23CEA111418BF4A
:10E080003CEA131400F0EC8081EA03051CEA111449
:10E0900044EAD57418BF1CEA131500F0C780A4EB3E
:10E0A00005044FF0004545EAC12145EAC32341EA92
:10E0B000505143EA525304F17F74994204F50034FD
:10E0C0004FEAC0204FEAC22208BF904200F09C8075
:10E0D0004FEA13650FF24016765D4FEA134506FBD3
:10E0E00005F7C7F1807706FB07F74FEAD737A7FB9D
:10E0F00003687642C8F58038A7FB06CE38BFA8F182
:10E10000010807FB08E64FF0000EA6FB028CE6FBB9
:10E1100003CEDCF1000CCEF1004E38BFAEF1010EA3
:10E12000A6FB0C584FF000074FF00005E6FB0E87EA
:10E13000A1FB08C6A0FB07CE16EB0E0645F10005B5
:10E14000E1FB076515F1E04E7EBFA4F580345FEA80
:10E1500046066D4116F1800745F100054FEA172785
:10E160004FEA066647EA0567A6F1DE46B6F1805F2C
:10E170004FEA15251FD9384624F0010C05EBC47170
:10E18000BCF1FE6F01EB0C1102D8F0BCBDE80081C0
:10E1900024425CBF01F5801E9EEAC47F02D4F0BC1D
:10E1A000BDE80081244238D4F0BCA1F1C041BDE8F3
:10E1B000004100F0ADBA4FEAD22242EA43524FEAA0
:10E1C000D323A7FB02864FEAD02040EA415007FB49
:10E1D00003661EEA0E0F4FEAD12105FB026658BF07
:10E1E000A6EB0056B6EB00564FEA520E4EEAC37E3F
:10E1F00018EB0E0E56EB530EBDD518EB02085E4120
:10E200007F1C55F10005B6E74FF480154FF000076D
:10E210004FF000064FF00008ADE7F0BC4FF00000F3
:10E2200001F1C04101F00041BDE8008111EA0C1F7D
:10E230000CEA131500D00CE013EA0C1F00F0258047
:10E240004FF00000F0BC81EA030101F00041BDE89D
:10E250000081F0BCBDE8004181EA030100F058BA3A
:10E26000F0BCBDE8004170B500F004FA097EFC3E48
:10E2700000F007B881EA03014FF0000001F000410F
:10E28000704781EA030100F043BAF0BCBDE80041E9
:10E290004FF0000021497047FFFDFBF9F7F5F4F25C
:10E2A000F0EEEDEBE9E8E6E4E3E1E0DEDDDBDAD831
:10E2B000D7D5D4D3D1D0CFCDCCCBCAC8C7C6C5C48F
:10E2C000C2C1C0BFBEBDBCBBBAB9B8B7B6B5B4B3A6
:10E2D000B2B1B0AFAEADACABAAA9A8A8A7A6A5A491
:10E2E000A3A3A2A1A09F9F9E9D9C9C9B9A99999855
:10E2F0009797969595949393929191908F8F8E8EF8
:10E300008D8C8C8B8B8A8989888887878685858484
:10E3100084838382828181800000FF070000F87F70
:10E3200051EA030C17D41CF5801F58BFBCF5801FA1
:10E3300000F10680994218BF704708BF90427047AD
:10E3400007D711F5801F58BF13F5801F19D49942C4
:10E350007047894270471CF5801F08D5BCF5801FA7
:10E36000F7D58B4218BF704708BF824270474FF401
:10E37000001C1CEB410F38BF1CEB430F01D28B423A
:10E38000704770B500F076F9922449004FF00051C3
:10E390004FF08053FFF760BE4FEA41034FEA5353FB
:10E3A000A3F58063D3F11E03C8BFD3F1210C0CDDAC
:10E3B0004FF0004242EAC12242EA505232FA03FCD4
:10E3C0008CEAE17CACEBE1707047102BC4BF0020FD
:10E3D000704703F5787CBCF1FF3F04D06FF000423A
:10E3E00082EA2100704770B500F044F94992248018
:10E3F00000207047F2E700004FEA1153A3F5806355
:10E40000D3F11E03A8BFD3F1200C08DB4FF000426C
:10E4100042EAC12252EA505232FA03F070470942EE
:10E420000BD4102BC4BF0020704703F5787CBCF1DF
:10E43000FF3F05D04FF0FF3070474FF000007047AE
:10E4400070B500F017F900BF499224800020704792
:10E45000F0E710F0004248BF4042B0FA80F310FAF3
:10E4600003F10AD0C3F11D0303F580634FEA415065
:10E4700002EB035202EBD12170474FF000007047CE
:10E48000B0FA80F310FA03F10AD0C3F11D0303F5CB
:10E4900080634FEA41504FEA035202EBD1217047AB
:10E4A0004FF000007047000051EA030C17D41CF530
:10E4B000801F58BFBCF5801F00F10680994218BF2D
:10E4C000704708BF9042704707D711F5801F58BFAB
:10E4D00013F5801F19D499427047894270471CF583
:10E4E000801F08D5BCF5801FF7D58B4218BF704739
:10E4F00008BF824270474FF4001C1CEB410F38BF2D
:10E500001CEB430F01D28B42704770B500F0B2F89C
:10E51000922449004FF000514FF08053FFF79CBD0B
:10E52000DFF848C170B51CEA111E1EBF1CEA1315A6
:10E530009EEA0C0F95EA0C0F00F06F8081EA03044D
:10E5400023EA4C134EEAD47E21EA4C1141F48011A7
:10E5500043F48013AE44A1FB024CA0FB0365AEF173
:10E560007F7E361955EB0C05A1FB034C4CF10003E3
:10E57000A0FB021C16EB0C06654153F10003094297
:10E5800018BF46F0010613F4007F0BD14FEA0331A8
:10E590004FEA0530340341EA155140EA16506FF056
:10E5A00003020AE04FEAC3214FEAC520F40241EA20
:10E5B000555140EA56506FF0020202EB2E4201EB39
:10E5C000025585EACE710AD05FEA440C18BF24F0E8
:10E5D000004450F1000041F1000120EAD47040F203
:10E5E000FE7C624500D270BDA84214BF4FF080444B
:10E5F0004FF04044002E08BF0024BEF1806FA8BF3A
:10E60000A1F1C041BDE8704080F282804FF000006F
:10E6100001F1C04101F0004170479EEA0C0F0CEA85
:10E62000131518BF95EA0C0F06D04FF0000081EAD1
:10E63000030E0EF0004170BD00F01CF88900013E91
:10E6400000F007B800F009B84FEA430C5FEA5C5CE1
:10E6500008D081EA030100F05BB84FEA410C5FEAA1
:10E660005C5CF6D14FF00000014970470000FF07E5
:10E670000000F87F0EF1020E2EF0030E5EF8046B20
:10E68000364205D4012A43EB030515F5001F12D8C5
:10E69000012841EB010C1CF5001F0CD80ED14FEAEC
:10E6A000D17C15F5001F0CEB4C0C0CF1020C08BFD3
:10E6B0004CEBD37C04E04FF0080C01E04FEAD37C34
:10E6C0000CEB4C0526FA05F606F00706B6F1040C2D
:10E6D00006D20EEB860CBDE870404CF0010C604792
:10E6E000DFE80CF0090B02024FF000414FF0000090
:10E6F000A1F5002170BD19461046012851EB010417
:10E7000018BFD4F5001484BF002001F0004170BD93
:10E710000808A0F500114FEA3101704753EA010CD7
:10E7200017D41CF5801F58BFBCF5801F00F1068070
:10E730008B4218BF704708BF8242704707D713F556
:10E74000801F58BF11F5801F19D48B4270479B4220
:10E7500070471CF5801F08D5BCF5801FF7D599427E
:10E7600018BF704708BF904270474FF4001C1CEB65
:10E77000430F38BF1CEB410F01D2994270470FB4D1
:10E780000CBC03BCFFF7C1BE91EA030F10B581F0CA
:10E7900000413FF5C1AB83F0004300F009B8000031
:10E7A00010B591EA030F48BF83F000433FF5B4ABC7
:10E7B000841A71EB030C07D212198CF0004C43EB56
:10E7C0000C03001B61EB0C01DFF8A4E14FEA1154CC
:10E7D000A4EB135C1EEA430F18BF9EEA445F00F0EF
:10E7E000B08023EA6E03524221EA0451C3EB6E0368
:10E7F00038BF5B1EDCF1200E25D322FA0CFE10EB95
:10E800000E0043FA0CFE41EB0E01CCF1200E03FA90
:10E810000EFE10EB0E0051F10001CCF1200E29D4B8
:10E8200012FA0EF201EB0451BDE8104058BF7047D8
:10E83000401C1CBFB2F1004F704700280CBF491CA0
:10E8400020F00100704712EB020E43EB030218BFE9
:10E850004FF0010E4EEA4202ACF1200CDCF11E0E2C
:10E8600054D943FA0CFE10EB0E0051F1FF31CCF1FC
:10E870001E0ED5D50EF1010E12FA0EFE404141EBEF
:10E88000010101EB445C5FEA5C5C10D910EBDE70C7
:10E8900001EB045138BFBEF1004FBDE8104018BF76
:10E8A000704700280CBF491C20F00100704730D28F
:10E8B0004FEAD42C11F5001124F400641BD0B1FAF6
:10E8C00081F20B3AA41AA41ED2F12003914030FA2F
:10E8D00003F31943904001EBCC71002C01EB045180
:10E8E000BDE81040A8BF704701F1C0414FF00000E3
:10E8F00001F000417047B0FA80F310FA03F100D143
:10E9000010BDE41A173C4805C90AE4E701EB0451BD
:10E9100010BD491001EB0451BDE810404FEA300032
:10E9200002E04FF0000170474A0008BF0042F8D0F3
:10E93000B2F5001F28BF704701F000414FF0000002
:10E9400070479EEA445F07D011EA5E0FBDE81040B1
:10E9500004BF002100207047BDE8104070B5FFF7EC
:10E9600089FE00BF40DFF63E83F00041104670474D
:10E970000000E0FF43004FEAD30C4FEA3C0C434059
:10E980001FBF40070CF1605113F0FE4F70471CF0A1
:10E99000006F03D100200CF0004170470CF00043E1
:10E9A00043EA507010B540EACC0000F074F800BFA4
:10E9B000000000924FEA0001FFF7AABE4FF00041AD
:10E9C0004FF00000A1F500217047000000EE100A92
:10E9D00000EE901AB4EE600AF1EE10FA78BF7047BC
:10E9E00000F00DB810B5FFF7F1FFEFF3008020F055
:10E9F000104038BF40F0004080F3008810BDBDE8F3
:10EA0000104010B500F047F80000000900F007B80A
:10EA10004FF0404010F1004FEFF30080704740107E
:10EA200058BFC0F14040491058BFC1F14041814238
:10EA3000EFF3008070474FF07E5209E011F0004282
:10EA400004D54042C1F1000138BF491E42F07E5258
:10EA50000B0002F1706212BF20235FEA00017047D1
:10EA6000B1FA81FCA3EB0C0301FA0CF120FA03FCD0
:10EA700002EBC352C3F1200341EA0C0110FA03FC7C
:10EA80005CEA416C42EB112018BF5FF0806C28BF3C
:10EA900020F0010070470EF1020E2EF0030E5EF81A
:10EAA000044B244204D44FEA4102B2F17F4F11D803
:10EAB0004FEA4003B3F17F4F0CD80ED14FEAD07C20
:10EAC000B2F17F4F0CEB4C0C0CF1020C08BF4CEB7D
:10EAD000D17C04E04FF0080C01E04FEAD17C0CEB54
:10EAE0004C0324FA03F404F00704B4F1040C06D236
:10EAF0000EEB840CBDE810404CF0010C6047DFE8E1
:10EB00000CF0070802024FF00040A0F5800010BD95
:10EB10000846420018BFD2F1807288BF00F0004062
:10EB200010BD4FF04070E1EE100A7047FF2141EA3E
:10EB3000D050C0057047000030ED00080000000014
:10EB400000000000000000000000000000020000C3
:10EB50001800000000000000000000000006101671
:10EB6000000610160000000000000000010203046F
:10EB7000060708090000000001020304010000006C
:10EB800000000240100000000000024001000000F0
:10EB900000040240100000000008024020000000B5
:10EBA0000008024008000000001802404000000079
:10EBB000001802403C040020000000009A99193E11
:10EBC0000000803F00000000000000000000803FC7
:10EBD0000000803F00000000000000005CED000825
:10EBE0000000000000000000000000000000000025
:10EBF00000040000300000000000000000000000E1
:10EC000044ED0008000000000000000000000000CB
:10EC100000000000000400001800000000000000D8
:10EC20000000000050ED000800000000000000009F
:10EC300000000000000000000004000018000000B8
:10EC400000000000000000003CED00080000000093
:10EC500000000000000000000000000000040000B0
:10EC6000180000000000000000000000000000008C
:10EC70004FBB610567ACDD3F182D4454FB21E93FD4
:10EC80009BF681D20B73EF3F182D4454FB21F93FC3
:10EC9000E2652F227F2B7A3C075C143326A6813C49
:10ECA000BDCBF07A8807703C075C143326A6913CF4
:10ECB000C4EB98999999C9BF711623FEC671BCBF60
:10ECC0006D9A74AFF2B0B3BF9AFDDE522DDEADBFC8
:10ECD0002F6C6A2C44B4A2BF0D5555555555D53FE0
:10ECE000FF8300922449C23F6E204CC5CD45B73FFB
:10ECF000513DD0A0660DB13FEB0D76244B7BA93F73
:10ED000011DA22E33AAD903F00000000000000005D
:10ED1000000000006E83F9A22915444ED15727FC4C
:10ED2000C0DD34F5999562DB4190433CAB6351FE05
:10ED300064656661756C745461736B0072656D6FA8
:10ED400074650000617474695F6573746900000024
:10ED500067696D62616C5F6374726C005461736BA0
:10ED60005F496E697400000088ED00080000002013
:10ED70008C010000C4010008F0ED00088C010020A7
:10ED8000DC7B000020020008C132104201037D2418
:10ED9000F41AAA0101180530022B073D12013C0AA2
:10EDA0000202083A0908214B803F048169104B8018
:10EDB000BF04600F2041CDCC2C4066663E41C3F5B8
:10EDC00040411A20081F80BFDB0FC940080A1C3EC3
:10EDD000401AA02429040F1120400267043B401967
:10EDE00024437A442CD7A3303406003FE17A943F81
:040000050800018965
:00000001FF
